:020000040800F2
:1000000060CB0024993000086B9704088530000805
:1000100085300008853000088530000800000000A9
:10002000000000000000000000000000F5300008A3
:100030008530000800000000C133000809B700083F
:1000400079340008793400087934000879340008DC
:1000500079340008793400087934000879340008CC
:1000600079340008793400087934000879340008BC
:1000700079340008793400087934000879340008AC
:10008000793400087934000879340008793400089C
:10009000793400087934000879340008793400088C
:1000A000793400087934000879340008793400087C
:1000B000793400087934000879340008793400086C
:1000C000793400087934000879340008793400085C
:1000D000793400087934000879340008793400084C
:1000E000793400087934000879340008793400083C
:1000F000793400087934000879340008793400082C
:10010000793400087934000879340008793400081B
:10011000793400087934000879340008793400080B
:1001200079340008793400087934000879340008FB
:1001300079340008793400087934000879340008EB
:1001400079340008793400087934000879340008DB
:1001500079340008793400087934000879340008CB
:1001600079340008793400087934000879340008BB
:1001700079340008793400087934000879340008AB
:10018000793400087934000879340008793400089B
:10019000793400087934000879340008793400088B
:1001A000793400087934000879340008793400087B
:1001B000793400087934000879340008793400086B
:1001C000793400087934000879340008793400085B
:1001D000793400087934000879340008793400084B
:1001E000793400087934000879340008793400083B
:1001F000793400087934000879340008793400082B
:10020000793400087934000879340008793400081A
:10021000793400087934000879340008793400080A
:0802200079340008793400086C
:100228009FED0B7B06EE100A9FED0B5BB7EEC66ADF
:1002380026EE077BBCEEC77BB8EE474BA4EE456BBA
:10024800FCEEC67B17EE101A17EE900A704700BF37
:10025800000000000000F03D000000000000F04138
:1002680080F0004002E000BF81F0004142001FBF63
:100278005FEA410392EA030F7FEA226C7FEA236C6C
:100288006AD04FEA1262D2EB1363C1BFD218414061
:1002980048404140B8BF5B42192B88BF704710F0F7
:1002A800004F40F4000020F07F4018BF404211F09A
:1002B800004F41F4000121F07F4118BF494292EA02
:1002C800030F3FD0A2F1010241FA03FC10EB0C002E
:1002D800C3F1200301FA03F100F0004302D54942BB
:1002E80060EB4000B0F5000F13D3B0F1807F06D368
:1002F80040084FEA310102F10102FE2A51D2B1F160
:10030800004F40EBC25008BF20F0010040EA030054
:100318007047490040EB0000013A28BFB0F5000FD4
:10032800EDD2B0FA80FCACF1080CB2EB0C0200FA8A
:100338000CF0AABF00EBC25052421843BCBFD040D9
:100348001843704792F0000F81F4000106BF80F453
:1003580000000132013BB5E74FEA41037FEA226C16
:1003680018BF7FEA236C21D092EA030F04D092F0E1
:10037800000F08BF0846704790EA010F1CBF002015
:10038800704712F07F4F04D1400028BF40F0004072
:10039800704712F100723CBF00F50000704700F092
:1003A800004343F0FE4040F4000070477FEA2262B9
:1003B80016BF08467FEA23630146420206BF5FEA8A
:1003C800412390EA010F40F4800070474FF000038A
:1003D80004E000BF10F0004348BF40425FEA000C51
:1003E80008BF704743F0964301464FF000001CE0F9
:1003F80050EA010208BF70474FF000030AE000BF4F
:1004080050EA010208BF704711F0004302D540428C
:1004180061EB41015FEA010C02BF844601460020FE
:1004280043F0B64308BFA3F18053A3F50003BCFA19
:100438008CF2083AA3EBC25310DB01FA02FC6344C6
:1004480000FA02FCC2F12002BCF1004F20FA02F2CD
:1004580043EB020008BF20F00100704702F12002C0
:1004680001FA02FCC2F1200250EA4C0021FA02F221
:1004780043EB020008BF20EADC7070477BB972B911
:100488000029BEBF00204FF0004106E008BF002849
:100498001CBF6FF000414FF0FF3000F057B8ADF1CE
:1004A800080C6DE904CE002909DB002B1ADB00F0EB
:1004B80069F8DDF804E0DDE9022304B07047404242
:1004C80061EB4101002B1BDB00F05CF8DDF804E078
:1004D800DDE9022304B0404261EB4101524263EB83
:1004E80043037047524263EB430300F04BF8DDF8D7
:1004F80004E0DDE9022304B0404261EB41017047AA
:10050800524263EB430300F03DF8DDF804E0DDE917
:10051800022304B0524263EB4303704753B94AB90C
:10052800002908BF00281CBF4FF0FF314FF0FF30F3
:1005380000F00CB8ADF1080C6DE904CE00F022F81B
:10054800DDF804E0DDE9022304B07047704700BF1E
:1005580010F8012B11F8013B012A28BF9A42F7D065
:10056800D01A7047034611F8012B03F8012B002A13
:10057800F9D17047034613F8012B002AFBD1181A4A
:10058800013870472DE9F0478C468E46089E15467F
:1005980004461946002B40F0D080724547D9B2FA7C
:1005A80082F74FB1C7F120030EFA07FC20FA03F3D4
:1005B800BD4043EA0C0CBC404FEA154EA8B2BCFB48
:1005C800FEF8230C0EFB18CC08FB00F943EA0C4399
:1005D800994528D9EB1808F1FF3204D2994502D978
:1005E800A8F102022B44A3EB0903A4B2B3FBFEFC5F
:1005F8000EFB1C330CFB00F044EA0344A04214D960
:100608002C190CF1FF3304D2A04202D9ACF1020339
:100618002C44241A43EA02401EB1FC4000233460F3
:100628007360BDE8F0874246DDE76346F1E7002ADC
:1006380079D0B2FA82F3002B3FD01946C1F12003DA
:1006480002FA01F52EFA03F20EFA01FE20FA03F37C
:1006580043EA0E034FEA154E00FA01F4B2FBFEFC22
:10066800AFB20EFB1C201A0C0CFB07F842EA004242
:1006780090455AD9AA180CF1FF3004D2904502D9F6
:10068800ACF102002A44A2EB08029BB2B2FBFEFCCA
:100698000EFB1C220CFB07F743EA02439F4246D994
:1006A800EB180CF1FF3204D29F4202D9ACF10202DE
:1006B8002B44DB1B42EA004202E0AEEB02030122BC
:1006C8004FEA154EAFB2B3FBFEFC200C0EFB1C33F9
:1006D8000CFB07F840EA034398452AD9EB180CF1BC
:1006E800FF3004D2984502D9ACF102002B44A3EBA9
:1006F8000803A4B2B3FBFEFC0EFB1C330CFB07F78C
:1007080044EA0344A74216D92C190CF1FF3304D24A
:10071800A74202D9ACF102032C44E41B43EA00408F
:100728000F46114678E71F2188E76046ABE7624627
:10073800BFE76046DBE76346EFE7734506D916B9BE
:10074800002108466DE7C6E9000EF9E7B3FA83F71A
:1007580087B9734501D3824207D8841A6EEB030325
:1007680001209C461EB900215BE73846FAE7C6E936
:10077800004CF8E7C7F1200CBB4022FA0CF51D43EA
:1007880020FA0CF12EFA0CF30EFA07FE41EA0E01DC
:100798004FEA154900FA07F4B3FBF9F81FFA85FE8A
:1007A80009FB18300B0C08FB0EFA43EA00439A4584
:1007B80002FA07F240D9EB1808F1FF3004D29A4543
:1007C80002D9A8F102002B44A3EB0A0389B2B3FBB8
:1007D800F9F809FB183308FB0EFE41EA03418E4580
:1007E8002CD9691808F1FF3304D28E4502D9A8F133
:1007F8000203294443EA0040A0FB0298A1EB0E0142
:100808004145CE46434602D306D14C4504D2B9EB06
:10081800020E68EB05030138002EA4D0B4EB0E02DB
:1008280061EB030101FA0CFC22FA07F34CEA03031B
:10083800F940C6E9003196E74046C5E74346D9E79F
:10084800073222F007022DE9F04FFF3285B01F462C
:1008580000F15803044622F07F020E4604217F2A45
:10086800A2F1800B06F18008C0E91633129B4FF005
:1008780000002174A381119BA060A373E0739FED16
:10088800247BDDE90EA9C4E9060084ED087B05D8C0
:1008980080F31188BFF36F8F084602DFB518204632
:1008A800294602F095F90730109B314620F00700E1
:1008B8002D1AC4F8880020462A46C4E9208BCDE9C1
:1008C8000193CDF800A03B4602F09AFC0023C4F83F
:1008D80074906365109BC4E91B7AA367EFF31182D8
:1008E800102383F31288BFF36F8F0B4B596A5C6236
:1008F800E16782F31188BFF36F8F9B680BB1D3F860
:100908008C302846C4F88C3005B0BDE8F08F00BFA5
:100918000000000000000000243F00240000000048
:1009280008B513F013FD4EF067FFD0B1643007EE41
:10093800900A9FED0D5BB8EE676B86EE057BB7EE10
:10094800C77BB4EE477AF1EE10FA77BF17EE103A8C
:10095800074823F0030040F0020078BFA0F1FF40F1
:1009680008BD0448FCE700BF0000000000408F40BD
:1009780002004000020080802DE9F0412DED028B3D
:1009880090F8A530B0EE408A86B004461BB9F7EE61
:10099800007A37EEC08AD4F884202F4B9A4212D1BD
:1009A800B7EEC87A04F184009FED296BB4EEC67BDC
:1009B800F1EE10FACCBF0121002112F063FE0120F4
:1009C80084ED268A05E0B4F89C30B3F5807F05D124
:1009D800002006B0BDEC028BBDE8F08104F15008A0
:1009E80040462BF00BFF0028F2D0DFED1C7A94F87C
:1009F800806068EE277A94F89C20276E206DFCEEC4
:100A0800E77ACDED037A9DF80C306EB18DF815308C
:100A180002238DF8142000210093012205ABB8476A
:100A2800404659F0C6F8CAE7012531468DF813202B
:100A38008DF814302A460DF113030095B847009538
:100A480005AB276E32462946206DE8E7AFF30080F4
:100A5800AE47E17A14AEEF3FC817070800007F439E
:100A68002DE9F04704460846904699462DED068B39
:100A780086B0616006219DF850609DF8547015F0AD
:100A88003DFDA060057C15F0010502D0824816F0F6
:100A9800DFFE9DF8583009FB08F00DF1100A2673A7
:100AA80084F82A307D309DF85C3084F828307E2325
:100AB80090FBF3F0C0010430C4E90489606253F08C
:100AC800B0FF06227549A561C4E90705204666F00E
:100AD80027FA022251462046ADF8108066F020FA27
:100AE800022251462046ADF8109066F019FAF62316
:100AF800032202A92046ADF808308DF80A5066F0A6
:100B08000FFA731EDBB2082B06D840F2551828FAE4
:100B180003F818F0010801D16148B8E7052E0AD09A
:100B2800072E07D0032E7FD1012384F829304FF0F8
:100B3800000802E0454684F82950B7EE088B0025E6
:100B4800B0EE089BB0EE0CAB45F34F13B1EE0C5B67
:100B5800C3EB032307EE103AC5F38203B8EEC77B55
:100B6800C3EB032337EE087B87EE096B07EE103AD9
:100B780005F00303C3EB0323FDEEC67BCDED017A3D
:100B8800B8EEC77B9DF8041037EE0A7B87EE056B3D
:100B980007EE103AFDEEC67BCDED017AB8EEC77BC5
:100BA8009DF8042037EE087B87EE096BFDEEC67BC7
:100BB800CDED017A9DF80430B8F1000F5BD08DF8C7
:100BC80010308DF811108DF812200135032251468E
:100BD800204666F0A5F9802DB6D1D7B1314D03A9CD
:100BE80020462A88AB78ADF80C2003228B7066F07B
:100BF80097F90B222C49204666F092F9D5F80300A4
:100C0800EB7905220490514620468AF8043066F0B4
:100C180087F9204666F072F9A06966F093F906B084
:100C2800BDEC068BBDE8F087092E84F829507FF4C7
:100C38007EAF9FED159B9FED168B07EE905AFF3503
:100C480003225146B8EEE77B204637EE097B87EE54
:100C5800086BFDEEC67BCDED017A9DF804308DF86A
:100C680010308DF811308DF8123066F059F9B5F55D
:100C7800FF4FE2D1B1E78DF810108DF811208DF8F3
:100C88001230A2E7AFF300800000000000C04F4020
:100C98000000000000C05F4040E90708A6CC070834
:100CA80085E00708C28C06089ACC070800000000F7
:100CB80010EE103A33F00042F0EE407A02D10120F3
:100CC80046F0DCBF002B01DA46F0E6BFB3F1FF4F78
:100CD80002DB30EE000A7047B3F5000FB8BF9FED96
:100CE8005E7A5E48BEBF60EE077A6FF0180117EEB5
:100CF800903A4FEAE352C3F316031844A8BF002101
:100D08007F3A0A4400F4000181F07E51194300EE55
:100D1800101A534902EBD05203F10F00F7EE007A94
:100D2800014030EE670A99BBB5EE400AF1EE10FAC1
:100D38000FD1002A00F0898007EE902A9FED490A1A
:100D48009FED497AF8EEE77A27EE800A07EE870AE0
:100D580070479FED3F7BF7EEC77BB6EE007A07EE54
:100D6800C07A60EE007A27EE277A12B930EE470A89
:100D7800704707EE902ADFED3B6AF8EEE77A07EE58
:100D8800E67A37EE400A9FED387A17EE870A704701
:100D9800F0EE007A70EE277A9FED345ADFED344A90
:100DA800344980EE276A1944C3F5571303F52273B3
:100DB8000B43002B07EE902A66EE065AF8EEE76A18
:100DC80025EEA57ADFED2C7A07EE275ADFED2B7A90
:100DD80045EE077A9FED2A5A07EE875ADFED297A02
:100DE80047EE274ADFED287A44EE877A67EE877A5E
:100DF80045EE257A1ADDB6EE007A20EE077A27EE60
:100E0800007A77EE877A67EE867A12B937EE677AD4
:100E1800ACE79FED146A46EE867A37EE677A37EECE
:100E2800400ADFED117A16EEA70A704770EE677A6E
:100E380067EE867A12B930EE670A70479FED097A35
:100E480046EEC77A37EEC00AEBE79FED100A704707
:100E5800555555555555D53F0000004C20FB4A00C7
:100E6800F0FF7F00D1F717378071313F25333A3EC5
:100E7800298E633E305CCFFF9788173E2549923E06
:100E8800ABAA2A3F4FD01C3ECDCCCC3E0000000080
:100E9800F8B510EE903A33F000472DED028B10EEC6
:100EA800101A0DD181F48001490011F5000F40F2AC
:100EB800A28270EE207ABDEC028BB0EE670AF8BD14
:100EC80021F00046B6F1FF4F084602D8B7F1FF4FB0
:100ED80008D9B1F17E5FECD183F480035B0013F590
:100EE800000FE4E7002925DAB7F1974F80F08C82EC
:100EF800B7F17E5F39D3FC15C4F1960447FA04F2C2
:100F080002FA04F4BC4229D102F00102C2F1020241
:100F1800B7F17E5F2AD1002B80F27382B5EE400ACA
:100F2800F1EE10FA1CD1C80FBDEC028BBDE8F840F9
:100F380046F0A4BEB7F1FF4F10D1B6F17E5F00F0C6
:100F48005A8205D9DFEDD47A002B60FEA77AB2E782
:100F5800002B80F25382F1EE607AACE70022D7E7EB
:100F6800B7EE007AC7EE007AA5E70022B3F1804F0A
:100F7800344640F04F82B6F1BF4F0CD2B6F1D05F85
:100F880002D960EE007A96E7F0EEC07A5EBB012ADD
:100F980040FE277A8FE721F04045B5F17E5FF0EEFD
:100FA800C07A17D1002BBCBFB7EE007AC7EE277AFC
:100FB800002980DAA6F17E56164305D1BDEC028BD6
:100FC800BDE8F84046F068BE012A7FF474AFF1EE40
:100FD800677A70E73EB9002BD9DA0029A4D0531EEE
:100FE80058425841A0E7CD0F013D52EA0500E5D02F
:100FF800B7F19A4F6CD9A9498E4208D8002B0BDA61
:101008000020BDEC028BBDE8F84046F029BEA4499B
:101018008E4208D9002BF3DC0020BDEC028BBDE822
:10102800F84046F00FBE9FED9A5BB7EE007A77EE78
:10103800C77AB7EEC55BB5EE007A07EEC75AB6EECB
:10104800007A05EE677A67EEA76A9FED966A27EE43
:10105800267ADFED956A27EE267ADFED946A17EE99
:10106800A67A27EE866A76EE077A17EE901A6FF35D
:101078000B0106EE901A36EEC66A77EE467AB7EEA0
:10108800007A6FF30B03013ABFEE008A2A4308FE89
:10109800078A07EE103A30EEC76A67EEA00A46EEF6
:1010A800260A66EE877A30EEA77A17EE101A00291C
:1010B80021F0004340F3E080B3F1864F40F2CD8049
:1010C800B5EEC08AF1EE10FA4CBF0120002098E777
:1010D80011F0FF4F01BF9FED767A67EE877A6FF0C8
:1010E800170017EE904A4FEAE45118BF00207F39E5
:1010F80001447048C4F31604844244F07E5606DD69
:101108006D48844240F3A7800131A6F5000600240B
:101118006A4800EB8400D0ED005A06EE106A75EEBE
:10112800867AF7EE006AC6EEA74A36EE657A27EEAB
:10113800245A15EE100A6FF30B0006EE900A604869
:1011480000EA660040F0005000F5800000EB4450D3
:1011580007EE900A06EEE77A77EEE57ADFED595A60
:1011680036EE676A65EE057A06EE667A9FED566A90
:1011780047EE865A9FED556A05EEA76ADFED545A89
:1011880046EE275A9FED536A05EEA76ADFED525ADD
:1011980046EE275A27EE247A36EE856A67EEA77A56
:1011A80026EE076A05EEA76A66EEA64AF0EE085A2A
:1011B80074EEA57A77EE867A17EE900A6FF30B0035
:1011C80007EE900A77EEE55A27EE277A75EEE45A8D
:1011D80066EEA76A36EE656A06EE057A9FED3F6A07
:1011E80076EE877A17EE900A6FF30B0007EE900AF7
:1011F80077EEE66A27EE866A37EE667ADFED386ABA
:10120800384867EEA67ADFED386A47EE267A00EBB3
:10121800840090ED007A77EE877A07EE101A33494A
:1012280001EB8401D1ED005A76EE276AB8EEC77A51
:1012380076EEA56A76EE876A16EE901A6FF30B01C2
:1012480006EE901A36EEC77A37EE657A37EE467AAA
:1012580077EEC77A13E701245AE756D1DFED246AFF
:1012680037EE677A70EEA66AF4EEC76AF1EE10FA06
:101278003FF726AF86234CE01E4A93423CD9B5EE91
:10128800C08AF1EE10FA4CBF01200020C5E600BF6D
:10129800E13D55555555D53F00000000F3FF7F3F10
:1012A8000700803F00AAB83F3BAAB83F70A5EC36BC
:1012B8000000804B71C41C00D6B35D00F0550708D0
:1012C80000F0FFDF55326C3E42F1533E05A38B3EE2
:1012D800ABAAAA3EB76DDB3E9A99193F0040763F0C
:1012E800C623F6B8E05507084F38763FE855070893
:1012F8003CAA38330000164307D137EE677AB4EEBC
:10130800E07AF1EE10FAB5DBB9E7B3F17C5F6DD99D
:10131800DB157E3B4FF4000018410844C0F3C75367
:10132800414A7F3B1A41024007EE102AC0F31600DB
:1013380040F40000C3F117031841002977EEC77A7B
:10134800B8BF404237EEA07ADFED386ADFED385A91
:101358009FED386A17EE103A6FF30B0307EE103A59
:1013680077EE677A67EE266A70EEE70ADFED327A83
:1013780027EE277ADFED317A00EEA77AB7EE000A7A
:1013880076EE877A77EEE66A37EE667A67EEA76AD0
:1013980007EE877A16EEA56ADFED295A46EE265A39
:1013A8009FED286A15EEA66ADFED275A46EE265A03
:1013B800B0EE676A05EEE66AF0EE006A67EE865AF6
:1013C80036EE666AC5EE866A36EEC77A77EE677AD3
:1013D80030EE670A10EE103A03EBC053B3F5000F76
:1013E80006DA46F0B3FA60EE087A64E50020A9E769
:1013F80000EE103AF7E7F7EE007A5CE5DFED137AD6
:1014080059E5F0EE407A56E5B7F1FF4F3FF495AD58
:1014180034460222B3F17C5F7FF4BDAD0029FFF6AC
:10142800BAADF1EEC07A46E5000080FF0072313FA8
:101438004CBB31330EEADD358CBEBF351872313FF7
:1014480055B38A38610B363BABAA2A3E0000000030
:1014580010EE102AB2F1FF4FF0EE407A04DB70EE86
:10146800007AB0EE670A70476B4B9A426ADC22F04A
:101478000043B3F17E5F0BD3BFEE007AB4EE470AA8
:10148800F1EE10FA02D1012046F0F8BB46F004BC98
:10149800B3F1645F0CD2B3F14A5F21BF60EE006A1A
:1014A800B6EE007A46EEC77AB0EE670A46F008BA9A
:1014B8005A4B1A449A424DD8B7EE007A77EE876AAB
:1014C80016EE902AD3157F3B002BD5BF36EEC77A90
:1014D80076EEE77A37EEC77A37EE677A87EE266ACE
:1014E8004F49C2F316028A42C9BF42F07C5142F00A
:1014F8007E51C2F500020133C8BF921007EE101AE0
:10150800F7EE007A77EE677AF6EE006A67EEA66A7B
:1015180066EEA76A002A41D1F5EE407AF1EE10FA9C
:101528001DD1002B71D007EE903ADFED3E6AB8EE80
:10153800E77AF0EE467A47EE267ADFED3B6A47EE29
:10154800267A8EE7B2F1B44FB6DBD3159FED376A32
:101558007F3BC5E79FED356A01220023D4E79FED65
:101568002C5BB7EEC55BB7EE007A05EE677A67EEDF
:10157800266A13B977EEE67A73E707EE103ADFEDDD
:10158800295AB8EEC77A07EE256A76EEC66A76EE6D
:10159800E77ADFED256A57EE267A62E7B0EE007A41
:1015A80037EE877ADFED224ADFED225A87EE875A37
:1015B80025EE057A47EE245ADFED1F4A45EE874AA5
:1015C800DFED1E5A44EE875ADFED1D4A45EE874A85
:1015D800DFED1C5A44EE875ADFED1B4A45EE874A79
:1015E800F0EE665A44EE875A65EE855A13B976EEE0
:1015F800E56ABFE707EE103A9FED0A5AB8EEC77AD8
:1016080007EE056A36EE256ABFE7DFED087A28E7B8
:10161800555555555555E53FD613D43EE0096A4111
:10162800F6043500D1F717378071313F000000000C
:101638009788173E4FD01C3E25333A3E298E633E8D
:101648002549923ECDCCCC3EABAA2A3F2DE9F84F96
:101658000B1F884602F00701D408A3EB000903F02A
:1016680007030B3100AF4FEAD90629F007090B44ED
:101678000546814404EBD3048368B9F802B09C4260
:1016880028BF1C461BF0010B16D1EA4688B06A46F3
:101698004A4BCDE90538032342F8103F4FF4C251B5
:1016A8005B46474800F040FED5468BF31188BFF3F0
:1016B8006F8F0423184602DF3146284646F0E7FEBE
:1016C800304435F83030C01A864217D0EA4688B020
:1016D8006A463C4BCDE90538032342F8103F002306
:1016E8004FF4C251364800F01FFE0023D54683F35D
:1016F8001188BFF36F8F0423184602DF314628464E
:1017080046F0C5FE8442824622D026D2344428467A
:10171800224646F061FFB9F802302146284643F0D8
:101728000103A9F8023046F0B2FE261805EBC603FD
:101738005B88DB0708D43146284646F0F1FE32467E
:101748002146284646F031FF2146284646F0A4FEA9
:1017580001221046BD46BDE8F88F06EB000805EBF0
:10176800C802528812F0010225D14146284646F0A7
:101778008EFE50448442ECD82846A4EB0A0A46F070
:10178800CFFE4146284646F082FE824507D23219EE
:10179800284646F021FF2846114646F07DFE42467F
:1017A8003146284646F001FFB9F8023043F00103FC
:1017B800A9F80230CCE70022CBE700BFE05F0708BA
:1017C800C08B0608046007082DE9F84F8A4600AF69
:1017D800002974D004680E1F361BF50826F007068A
:1017E80004EB0608B8F802B01BF0010B16D1E94665
:1017F80088B06A46334BCDE90531032342F8103FE0
:101808004FF4C2515B46304800F08EFDCD468BF355
:101818001188BFF36F8F0423184602DF294620463C
:1018280046F035FE284434F83030C01A854217D0C7
:10183800E94688B06A46254BCDE9053A032342F8C4
:10184800103F00234FF4C2511F4800F06DFD0023E4
:10185800CD4683F31188BFF36F8F0423184602DF48
:10186800B8F802302946204623F00103A8F80230D0
:1018780046F00DFE05EB000804EBC8035B88DA07A9
:1018880008D44146204646F04BFE424629462046AB
:1018980046F08BFEA65BAE1B04EBC6035B88DB073A
:1018A80009D43146204646F03BFE2A4635463146A5
:1018B800204646F07AFE2946204646F0EDFDBD4614
:1018C800BDE8F88F2D600708C08B0608046007087C
:1018D800024808B547F0BDF9002008BD5A6007085E
:1018E8000E4A0346904202D30D4A904211D30D4A44
:1018F80022B1934202D30C4A93420AD30B4A52B103
:101908000B48834234BF01200020934238BF002097
:101918007047012070471046704700BFD4840608FE
:10192800600008080000000000000000000000003F
:10193800000000002DE9F04F9BB004468B4600AF35
:10194800D7F890A0FA637B6349B903784678807822
:1019580000EB830020445E4522D8A0EB040B0AF07C
:10196800010394F80280FB62B8F1000F0CBF4FF03E
:1019780000090AF00109E3783B6313B11AF0020F7A
:1019880017D1B9F1000F14D1FB6B1BB17A6B594613
:10199800204698475D4628466C37BD46BDE8F08F1F
:1019A800451C0BF1010B2846FEF7E4FD01302844E5
:1019B800D1E7CAF3C003FB612378BB629B00BB611C
:1019C80063683B62BB6A04EB8301FB6B002B7ED12F
:1019D8005D468844B9F1000F1DD08B469946A94E43
:1019E8001BF8013B54F82300002808BF3046FEF7D7
:1019F800C1FDD7F8943001304BB1D7F898304B453A
:101A080082BFD7F8943023F8190009F10109C345BA
:101A18000544E5D1D8461AF0050F0AF002034FF045
:101A280000060CBF4FF0020B4FF0010BFB633B6B42
:101A38009E42B0D298F8013008F1020854F823A069
:101A48005046FFF74DFFFA69034602B3B86318F82A
:101A5800021C386A47F0DEF8BB6BC0B1EA468AB0B0
:101A68006A46894B05933B6ACDE906314FF400730A
:101A7800ADF82030854B42F8103F00234FF4125147
:101A88008348023D00F050FCD5460136CFE723B12C
:101A9800FB6A2BB9A5EB0B05F7E7FB6B002BF4D022
:101AA8007848BAF1000F18BF5046FEF763FDD7F823
:101AB800943053B1D7F8983099453FBF431CD7F8B5
:101AC800942022F8193009F101090544DDE7B9F13C
:101AD800000F6CD0434607F148000026102B28BFA2
:101AE8001023BB6397F83890BA6B796266F018FADE
:101AF800796A002201EB08037A620AF002027B612C
:101B080002333A610AF00402FA607A6A396B8A424F
:101B180066D363781AF0020FF96A7B624B440CBFF4
:101B280072080022DBB2002940F0A9801AF0040FE5
:101B380014BF3146002163702046A170E270B96974
:101B48007A6BFB6B9847051EFFF625AFBB6A3146DB
:101B58007A6B07F1580023707B6A84F802806370FF
:101B68003B6BE370FB6B9847061EC0F2C5803A6B6F
:101B7800BB69386B03EB4203ABEB0301D7E90D23D9
:101B8800C91A7B6903EB4000FB6B98470028C0F239
:101B9800B5802E444FF0000807F1480A3518C845AB
:101BA80078D300217A6BFB6B08469847F3E6B8F1C7
:101BB800000F0CD01AF0040F0ED0434607F158005E
:101BC800102B28BF1023BB6397F838608CE7464674
:101BD800C146C7F838808CE74E46C7F8388088E792
:101BE80013F8015C13F8021C54F82500BB60FFF7DA
:101BF80077FE0246F869BB6838B1386AC7E901322E
:101C080047F008F8D7E90132F0B912B3FA6A72B1AD
:101C1800B9F10F0F18D809F1280107F1400009F1AF
:101C2800010201445FFA82F901F8205C0CE0FA68CD
:101C380052B10F2E08D806F1280107F14000721C96
:101C48000E1806F8105CD6B27A6A023301327A624C
:101C58005BE73A69002ADBD10F2EF5D806F1280098
:101C680007F1400C721C02366044F6B200F8101CF2
:101C780007F1680151FA82F202F8105CE4E70021EA
:101C880059E700BF886007088F6007080400000153
:101C9800008B060818F80A3054F823B087F8473044
:101CA800D7F8943033B3D7F89830984522D2D7F87C
:101CB800943033F818607A6B012107F14700FB6B09
:101CC800984700281ADB0E4B0544BBF1000F08BFEC
:101CD8009B4626B95846FEF74DFC461CB6B27A6BB1
:101CE80031465846FB6B9847002807DB054408F146
:101CF800010854E70026DEE735464CE605464AE685
:101D080088600708014B1860704700BF80010024F5
:101D1800044608B5EFF31183102383F31288BFF349
:101D28006F8F01F0EBFB01F053FC4AF04CFE2046AC
:101D380001F0CAF9024846F08CFF47F02EFDFCE797
:101D480043610708054B00205A6822F002025A60D6
:101D58005A6822F001025A60704700BF0010005C08
:101D680008B5416805480C3183681B681BB1984762
:101D780000EAE07008BD6FF05700F9E70C86060826
:101D88000A2810B502D90024204610BD044B53F888
:101D9800204020464CF0D5F90028F5D1F3E700BFE4
:101DA8007490060808B501F0F9FB01F079FB0C4BBB
:101DB8000C4A1A600C4AD36823F03F0343F004032B
:101DC800D3600A4B1A6841F20303B3EB124F06D1F2
:101DD800074AD2F8083143F00103C2F8083108BDB8
:101DE800800900240090D003004802580010005CCD
:101DF800008000512DE9F047044607464FF00109DD
:101E0800DFF84C8094FAA4F5B5FA85F509FA05F3DC
:101E18002E0108EB05156FEA030A24EA03042B7B5D
:101E280063B158F806301B696BB94644022228464C
:101E380007EA0A077368196847F0C0FA002CE1D16D
:101E48003846BDE8F087284698470028F6D1ECE7E1
:101E5800888C060810B5002288B00E490E484CF050
:101E6800D9FD0022002300240C490D480094CDE937
:101E780006230E234FF44072CDE90334CDE9014423
:101E8800084B0DF05BFC084905484CF011FC204656
:101E980008B010BDB51E0008A82B0024005100246E
:101EA800C0260024D92100085162070801480DF016
:101EB8008FB900BF601400242DE9F0478046204800
:101EC8000F4647F053FA0646002832D00025284628
:101ED800BDE8F087237B83B12368DB680BB120461C
:101EE8009847636883F8069023681B69CBB96368D1
:101EF80002222046196847F061FA01361034544529
:101F0800E8D3B8F1000FE2D0002DDFD02846FFF764
:101F180071FF0546002FF7D0002164204CF0CAFC61
:101F2800F2E7204698470028E1D009FA06F31D4356
:101F3800E3E7044C0546DFF810A04FF00109DEE79F
:101F4800983A0024888C0608988C0608014B53F8A8
:101F580020007047E090060808B5034608462BB1F4
:101F6800044A136000F050FC002008BD6FF0150013
:101F7800FBE700BF8401002410B5044C237813B993
:101F880003480DF025F90123237010BDE64C002409
:101F98006014002410B504460B4847F0E7F95CB11B
:101FA8000A4BBFF35B8F53E8001F013943E8001267
:101FB800002AF8D1BFF35B8F05480EF0E1F9054818
:101FC800BDE810400DF004B9903A0024943A00247A
:101FD800A82B002460140024064B0022BFF35B8F5B
:101FE80053E8000F43E800210029F9D1BFF35B8FC4
:101FF800704700BF903A002470B5FFF7EDFF084C1A
:102008000546084EB44200D370BD63685B792BB1B6
:1020180023685B6813B12946204698471034F1E7D6
:10202800888C0608988C060810B5044C044920468C
:1020380046F01BFF034B1C6010BD00BF7813002443
:10204800CC900608883A002400230D4A4FF47A7190
:102058000C4810B513700C4A13600C4A1360FFF754
:102068007BFFFFF7E1FF0A4B0A4918468B4200D372
:1020780010BD1A1A5C681033121101322271F5E78B
:10208800E74C00248F930408903A0024943A0024E3
:10209800888C0608988C0608014642F210720023C4
:1020A800014846F003BF00BF78130024014846F0FA
:1020B80099BF00BF78130024024B0146186846F008
:1020C800ECBF00BF883A0024014847F021B800BFA0
:1020D80078130024274B70B51B78002B47D0FFF7E7
:1020E800E5FF044600283FD1234B244D1B68002BF5
:1020F80012DD4CF047FC0A220023FEF70FFAD5E95F
:102108000032C01A40F2E93361EB0201984271F1E2
:10211800000101D3FFF770FFD5E9003213F57A7398
:1021280042F10002C5E900320CB3BDE87040FFF788
:10213800CBBF6B685B7923B12B68214628461B68A7
:1021480098471035B542F4D32046FFF7B5FF0C4B3E
:10215800BFF35B8F53E8001F013943E80012002AE0
:10216800F8D1BFF35B8FBFE7064D074EEAE70020C3
:1021780070BD00BFE64C0024903A0024A02B002438
:10218800943A0024888C0608988C060870B50D4D82
:10219800297861B90C4C01200C4EFFF78DFEB44232
:1021A80006D3FFF797FF0028FBD101232B7070BDE2
:1021B80063685B791BB1236820469B689847103495
:1021C800EDE700BFE74C0024888C0608988C0608C9
:1021D80000212DE9F8430846FFF76EFE044648B390
:1021E8004FF4FA784FF000091B4B01F053F91B4AE2
:1021F8001B58136033B11A4B1B68092B02DD1948B1
:102208000CF0E6FF0025184F44B12046FFF7F2FD19
:10221800044618B94FF0FF384FF0FF39FFF75AFF5F
:10222800064628B9B5B90F4842464B460DF00CF89A
:102238003546E9E74FF0FF384FF0FF39D4E72B6810
:102248009B691BB100222846114698471035BD42AC
:10225800F5D3E8E7054DFAE7080000008C3A0024BA
:10226800943A002460140024988C0608888C060888
:1022780013B5184847F07AF8174B1B7873B1EFF38A
:102288001184102383F31288BFF36F8FFFF722FFA7
:1022980084F31188BFF36F8F02B010BD0F4B1B681A
:1022A800002BF9D050B9002200230D48CDE90023B6
:1022B80042F2107200230EF03DF8EDE70928EBD149
:1022C80007480EF05DF8074802B0BDE810400CF072
:1022D8007FBF00BF943A0024E74C00248C3A0024C6
:1022E800A82B002460140024064B10B504461B6874
:1022F80098472146A060044846F055FEBDE81040C6
:10230800FFF7B6BF8401002478130024044A054B64
:102318009B1AB1EBD30F34BF52F83100002070473D
:10232800F88A0608888C06082DE9F04F8FB0C1F3AB
:102338004A260D46904604AF0C0DB8607B60002E0F
:1023480061D04FF000090A234FF0040B07F1140A7B
:10235800FE604A46C7F824904046C7E907990093AB
:1023680007F11C03CDF808B0CDF804A0F968FFF711
:10237800E1FAB0F5006F03461CD36C468AB0D8F872
:10238800041004AB24481A46C3E9050140F2FF7162
:10239800D9614FF400711984204B42F8103F4FF473
:1023A80012514B461E48FFF7BFFFA5462C37BD46C6
:1023B800BDE8F08FC0F30A0604F117003B6018442B
:1023C80066F3532520F007008008FFF765FE0446F2
:1023D80080B13B6800F11001124A4046F961C7E933
:1023E80008390A23009307F11C03CDE901ABF9680A
:1023F800FFF7A0FA66F353257B68B96820462A469A
:1024080046F0FCFFD2E704F1170020F0070080082F
:10241800FFF742FE0446EDE7626207080400000188
:10242800788B0608D79304082DE9F04F87B0054646
:10243800884614469946DDE9127ADDE9106BBFB18A
:1024480010213B465A460020CDF800A0CDF814A034
:1024580046F006FAB0F5006F01460BD340F2FF7361
:10246800184A0221184807B0BDE8F04F47F01FB8D6
:102478003946384604F0070305F00704E40044EA47
:10248800831444EA402444EA065406F117000391F1
:10249800084420F007008008FFF7FEFD054640B11C
:1024A8003FB13B465A4603991030CDF800A046F09C
:1024B800D7F94B4622464146284607B0BDE8F04FBB
:1024C80046F09CBFA1620708788B0608406820B1D7
:1024D800034BC01A40F3CF0070474FF0FF307047EE
:1024E800F88A06080EB403B503AB0146054853F84D
:1024F800042B019301F00AFA02B05DF804EB03B073
:10250800704700BF19950408CA0605D48B064CBF4E
:1025180002490349FFF7E6BF704700BF2894070840
:102528008E8B07082DE9F04F8BB0994604460D466F
:10253800179B9DF8588007931A9F0692DDE918A308
:102548000593B8F1000F00F0BC80834B07F0020B35
:1025580013F80830089307F48073099346F02CFFAA
:10256800024600287AD07D492046FFF7BBFF064681
:10257800BBF1000F08D017F0440F71D12A467849F3
:102588002046FFF7AFFF064407F0010353B1754B30
:102598002046754953F82820744B002A08BF1A466C
:1025A800FFF7A0FF07F48073002B07F0080318BF9C
:1025B8004FF00009002B7FD06D4B20466D4953F832
:1025C8002820FFF78FFF0546069B2BB11A466A495C
:1025D8002046FFF787FF0544B9F1000F0DD0089B8F
:1025E800002B6CD06549664BB8F1040F18BF19462B
:1025F8004A462046FFF776FF054435446148079B65
:102608001BB12246604946F0D4FA059B002B00F026
:102618008E80059B002639462046102B28BF1023A4
:102628009946FFF771FFB54252DC002633461AF887
:10263800032020465549FFF755FF0136102E4DD08F
:10264800710703D152492046FFF74CFF4E453346E8
:10265800EDD350492046FFF745FFEEE7064687E7EA
:102668004D4B186800288ED04C4B4FF47A7B4FF0B6
:102678003C0C1B68B5FBF3F5B5FBF0F100FB1155FD
:102688004FF461630BFB05F5B1FBF3F2B5FBF0FE0C
:1026980003FB121100FB1E55B1FBFCF30BFB05F508
:1026A8000CFB1311B5FBF0F5009120463C49CDE930
:1026B80001E5FFF717FF66E707F0080584E73049EB
:1026C80096E7B9F1010F45460CBF2E48354896E705
:1026D8002F4920460136FFF705FFA4E700263249B7
:1026E8002046FFF7FFFE33461AF8032020462F49FD
:1026F800A2F120035F2B28BF2E22FFF7F3FE01363D
:10270800102E0DD0720703D121492046FFF7EAFEAB
:10271800B1453346E8D81E492046FFF7E3FEEEE709
:10272800059BCA44B3EB090305937FF472AFB8F174
:10273800000F0AD0FB0704D50C4A20460A49FFF7C8
:10274800D1FE39462046FFF7DFFE20460BB0BDE834
:10275800F04F46F0D0BE00BFD5CC0708E7620708A7
:10276800EB620708F0900608E1920708D9620708AB
:10277800049106081163070817630708DE62070853
:10278800E262070819950408153900081B63070851
:1027980015CC070813CC0708A03A00249C3A00245B
:1027A800F56207084F95040821630708289207086F
:1027B80042F20F73114A8B4273B5044628BF0B4689
:1027C80005680521684641F0D5FE636806460B2278
:1027D80028465B680A4946F080FE636832466946C7
:1027E80028465B6846F079FE63681B2205495B68EA
:1027F800284646F072FE02B070BD00BF1777070882
:10280800C9CC0708ADCC070800210123064A90422D
:1028180006D8064A01B901231360054B18607047B2
:10282800400801215B00F2E740420F009C3A002477
:10283800A03A0024F8B50D4604464618054FB442A0
:1028480001D12846F8BD14F8011BBB6801485B6834
:102858009847F4E73C880608014B0360032070475B
:102868004C910608104B70B51C680D46B4B10F4B5F
:10287800196800238B4202DB6FF0010070BD22460D
:1028880012F8146B864202D001331446F2E7E0686E
:102898004BF057FC28B100202C60EFE76FF00C00DC
:1028A800ECE76FF01200E9E7900100247C9106083C
:1028B8002DE9F8430646FDF75DFE0546EFF311885E
:1028C800102383F31288BFF36F8F114B1C68D3F862
:1028D80004909C4208BF002434B988F31188BFF3E0
:1028E8006F8F2046BDE8F883A7683846FDF742FE9B
:1028F800A84206D12A463946304665F05DFB0028D5
:10290800EBD04C4501D02468E6E70024E5E700BF9A
:10291800940100242DE9F0410E461546FFF7C8FF43
:10292800044628B3C3681BB35F690FB3062E07D0EC
:10293800072E20D02A4631463B46BDE8F0411847CD
:10294800838A3BB92A463146B84750B9A38A01332E
:10295800A38206E04FF6FF72934204D00133A382AC
:102968000020BDE8F081124A0121124846F096FD88
:102978006FF01500F5E745B12A7832B100223146EB
:1029880082822A465B699847EAE7A38A012B08D125
:102998002A4607212046B8470028E2D1A38A013BEE
:1029A800D6E70BB1013BDAE7034A0221DDE700BFB6
:1029B80096630708108B0608B863070810B5044625
:1029C80008B1806838B9104A1048012146F066FD00
:1029D8006FF0150010BDFFF76BFF08B10C4AF3E765
:1029E800A082EFF31181102383F31288BFF36F8F56
:1029F800084B5A68C4E9003214605C6081F311889E
:102A0800BFF36F8FE6E700BFD6630708108B060891
:102A1800EF6307089401002480B505460E46174663
:102A280098460DF0ABF9DFF82090034600F032FD30
:102A38000446424649F8003039463046A84754F81B
:102A4800090000F0A3FC00BF0800000003480021B3
:102A5800034A08B5121A46F07CFE08BD0017002488
:102A6800E45000240748084A0849121A08B546F0F5
:102A780072FE0748074A0849121ABDE8084046F09E
:102A88006ABE00BF00000024CC16002460000808BD
:102A98000000002400000024600008082DE9F84F19
:102AA800804600AF0C4600296AD0E9468AB0A36880
:102AB8006D46D1E900123B484FF0050A6E46CDE954
:102AC8000501CDE9072346F810AF002332464FF43D
:102AD80021513548FFF728FCCD466369AD46D4E956
:102AE80003123248C5F810A0C5E90501C5E9072356
:102AF800002332464FF421512B48FFF715FCCD46F1
:102B0800E3692B4A0121284846F0D1FC00252646D6
:102B1800DFF8B0B04FF00A0A264A0121224846F0F1
:102B2800BDFCE9468EB0D6E908C0D6E90A136A4664
:102B3800CDF81CC005F1010CCDE908C0A81CCDE9F1
:102B48000A01E91CCDE905B5CDE90C1342F810AF2F
:102B58000435002345F240011348FFF7E5FB102D2B
:102B680006F11006CD46DCD1236E134A01210E482A
:102B780046F09DFCA369114A01210B4846F097FCD9
:102B8800B8F1010F07D1EFF305830D4A103B414619
:102B9800054846F08CFC214640460BF055FFBD46E3
:102BA800BDE8F88F27640708B88B0608566407083D
:102BB80085640708946407081165070820650708F5
:102BC8004E650708CE64070830BFFFF7FDBF00BF9A
:102BD8002DE9F0410B4E0546DFF83080324606EB12
:102BE8000807CC1B0849204665F09AF9A019083C4B
:102BF8004246002165F0BBF907F10800C5F890408E
:102C0800BDE8F08100000000988C0608080000006C
:102C180010B5204C2049214846F0AAFDA36A990125
:102C280036D51E481E4946F0A3FD1E20A36ADA01C8
:102C380004D51A481B4946F09BFD1F20154CA36A72
:102C48001B0304D51548184946F092FD2120A36AB4
:102C5800590304D51148154946F08AFD22200D4C28
:102C6800A36A9A0304D50D48114946F081FD232033
:102C7800A36ADB0304D509480E4946F079FD2420F0
:102C8800044A936A6FEA03436FEA1343936210BDE1
:102C98001D20CBE700ED00E061650708B88B06084A
:102CA800796507088C650708A6650708C4650708DD
:102CB800E96507080366070870B506460D46284CFF
:102CC8002849294846F054FDA36AD9043CD526482A
:102CD800264946F04DFD1720A36A1A0504D5224857
:102CE800234946F045FD18201D4CA36A9B0512D5C3
:102CF8001D48204946F03CFDA36BA26A100409D583
:102D08001D4A0121184846F0D2FB1EB1A36A23F4DC
:102D18000043A3621920124CA36A590504D512482E
:102D2800164946F025FD1A20A36ADA050ED50E4885
:102D3800134946F01DFD1B20094A936A43F47F435B
:102D4800936200232B7070BD1620C5E7A36A9B040D
:102D5800F2D505480B4946F00BFD1C20ECE700BFF7
:102D680000ED00E02E660708B88B060844660708E1
:102D780055660708686607088166070896660708A3
:102D8800B1660708C96607082DE9F84380468946F1
:102D98001746354D3549364846F0EAFCAB6ADE063B
:102DA80027D511243349324846F0E2FCAB6A1D07A7
:102DB80004D5122430492E4846F0DAFC2A4DAB6A75
:102DC800980718D52D492A4846F0D2FC6E6BAB6A95
:102DD800190646D52A4A33460121254846F067FB9D
:102DE800B9F1000F03D0AB6A23F08003AB62132460
:102DF80003E01024DAE76FF015061B4DAB6ADA071B
:102E080004D514241F491A4846F0B2FCAB6A9B0645
:102E180004D515241C49164846F0AAFC124B9A6A98
:102E2800D50602D49A6A90070AD55B68190507D5B2
:102E38004146304600F02CFA10B180F3098802248C
:102E4800094B9A6A920603D55A6A22F400525A62CA
:102E58009A6A204642F0FF029A6200233B70BDE85E
:102E6800F8836FF01506C2E700ED00E0F866070882
:102E7800B88B06080E6707085566070841670708F4
:102E8800596707086F670708C9660708F0B5674BF1
:102E98009DB005460026586800AFC0F3080386F3C6
:102EA8001188BFF36F8F02F07F44B4F17F4F07D1D1
:102EB80002F00C04082C0ED15D495E4846F058FC1F
:102EC8005D495C4846F054FC00210846FFF7E6FDE2
:102ED8007437BD46F0BD14074CBF0D460126002DC2
:102EE800EED00022FA71DA1E092A7FD8DFE802F054
:102EF800057679727E7E7E7E7E7C50494D4846F00E
:102F080037FC4A4C0023FB71E36A9A0705D54C4904
:102F1800484846F02DFC00242DE0E36A002B01DA36
:102F28004849F5E7E36A5B00F5D54749414846F06B
:102F38001FFC6369AA6943F480736361BFF34F8F11
:102F4800BFF36F8F32F8023C626922F480726261CB
:102F5800BFF34F8FBFF36F8F03F47F42B2F55F4F1C
:102F680021D1DBB2022B1ED12B68384A012131480E
:102F780046F09DFA2C68FB79002BA9D168222946D6
:102F880007F1080064F0CCFF7B6A002E4BD0C3F336
:102F9800080222B96FEA53236FEA43237B6207F1E1
:102FA8000801204692E7214B9A6AD2B22AB1FA1D4B
:102FB80001212846FFF7E8FE0EE09A6A12F47F4FD7
:102FC80004D0F91D0120FFF777FE05E09B6AB3F5F1
:102FD800803FA0D3FFF71CFE0446CCE7FA1D002172
:102FE800E7E7F91D0020EEE7194991E710F4F87FAB
:102FF800184A6C468AB0184918BF11466A46103BF1
:10300800164807934FF40073ADF82030144BCDE900
:10301800050142F8103F00234FF411510548FFF70E
:1030280083F9A54677E76FF30803B7E700ED00E0FB
:10303800BC670708B88B0608E7670708236807080E
:103048003A6807085B680708696807088868070816
:10305800A4680708A36707088E670708C8680708F1
:1030680004000001044B5A6942F010025A615A697F
:1030780022F008025A61704700ED00E0EFF3088083
:10308800EFF3098101B57246FFF700FF01BD00BFEC
:103098000B4880F3088846F056F9102080F3118811
:1030A80008484FF40861401880F30988EFF314804A
:1030B8000221084380F31488BFF36F8F00F078F87B
:1030C80060CB002400620024BFF34F8F0549064BF4
:1030D800CA6802F4E0621343CB60BFF34F8F00BFAE
:1030E800FDE700BF00ED00E00400FA051EF0040F44
:1030F8000CBFEFF30880EFF30980816911F8021C17
:103108000229FFD001B5724646F027FB01BD00BF7A
:1031180009010028C9B206DB00F1604000F56140F2
:1031280080F80013704700F00F00014B19547047E6
:1031380014ED00E000B2002807DB0123410900F08C
:103148001F00024A834042F82130704700E100E046
:1031580000B200280CDB4309012200F01F000549DA
:103168002033824041F82320BFF34F8FBFF36F8F86
:10317800704700BF00E100E04209054B00F01F0066
:1031880053F82220012303FA00F01040704700BFD3
:1031980000E100E0044B054A23F07F039360BFF38E
:1031A8004F8FBFF36F8F70470000000800ED00E0FD
:1031B80008B5FFF7EFFF114BD3F8882022F470020F
:1031C800C3F88820D3F8882042F4A002C3F88820E6
:1031D8004FF04042C3F83422BFF34F8FBFF36F8FD5
:1031E8000023E1EE103AFFF731FCFFF73BFC00F05B
:1031F80033F946F0DFFA0BF053FD00BF00ED00E0B5
:103208008189203A41F0020181814FF47D41C0F863
:10321800DC101360009B08495360019B21F00101F9
:103228009360029B9161D3604FF08073D361002358
:103238000265C0F894307047212A0008838913F08A
:10324800020F124B03D190F8DD20D20611D45A6B2D
:1032580042F080425A63D0F8DC3019075CBF43F073
:103268000803C0F8DC30838943F00203838180209F
:1032780070475A6B22F080425A63D0F8DC301A0744
:1032880044BF23F00803C0F8DC30F0E700EF00E0AB
:103298000A4A0346906878B113F1160FD0F88000F7
:1032A80005D0A0F18002934205D3834203D2814224
:1032B80028BF002070470020704700BF243F00242B
:1032C800104B9B6883421AD1EFF30580B8B9EFF32E
:1032D8001181102282F31288BFF36F8F9A8922F02E
:1032E80002029A81EFF3148323F0040383F3148812
:1032F800BFF36F8F81F31188BFF36F8F70476FF043
:1033080015007047243F002415460E46002208B5D4
:10331800E1EE102AEFF3148222F0040282F31488FB
:10332800BFF36F8FBFF36F8F0B4A0C4B9060D0F8D1
:1033380090201A6000F06CF92C4686F3098800206A
:10334800034B98472046002100220023014C2047C8
:1033580095970408212A0008243F0024D03A002425
:10336800014B10221A61704700ED00E0054B9A6985
:103378009B689A4204D0044A536843F080535360D0
:10338800704700BF243F002400ED00E0084B9B6815
:1033980083420BD1EFF3058343B1064B5A6842F0E1
:1033A80080525A605A6A22F400425A624BF085B938
:1033B800243F002400ED00E024498A6882F8DDE01B
:1033C8004FF030001044EFF3098C80E8F01F1EF036
:1033D800100F03D102F19C0080EC108A102080F3BA
:1033E8001288BFF36F8F1A4F4FF000668A698A60A0
:1033F8003E60D2F89000174C206092F9DDE0D2F8D8
:1034080094000023C2F8943080F311881EF0100F46
:1034180003D00023E1EE103A03E002F19C0090ECA7
:10342800108AEFF3148323F0040383F31488BFF3A3
:103438006F8F04B5104600F0EBF8BDE8044002F1C8
:10344800300090E8F01F8CF309887047243F00246F
:1034580004ED00E0D03A0024002304481021C218EB
:1034680001337A2B82F80013F9D1704700E100E0AC
:1034780008B5EFF30583064A103B02EBC30152F887
:10348800330049688847BDE80840FFF76FBF00BFB1
:103498006C0F00240148006870470000D03A0024EF
:1034A800154A70B5536913F4803323D1C2F88430B8
:1034B800BFF34F8FD2F8803043F6E074C3F3C900EE
:1034C800C3F34E335B0103EA0406014646EA8175FD
:1034D8000139C2F86052F9D2203B13F1200FF2D122
:1034E800BFF34F8F536943F480335361BFF34F8F5A
:1034F800BFF36F8F70BD00BF00ED00E07FB51A4AC3
:103508005369DB032ED50023C2F88430BFF34F8FF5
:10351800536923F480335361BFF34F8F01ABC2F873
:103528007032BFF34F8FBFF36F8FD2F8803043F6FE
:10353800E074C3F3C9000193C3F34E335B0103EA9C
:103548000406014646EA81750139C2F87452F9D277
:10355800203B13F1200FF2D1CDE90211BFF34F8FB9
:10356800BFF36F8F04B070BD00ED00E0002910DDDF
:1035780000F01F030B44BFF34F8F07490344C1F802
:10358800680220301A1A002AF9DCBFF34F8FBFF304
:103598006F8F0020704700BF00ED00E00B4B5A69A9
:1035A80012F4003211D1BFF34F8FBFF36F8FC3F8FE
:1035B8005022BFF34F8FBFF36F8F5A6942F4003226
:1035C8005A61BFF34F8FBFF36F8F704700ED00E074
:1035D800BFF34F8FBFF36F8F064B5A6922F4003247
:1035E8005A610022C3F85022BFF34F8FBFF36F8F89
:1035F800704700BF00ED00E0024B0121024A03487A
:1036080000F090B80000042400000024A8910608E7
:1036180010B50446FFF712FE03460648D4F880208A
:103628000121D21AC0E90023034B8360BDE8104092
:1036380000F082B8D43A002400000B1508B5034600
:103648001048D0F89020C2F30722013A934207D9D4
:103658000D4801210D4A45F02AFF6FF0150008BDFD
:10366800C0F898300A6822F01F021A4342F010028C
:10367800C0F89C208A6842F00102C0F8A0201846D1
:10368800EDE700BF00ED00E0A08B0608DF68070843
:10369800F0B50E4685B01F4604460025B5420DDA42
:1036A800606810B397B1431E18420AD0104A2B46DF
:1036B8000121104845F0FBFE6FF01502104605B0D9
:1036C800F0BD7F28F2D921680B42EFD1236801A908
:1036D800019346F070F8A3680343D0B20393FFF751
:1036E800ADFF10F1160FE7D0421C01350C34D5E7B9
:1036F80005690708A08B0608044B0522C3F8942027
:10370800BFF34F8FBFF36F8F704700BF00ED00E02E
:10371800BFF35F8F024B0022C3F89420704700BFAD
:1037280000ED00E010B5034C01232278FFF7B0FF4D
:10373800207010BDE94C00240B4A08B5002312780C
:10374800FFF7A6FF10F1160F07D0084A0021D2F89C
:103758009030C3F30723984200DB08BDC2F89800F5
:103768000130C2F8A010F2E7E94C002400ED00E0B7
:10377800604861492DE9F043D0F8903085B00C6875
:10378800C3F307239C4200F2B280FFF7C1FF4968E8
:103798000022944201F10C011AD1584F68464FF0AB
:1037A8000008574D3C70FFF757F8564C8146564E67
:1037B800C14520D13B7800204E49D1F89020C2F372
:1037C80007229342C0F28D800020FFF795FF52E058
:1037D800C0F8982051F80C3C23F01F031343013222
:1037E80043F01003C0F89C3051F8043C43F0010347
:1037F800C0F8A030CDE700984FEA081C00EB08118C
:10380800CB682340B3F5000F4ED00BD8B3F5001F9B
:1038180034D0B3F5800F3CD0B3F5801F16D008F133
:103828000108C5E7B3F1007F46D0B3F1805F4BD004
:10383800B3F1807FF3D150F80C30886845F0BBFFB6
:1038480040F088504A6840F4801009E050F80C3085
:10385800886845F0B0FF40F088504A6840F430204E
:10386800039001A93878CDE90123FFF7E7FE002886
:1038780033DA6FF0150005B0BDE8F08350F80C306E
:10388800886845F098FF40F088504A6840F4002066
:10389800E6E750F80C30886845F08DFF4A6840F03C
:1038A800007040F40030DBE750F80C30886845F0D1
:1038B80082FF4A682843D3E750F80C30886845F0FF
:1038C8007AFF4A683043CBE750F80C30886845F0F7
:1038D80072FF4A6840F08850E3E73B7801333B7059
:1038E8009DE7C1F898300133C1F8A00065E74FF0B3
:1038F800FF30C0E700ED00E0A0900608E94C002486
:10390800000004110000F0FF00000410F0B587B0BB
:1039180007460E4614460021102268461D4664F0EC
:1039280026FB02232A4621468DF802306846044BBE
:10393800CDE90476019340F0B1FF07B0F0BD00BFB8
:10394800E597040808B5024B1B689847002008BD96
:10395800E03A0024034B044A1860937843F00203CA
:1039680093707047E03A00249C01002408B505488C
:1039780045F06FF9002383F31188BFF36F8F042399
:10398800184602DF2B6907080649074821F0070196
:10399800C1F1105208B502F5802244F020FF002042
:1039A80008BD00BF73F10024E43A00244FF0FF3251
:1039B8004FF0FF3301480BF013BB00BFAC010024EC
:1039C80001480BF07FBB00BFAC01002438B50546A9
:1039D800FFF7ECFF082108482A4644F056FE044643
:1039E80028B925B1054B0C22FFF754FD1A50FFF7F3
:1039F800E7FF204638BD00BFE43A00240C00000071
:103A080038B504460D46FFF7D1FF082221462B465C
:103A1800074844F0ACFE044628B925B1054B0C22F2
:103A2800FFF738FD1A50FFF7CBFF204638BD00BF1F
:103A3800E43A00240C00000010B50446FFF7B6FF76
:103A480003482146FDF7C0FEBDE81040FFF7B8BFA8
:103A5800E43A002470B541690446867A0A4D59B1A2
:103A6800437ADB0706D42C2303FB06535B6A1B68E7
:103A78009B689847002363612C20214600FB065071
:103A8800BDE870404AF03ABDB41400242C22024B21
:103A980002FB0030704700BFB4140024827A2C2146
:103AA800054B01FB02339A6A1B7F801A1B3323F0F4
:103AB8000303B0FBF3F07047B414002438B52C248A
:103AC800827A064B04FB02335B6AD3E901240C605B
:103AD8001568FFF7E3FF04FB005038BDB414002459
:103AE8002DE9F04385B0054690461C46684603918B
:103AF8004AF04AFFDDE90067EFF31189102383F3E9
:103B08001288BFF36F8F6B8B002B41D02A8B9A42A0
:103B180025D90022002328460BF024FB0446F0B1E7
:103B280089F31188BFF36F8F039B002B41D0324676
:103B38003B4668464AF04DFFA27A2C21254B204689
:103B480001FB023303A95B6A1B681D68DDE90023DA
:103B5800A847606170BB2046FFF77CFF24E0698BB3
:103B68004B1E6B8389F31188BFF36F8F2B7F2A8BD2
:103B78001B33AC6A521A23F0030302FB0344154BB0
:103B8800154AEB1A9B105343A3722B7FE372CBE7C2
:103B980089F31188BFF36F8F2346424628460BF0FE
:103BA800E1FA04460028BFD10024204605B0BDE84C
:103BB800F083636101230025E27A04F11800238170
:103BC8002946039B6560638264F0D1F963692582A5
:103BD800E360EAE7B4140024A38B2EBAF8B50024F6
:103BE800114D2C2600B9F8BD00F108024768BFF353
:103BF8005B8F52E8003F591E42E8001CBCF1000FE1
:103C0800F7D1DBB2BFF35B8F012BECD1837AC460B1
:103C180006FB035344601B6A13B198473846E1E733
:103C2800FFF718FFFAE700BFB4140024F7B50646FB
:103C38000D461446124F38464AF083FAE0B1BB6885
:103C4800AAB2314638461B689847002802DB002094
:103C580003B0F0BD002CFBD1AC42F8D22F1B042FCF
:103C680028BF042707F0FEFD01A901903A46301944
:103C780064F056F93C44EFE76FF01200E8E700BF44
:103C88000488060838B504460CF054F8204645F078
:103C980025FEA069C8B194F86C30DB070DD56FF02C
:103CA8007705154A0221154845F016FE201D45F0F6
:103CB8001CFE0CF053F8284638BD4AF042FA38B9D1
:103CC8000F4A01210D4845F007FE6FF01205EDE798
:103CD800204600F0CBFF05460028E7D10146242204
:103CE80004F1280064F043F994F86C3043F00103C0
:103CF80084F86C30DAE700BF43690708508C06087F
:103D08006D69070870B504460CF014F8204645F0B4
:103D1800E5FD94F86C30DA070DD44FF0FF35254AED
:103D28000221254845F0D8FD201D45F0DEFD0CF0A8
:103D380015F8284670BDC3F340019B0707D51F4AF5
:103D480002211D486FF0770545F0C6FDECE7A06934
:103D580047F07AFA0646A06947F006FB054628B1FF
:103D6800174A0121144845F0B7FDDDE7A36F4BB1B1
:103D78003146204645F099FF0546A0B1A06947F0B5
:103D88001FFBD1E7A06947F097FAA0670028EFD199
:103D98000C4A012108486FF00B0545F09DFDA0690C
:103DA80047F00EFBC0E794F86C3043F0020384F848
:103DB8006C30B9E790690708508C0608B66907089F
:103DC800DC690708F869070838B590F86C300446CC
:103DD8009B0708D46FF07705134A0221134845F072
:103DE8007BFD284638BD45F079FD0021204601F0CD
:103DF800D7F820B10E4A01210C4845F06DFDA069A5
:103E080047F0DEFA054620B10A4A0121074845F085
:103E180063FD94F86C30201D23F0020384F86C30A5
:103E280045F063FDDDE700BF146A0708508C0608FB
:103E38003B6A0708596A07082DE9F043904685B0A0
:103E480006460C4645F053FD0546B8F1000F07D06D
:103E5800304645F051FD012810D1B5FA85F56D09B8
:103E6800013429463046E2B245F038FF814650B960
:103E7800334A23460121334845F019FB00242046E4
:103E880005B0BDE8F0834768B8F1000F09D038687D
:103E980001AB796803C33A7A01AF1A7007238DF82A
:103EA8000530F18D30467B88994228BF194646F087
:103EB80066F804460028E1D0038A00F10C08428A1B
:103EC8004169D21AC36840465B1A3946D21A3B7810
:103ED8009A4228BF1A4645F0D4FCD9F80C90B9F19B
:103EE800000F08D1218AF38D9942C8D9C91A4046D2
:103EF80045F0E2FCC3E7D9F8040083681B6B13B9EB
:103F0800D9F80090EBE7294698470028F8D0071F12
:103F180057F8041F0029F3D008780028F0D0628AE7
:103F2800238AA2EB030C6269E3689B1AACEB0302D9
:103F3800904294BF024692B2404645F0A2FCE7E7A1
:103F4800896A0708308C060838B50446806F45F042
:103F580079FC054645F05AFC2046294601F06EFAE0
:103F6800044638B104480121044A45F097FA284626
:103F7800FFF734FE204638BD308C0608AF6A0708C4
:103F880038B580210446806947F0B9F9054678B10B
:103F98000146204601F052FA044638B1064801218C
:103FA800064A45F07BFA2846FFF718FE204638BD3A
:103FB8006FF00B04FAE700BF308C0608CE6A0708DA
:103FC8002DE9F04F002393B004460F46059315469C
:103FD8000B7E33F080060AD06FF00406AD4A01214B
:103FE800AD4845F05BFA304613B0BDE8F08F82B1BA
:103FF8000846FFF7F3FD7B7EDA0704D49D07F2D568
:104008003B7E002BEFD1204613B0BDE8F04FFFF701
:104018009BBF4A7E00F12809900705D5802B09D15E
:104028003846FFF7DBFDDEE7910700F04384002BFD
:1040380040F04084D3071ED53B8A082B12D1FA687A
:10404800394600201368A3625368C9F8043045F064
:1040580000FC059080B190480121904A45F01EFA75
:10406800059805E08C4801218D4A45F017FA384635
:10407800FFF7B4FD1EE0059794F828500023FFF7DA
:1040880009FA884A15F0600F8350C5F341131CD014
:10409800032B40F065836FF08505824BFFF7FAF933
:1040A8001B58002B00F0A783002D00F06B830598A8
:1040B8000028DDD1484645F052FD0346A069002B93
:1040C80000F03384802100F039BC484645F047FDB4
:1040D80094F82930002840F02D81013B0A2BDAD8CA
:1040E80001A252F823F000BF314200089F400008A7
:1040F800B94200089F4000081D4100089F40000881
:104108009F4000089F400008834100089F40000826
:10411800F9410008A069618D03697F2993F880300F
:10412800B9D8A28D002AB6D1E28D002AB3D1EE0605
:10413800B1D194F83020022A02D14FF0FF35ACE714
:104148001D070BD5C9B245F043FD054648B1638D3F
:10415800554A0121504845F0AAF99EE7012384F801
:10416800393094F83030012B05D1638D1BB984F8B0
:104178003030002591E70123F9E7204645F0B7FBE9
:10418800628D0146FF2A86D8E38D002B83D194F8EF
:104198002830D8067FF47FAF94F83030002BCCD08D
:1041A80092B9618D94F838308B42E2D0C9B220467A
:1041B80000F0F6FE638D054668B13C4A0121009087
:1041C800354845F07EF968E7D2B2204645F0ACFDA7
:1041D8000028E6D1B1E7002B4FF00501204614BFB7
:1041E8000222012284F830201A4645F010FFC0E769
:1041F80005F01F05012D7FF44EAFE38D002B7FF4F2
:104208004AAF628DFF2A3FF646AFA18DFF293FF6E0
:1042180042AF94F83030022B8FD1D2B22046C9B2C7
:1042280045F032FE054638E7E38DA68D002B7FF476
:1042380032AF94F83030002B3FF47FAF012B02D11E
:10424800002E7FF47AAF15F01F0515D0022D90D1FE
:10425800B4F82A80B8F1000F8BD1F6B22046314667
:1042680001F054F9421C05463FF417AF4246314667
:10427800204645F07AFC10E7002E7FF45EAF638D90
:10428800012B7FF476AF94F86C3066F3C30384F89F
:104298006C306EE7F16A0708308C0608296B07084E
:1042A800126B07080C0000004B6B07086D6B0708C2
:1042B800A38DE28DDEB2002A7FF4EDAE628D022A74
:1042C80010D105F01F05190A35437FF4E4AE012229
:1042D800A06945F05AFC00287FF4DDAE012384F87C
:1042E800393046E794F8301000293FF426AF012909
:1042F80002D1002B7FF421AF15F01F050FD0022D3E
:104308007FF437AF002A7FF434AF3146204601F0FE
:10431800DBF8431C05463FF4C0AE0122A7E7002B9B
:104328007FF40BAF012A7FF424AF94F86C3043F08C
:104338000803ACE70A2B63D8DFE813F00B00620030
:1043480062006200620062003A006200DD01620001
:10435800F201E38D022B53D194F83030002B4FD06B
:10436800012BA18D01D100294AD115F01F050ED0CE
:10437800022D17D000260221204645F000FE0546F2
:1043880018B131460C3045F08DFA0595F1E6002953
:1043980036D194F86C309E08C3F3001306F0020679
:1043A8001E43E8E7C9B2204645F00DFE0646E2E79F
:1043B800618DED064FEA1123C9B207D000230AA97F
:1043C80020460A9345F020FC0A9DDEE7013B0E2BB0
:1043D80016D8DFE813F00F0030003800150015007C
:1043E800D20036001500150015001500150015003F
:1043F80015000F01204645F07AFA18B1012818D0A7
:104408000025C2E7266F002EFAD0B4F82E80204689
:104418003378984528BF9846414645F0B0FD054693
:104428000028B2D04246314605F10C0045F029FA81
:10443800ABE7666FE7E700222046FFF7FDFC05467D
:10444800A3E70122F8E70A462046032145F0DBFAF4
:1044580080460028D4D045F07DFBE58D98F81530CE
:10446800B8B998F8146020468DF82930AE428DF816
:104478002860D8F8103028BF2E461B883146ADF882
:104488002A3045F07CFD05460028B9D032460AA9F5
:10449800CAE7B64A4FF0000A8DF81130D8F808304C
:1044A8008DF810A01A40B24B9A4255D1102106A897
:1044B80005F0B6FE061E36DB0AAB102E06AAAD487E
:1044C800984628BF1026564503F1020334D8B60093
:1044D8000236F6B28DF81060AE42204628BF2E464E
:1044E800314645F04CFD0546002889D0022EB346DA
:1044F80000F10C0A04A928BF4FF0020B5046A6EBA6
:104508000B065A4645F0BDF9C346730808EB560238
:104518005A4528D1F0077FF538AF18F803105046F0
:1045280045F0B8F931E758367FF46AAF924A01216D
:10453800924844F0B3FF63E712F8011B0AF1010A3D
:104548004FEA111C01F00F0110F80CC0415C03F890
:1045580002CC03F8011CB6E798F81460D8F810806C
:104568008DF81060B8E71BF8011B5046CDE902230F
:1045780045F098F9DDE90223CAE72046002645F010
:10458800B6F9CDF82A60CDF82E60D4E91C5300287E
:1045980008BF1D460A2320468DF8283006238DF8CB
:1045A800293045F0A9F901287FF42AAF002D3FF4FE
:1045B800ECAE6B882046ADF82A302B798DF82C307C
:1045C8006B798DF82D30AB798DF82E30EB798DF82D
:1045D8002F306B7C8DF830309DF82830E68D9E4268
:1045E80028BF1E46314645F0CAFC054600287FF420
:1045F8004DAFCAE6204645F07AF920B101287FF48C
:10460800FFAE636F00E0236F002B3FF4F9AE5B88C9
:10461800B3F5007F7FF6F4AE594B04F14C060A93CC
:1046280000238DF82C30E36C9E4208BF0023BDF8B0
:104638002A2093B1597D0F2908D1197D0A44ADF874
:104648002A209DF82C2001328DF82C20226D9A42C8
:1046580001D01B68EBE7BDF82A20B4F82E8020466D
:10466800904528BF9046414645F089FC05460028FC
:104678003FF4C6AE9DF8282000F10C0A0AA942456D
:10468800504628BF424645F0FCF89DF8283043457F
:1046980094BFA8EB0308A8EB0808B8F1000F3FF493
:1046A80074AED4F84CB0B3453FF46FAEBBF1000F15
:1046B8003FF46BAE9BF815300F2B15D19BF81420E7
:1046C8005046DBF81010424528BF424645F0D9F85D
:1046D8009BF81430434594BFA8EB0308A8EB0808DF
:1046E800B8F1000F3FF451AE236D5B453FF44DAE7A
:1046F800DBF800B0DAE794F83030002B3FF480AEF6
:10470800E18D01297FF47CAE94F83860204645F0AD
:1047180036FC054600283FF438AE31460C30FFE63B
:1047280005F01F05012D7FF46BAE204645F0EAFA2F
:1047380000283FF465AEA38D4268FF2B3FF660AEBC
:1047480012799A42FFF45CAEDAB20F2A3FF658AEFD
:10475800E18D01297FF454AE234493F83A60D5E7FC
:1047680005A9204645F050FA5CE500BF00FF0200AD
:1047780000030200DACC0708906B0708308C0608A3
:10478800050F05004AF0FEF80A220023FBF7C6FED3
:104798006C4BBFF35B8F1968BFF35B8F41F28732B5
:1047A800461A9642684A41D9BFF35B8F53E8006FB7
:1047B8008E4204D143E8000CBCF1000FF6D1BFF3E0
:1047C8005B8F33D1BFF35B8F52E8003F42E8005163
:1047D8000029F9D1BFF35B8F23B15C4A02215C4801
:1047E80044F065FE5B4A0221594844F057FE5A4B93
:1047F800FEF750FE1D58002D7FF459AC7B7EE28DEC
:10480800D9071FD5484645F0AAF9D8B9DAB12946DB
:10481800A06946F060FD0146059000283FF44AACC7
:10482800204613B0BDE8F04F00F008BEBFF35B8F21
:1048380052E8003F013342E800310029F8D1BFF3C4
:104848005B8FD4E73AB92046FFF79AFB00287FF43C
:1048580031ACFFF7D8BB484645F081F9059D18B93A
:104868002846FFF7BBF9EEE7002D3FF423AC2946B5
:10487800204600F0E3FD10B12846FFF7F9BBA06918
:10488800036993F8801011F004017FF4BCAB46F083
:1048980036FD054600283FF40DAC0146204600F0E1
:1048A800CDFD00283FF4AFAB2C4A0121284844F045
:1048B800F5FDE1E752077FF5FDAB002B3FF4B0AB08
:1048C8003846FFF78BF994F83930002B3FF48BAB5F
:1048D80094F82930052B0CD1618DA069C9B245F037
:1048E80077F9054628B1638D1D4A0121184844F01F
:1048F800DEFD94F82930032B11D1638D022B0ED1E4
:10490800A18D0022A0690E0A314645F03EF9054600
:1049180028B1144A334601210D4844F0C8FD00234C
:104928002E4684F83930FFF75EBBE38D002B3FF449
:10493800C9AB0599003918BF0121C90146F0E2FB4E
:10494800FFF761BBF43A0024F03A0024B26B070881
:10495800308C0608C66B07080C000000EF6B0708D0
:104968004B6B0708136C07080B78062B10B414D18F
:104978000369D3F89C20EFF31184102383F3128882
:10498800BFF36F8F00204B681860506A60B9C2E9A6
:10499800083384F31188BFF36F8F00220023044883
:1049A8005DF8044B49F0CCBC03605362F1E700BFEB
:1049B8003014002430B589B00022002300241E4999
:1049C8001E480094CDE906236FF007034FF4806278
:1049D800CDE90334CDE90144194B0AF0AFFE19497A
:1049E800164849F065FE184B18498B4207D3184BF7
:1049F800002018498B4210D3002009B030BD03F1C4
:104A08001402BFF35B8F52E8000F42E80045002D07
:104A1800F9D11833BFF35B8FE7E703F11402BFF353
:104A28005B8F52E8004F42E80005002DF9D118339A
:104A3800BFF35B8FDEE700BF80540024E02B002427
:104A4800B94A00088E9107080C1600246C16002439
:104A58006C160024CC16002438B50D4645F052F9E2
:104A680030B9114A01211148BDE8384044F016BD5B
:104A7800C46804B938BD2B78032B05D0052B0ED09C
:104A8800022B08D02468F4E7606883685B69002B10
:104A9800F8D09847F6E7606883689B69F7E760682D
:104AA8008368DB69F3E700BF3A6C0708408C0608A7
:104AB8002DE9FF4110274FF0FF334FF0FF3201A9D6
:104AC80065480AF029FA039B1B69D3F89C40236ABE
:104AD80093B1EFF3118287F31288BFF36F8F216AC6
:104AE80029B1606A0B688142236208BF636282F35E
:104AF8001188BFF36F8FC9B99DF80430062BDAD03F
:104B0800072BD8D801A252F823F000BF594B000850
:104B18004D4B0008814B00085F4B0008B54B00085F
:104B2800A34B0008BF4A00084F4C00080B7E2046E4
:104B3800D1F81E205D0602D1FFF742FAC7E745F01B
:104B480031F9C4E700220121204645F060FAB2E7B6
:104B580000221146F8E794F86C3043F0040384F817
:104B68006C3094F83030022B03D101A92046FFF7AE
:104B780073FF00220321E7E794F86C3023F0040365
:104B880084F86C3094F83030022B03D101A9204608
:104B9800FFF762FF00220221D6E794F83030022B9B
:104BA80089D101A92046FFF757FF84E794F86C30B4
:104BB800A66923F0040384F86C30D6F808803369BA
:104BC800BFF35B8FD3F8A030BFF35B8F9A071ED576
:104BD800D8F83C3030469847D8F824300021304681
:104BE80098470546D8F840303046984795B11B4A53
:104BF80001211B4844F052FC00220421204645F0C4
:104C080006FA002D3FF457AF2A4607219CE74FF0DC
:104C1800FF35ECE72946204600F0C2F9054608B101
:104C2800104AE5E7A06946F089FB831E84F83050F6
:104C38005842584194F86C3023F0680343EA401313
:104C480084F86C30D8E7084A0121054844F026FC6E
:104C5800029A062178E700BF30140024696C07081F
:104C6800408C0608976C0708C36C070838B50246DD
:104C780005460C49806946F0C7FB044630B10A4A2C
:104C880001210A4844F00AFC204638BD85F838005E
:104C9800284600F043F904460028F5D0A86946F0F4
:104CA800E6FBF1E771490008D36C0708408C060859
:104CB800F8B501231D460C68002C35D063F07F023F
:104CC800D6B202F07F02103224FA02F7FF0716D597
:104CD800046824FA02F7FF0708D433461348012171
:104CE800134A44F0E4FB6FF01500F8BD05FA02F230
:104CF80024EA020404600C6824EA02040C60DC4024
:104D0800E6070ED5026822FA03F4E40700D4E5E7C3
:104D180005FA03F422EA040202600A6822EA04029D
:104D28000A600133102BC6D10020DEE7708C06081C
:104D3800FA6C07082DE9F04F002691B05368D46843
:104D48000A900891069202930E96039674B9039BF3
:104D5800029A093316719BB293701B0AD370069B93
:104D6800DC68002C40F0C680A346ADE060684FF0D8
:104D7800000A8368CDF83CA01B6B002B00F0AB80C9
:104D880008999847002800F0A680A0F10409354644
:104D9800C4E903AA59F8043F0BB11A789AB9B54285
:104DA80040F29680E3680F9A1343E3606068836873
:104DB8009B6A002B00F0918098478346002800F0FA
:104DC8008F80534A7CE05A780B2A08BF9D70D9F827
:104DD80000305A78042A10D1E2680F990A43E26039
:104DE800DA78002A5BD101229D702369AA40013537
:104DF8001343EDB22361CDF83CA0D9F800707B785D
:104E0800052BC7D10A9B6FF0120B4FF001089B6965
:104E1800099379793A790E9B42EA01225FFA88F17F
:104E28000493ADF8362097F90220002AB3BF41F069
:104E380080014FFA88F342464BB2B7BF21F0800297
:104E4800079310320793049B23FA02F0C0072DD46E
:104E58000F9B23FA02F20593D30727D4BB79FA787C
:104E6800099800930DF136030B9146F0C1F80B99A0
:104E78008346D8B9079BB970002B4FF001030498FB
:104E8800B8BF21F08001BDF83620B8BF1031BA8014
:104E98008B40059918431943CDE90E017AE76A1E3C
:104EA8000FA90EA89A70FFF703FFA4E708F10108FD
:104EB800B8F1100FADD1BBF1000F3FF46BAF154A3D
:104EC8000121154844F0EAFA584611B0BDE8F08FC0
:104ED8006FF0150BF3E7354668E76FF0850B70E761
:104EE80060682E46089944F02DFF039B246803440C
:104EF80003932BE7E36804F10C010EA8A360FFF706
:104F0800D7FE08B924682CE76FF0150BDCE700BF63
:104F18003B6D0708176D0708708C060870B5836924
:104F28000546026F1B6993F88030C3F34113022BC7
:104F38000CD0032B0CD0012B0CBF10230823D371EA
:104F4800EE6D3EB96E6DBEB9344611E02023F6E72A
:104F58004023F4E7324601212846FFF7EBFE0446DA
:104F680040B173685B790B4A01210B4844F09FFA02
:104F7800204670BD3668E4E7324600212846FFF730
:104F8800D9FE044618B173685B79044AECE73668C1
:104F9800D9E700BF5F6D0708708C0608826D0708A7
:104FA8002DE9F04105460E4644F0A1FC804695F8EF
:104FB800383033B3284644F0A5FE0746F0B1014621
:104FC800284644F00FFF10220446002105F13A005C
:104FD80062F0CDFF002385F83830FF683FB984B10F
:104FE80019491A4844F06DFE2046BDE8F0817868FA
:104FF80083685B6A03B198473F68EFE76FF03C044A
:10500800EEE71EB985F838600024EDE732464146E0
:10501800284644F063FE074690B10246284644F00D
:105028000BFF04460028DFD185F83860FC68002CA7
:10503800EAD0606883681B6A03B198472468F6E77A
:105048006FF03C04D0E700BF3B6A0708288C0608CD
:105058002DE9F04105460F461446D2F8048044F085
:1050680034FE95F86C30D9070BD56FF00F07464919
:10507800464844F026FE281D44F02EFE3846BDE87A
:10508800F081012F0AD1284644F036FC30B9404956
:105098003E486FF0850744F014FEECE798F80730B7
:1050A8009A0607D5AB691B6993F880309B0701D432
:1050B8003849EDE71FB1012F06D03749E8E7EB6D16
:1050C8002BBB05F1540603E06B6DABB905F15C062B
:1050D800336800220BBBD5E91C23002F08BF1346F9
:1050E80062685B7C03F10103DBB25371D5E91C12E2
:1050F80008BF0A46537422E09C4206D12749234838
:105108006FF0150744F0DDFDB5E71B68DDE79C424D
:1051180001D12349F3E71B68D2E79C4221D12368D8
:10512800CAB972683360944200D173600023236067
:1051380063685B791B4A0221144844F0B8F9A168F6
:10514800B9B1284644F079FC074668B116490F48BA
:1051580044F0B7FD8FE7136073689C4208BF726024
:10516800E4E71A461B68B5E7A06844F0F3FC88F842
:1051780006000023236073681BB9C6E900440027B2
:1051880079E71C607460FAE7D36D0708288C060875
:10519800F56D0708AF6D0708136E0708336E07082B
:1051A800506E07086D6E07088A6E0708F8B5054641
:1051B80000AF29B301290BD1184C194E2BE06368B5
:1051C80028461968FBF7C4F9B8B11834B442F6D3C5
:1051D8006C4688B06A46134BCDE905354FF4007329
:1051E800ADF81C30104B42F8103F00234FF4E25149
:1051F8000E48FDF799F8A54600242046BD46F8BD9F
:105208000B4C0C4EE2E7636828461968FBF7A0F9D7
:105218000028F2D01834B442F5D3D9E76C1600242C
:10522800CC160024C16E070803000001388C06085C
:105238000C1600246C16002401F07F0311F0800F77
:1052480070B518BF1033012504469D4090F83030E2
:10525800022B06D00C4A01210C4844F01FF900200B
:1052680070BD90F8386044F042FB01462046324653
:1052780044F034FD0028F2D0C0680028EFD08368DD
:105288001D42EDD10068F8E7DF6E0708388C060884
:105298002DE9F84305460846114616461F46FFF70E
:1052A80085FF044600284AD0284644F044FD95F876
:1052B8006C30DA0702D5234A01210CE0D4F80480C7
:1052C80004F11409BFF35B8F6369BFF35B8FDB07DE
:1052D8000CD51D4A02216FF00F041C4844F0DEF87B
:1052E800281D09F0EFFE2046BDE8F883D8F8043001
:1052F8001BB1AB4201D0164ADEE73A463146284692
:1053080044F0ECFCC0B10023236003698BB9C0E909
:105318000344BFF35B8F59E8003F43F0010349E8BA
:105328000032002AF7D1BFF35B8F0024C8F804507D
:10533800D6E71C600461ECE76FF03C04D0E76FF03F
:105348001204D0E7D36D0708046F0708388C0608E5
:10535800266F07082DE9F04F83B00E468146904628
:1053680000AF4C687B6097F830303B6044F0BFFA80
:10537800A36801461B6B33B96FF0150420460C3740
:10538800BD46BDE8F08F204698470028F4D0051F99
:10539800002406F10C0A55F8041F09B10B782BB943
:1053A800002C14BF00246FF03C04E7E74B78042B73
:1053B8000ED1002C3CD18B787A689342EBD1CB7814
:1053C8003A689342E7D10B79002BD7D00124E2E762
:1053D800052BE0D1002CDED0B8F1010F91F802B016
:1053E80009D0B8F1020FF1D152465946D9F8180040
:1053F80044F0AFFD04E05246D9F8180044F08EFDA1
:1054080004460028E2D06D468AB0F3686A46094926
:105418000990CDE907B30623CDE9051842F8103FF6
:1054280000234FF441510448FCF77EFFAD46A5E741
:105438000024A3E7666F0708688C06082DE9F04189
:105448000B7E0C460546590637D16BB344F08FFAEC
:1054580040B11B4801211B4A44F020F84FF0FF30AF
:10546800BDE8F0812846D5F87080268AEF8D44F093
:105478003EFAF8B1421E534253419B01228A9AB127
:10548800BE423246E98D28BF3A4691420CD9B2FB5A
:10549800F3F103FB11223AB994F91830002BBEBF7F
:1054A800637E43F0080363762146A869BDE8F041AE
:1054B80045F084BE98F80730E0E76FF01500CFE7B5
:1054C800588C0608A26F070870B5064680690C4616
:1054D80045F018FE054638B10A4A234602210A4813
:1054E80043F0E5FF284670BD14F0800F4FF001022D
:1054F800736B1CBF24F080041034A2401A437263FB
:10550800F0E700BFB66F0708588C060870B5054667
:1055180080690E4645F021FE044638B1064A3346F6
:105528000221064843F0C3FF204670BD314605F10D
:10553800340044F0E5FCF7E7CD6F0708588C0608FF
:1055480070B50646EFF31181102383F31288BFF379
:105558006F8F1B4D2A6881F31188BFF36F8F5268D4
:1055680092F86C20D20705D40A220023BDE87040C7
:105578000AF096B8EFF3118283F31288BFF36F8FA6
:105588002C682CB1696823688C422B6008BF6B605B
:1055980082F31188BFF36F8F44B1606804F108018A
:1055A800C36998472146074848F067FE2B6833B11E
:1055B800304600220023BDE870400AF039B870BDBB
:1055C800F83A0024BC13002430B585B00546002302
:1055D8001548CDE90012002203A909F003FC024690
:1055E800E8B9039BDDE900015D60083383E8030047
:1055F800EFF31180102383F31288BFF36F8F039B9F
:105608001A600A4A516861B9C2E9003380F3118807
:10561800BFF36F8F0022002305480AF009F805B090
:1056280030BD0B605360F1E7BC130024F83A002446
:105638000000002473B5102504698DF80710EFF3F6
:10564800118685F31288BFF36F8F01220DF10701D0
:10565800206C43F0C4FD86F31188BFF36F8F0128D7
:1056680016D049F01FF8E8B1124B0122BFF35B8F47
:1056780053E8001F002903D143E800200028F7D190
:10568800BFF35B8F04D10C4A02210C4843F006FF9C
:10569800237F2BB10A22002304F1480009F0C8FF38
:1056A80002B070BDA37E002BDED000210A2049F095
:1056B80001F9C4E7003B0024F76F0708208C0608AF
:1056C80038B5056900240E492B6C05F14800C3E97B
:1056D8000144DC60AB6BC3E90144DC6048F0D6FFF1
:1056E80005F17800074948F0A5FF074905F12800AA
:1056F80048F0A0FF284644F0AFFC204638BD00BF64
:105708003558000885590008595A00082DE9F34111
:10571800036906460D46D0F804801C690F7E002AEE
:1057280032D00B8A71323E4807BF02213D4A01211F
:105738003D4A00933B4643F0C4FE2F7E304644F07A
:1057480002FD874204D1042104F1880044F0B3FD2E
:105758002F7E304644F005FD874204D1052104F12F
:10576800880044F0A8FD2F7E304644F0DEFC8742D6
:1057780003D104F18C0009F08DFD2946404602B0A2
:10578800BDE8F04144F01CBC44F0DDFCB84214D143
:105798002A8AE968A06B43F022FD28B1236A1BB16D
:1057A80004F1280009F0D4FE04F18800042144F033
:1057B80082FD04F1780009F0CBFE2F7E304644F0DC
:1057C800D0FC874215D1236A1BB104F1280009F0E7
:1057D800BFFE052104F1880044F06DFD237F9BB9CD
:1057E80000234FF47A7204F1480009F021FF0123E5
:1057F80023772F7E304644F098FC8742BDD104F1D0
:105808008C0009F0E5FCB8E7236C5A89DB889A42DA
:10581800EFD00022002304F1480009F009FFE8E76F
:10582800208C0608167007083A7007082DE9F0471B
:1058380050F8483C00F14007054600215B683846AF
:10584800D3F8009044F068FC002868D0012138465D
:1058580044F062FC8046002861D155F8083C5A891A
:10586800DB889A4203D115F82D3C002B57D0BFF3A3
:105878005B8F57E8004F44F0200347E80032002AC6
:10588800F7D114F02004BFF35B8F48D1484644F0A9
:1058980068FC002282460023224843F0BCFF0646EB
:1058A80050B93846052144F006FD28460A2200234F
:1058B800BDE8F04709F0BCBE80F818A015F82C3CEC
:1058C80033B1428AC16855F8080C43F0A8FC044675
:1058D800214606F10C0043F0CEFF5CB1D9F8040074
:1058E80044F0C7FCB4FBF0F303FB1044B4FA84F8AB
:1058F8004FEA58183146484605F82D8C44F048FBC5
:1059080068B10121084A094843F0C8FD3046FEF74E
:1059180065F938460521BDE8F04744F0CCBCBDE840
:10592800F08700BFB41400245B700708208C0608B9
:1059380038B5034640681B695D68AC68A37A84F88B
:10594800223094F82D3084F82330A376696849B161
:10595800237C3BB944F071F830B1064A012106486E
:1059680043F09CFD002038BD686844F0F3F82074CB
:10597800F8E700BF6D700708208C060870B550F86E
:10598800782C00F11004034600215268204615685F
:1059980044F0C2FB002851D00121204644F0BCFB52
:1059A80000284BD153F8402C686893889189166970
:1059B8005B1A9BB2F61A44F05CFCB0423ED8BFF3C7
:1059C8005B8F54E8003F43F0100244E800210029AF
:1059D800F7D1DB06BFF35B8F06D5194A02211948B8
:1059E800BDE8704043F05ABD284644F0ACFB0022A5
:1059F80006460023144843F00EFF0446F0B106762D
:105A0800686844F036FC638A984203D2686844F0B8
:105A180030FC83B221462846638244F0B9FA68B163
:105A2800284644F090FB034606480121074A43F004
:105A38003EFD2046BDE87040FEF7D0B870BD00BFFF
:105A480097700708208C0608B4140024B77007085C
:105A580038B550F8083C044633B92C4A01212C4883
:105A6800BDE8384043F01ABD50F8283C00F1600505
:105A780002215B681A68002383828383284644F0E6
:105A88004BFBB8B1106954E902319847637D1BB1EB
:105A980004F1500009F05CFD0521284644F03CFB68
:105AA80098B9637F6BB10022002304F1200009F04C
:105AB800BFFD0AE00321284644F02EFB0028E1D16F
:105AC800E4E714F80D3C002BEDD10221284644F000
:105AD80023FB38B12369DA885B899A4202D02046D1
:105AE80009F036FD0321284644F016FB60B1A2698F
:105AF8009388918912695B1A9BB29A4204D0204616
:105B0800BDE8384009F024BD38BD00BFDC70070887
:105B1800208C0608D3B50026002704460648CDE9A0
:105B2800006743F07CFE20B1230604765CBF0023A7
:105B3800038202B0D0BD00BF381500242DE9F04320
:105B480083B000231D4C4FF00108056902AF1C4EBD
:105B580005F1240928602B7785F82030B4422346C4
:105B680001D3002019E095F820201034CAB16C4602
:105B780088B01B6802AA1349C2E905134FF40073E1
:105B88009383114B42F8103F104800234FF4E25121
:105B9800FCF7CAFB6FF00B00A5460437BD46BDE80D
:105BA800F08385F82080484654F8043C009354F864
:105BB800101C54E9032344F06EFECFE72C170808A5
:105BC8003C1708083E71070803000001788C060896
:105BD8001FB5CDE9010103924FF0FF324FF0FF33BB
:105BE80001A9034848F0ACFB002005B05DF804FBB0
:105BF800001400241FB500230190CDE902334FF0B3
:105C0800FF324FF0FF3301A9024848F099FB05B075
:105C18005DF804FB001400242DE9F04117460E46F8
:105C28000446006844F08BFC31463A468046FFF74C
:105C380071FFD4F87B3005460146DB1B2068C4F8A9
:105C48007B3044F0A5F988B10B4A434601210B4843
:105C580043F02DFC3146204644F04FFD2846FDF721
:105C6800BDFF2046BDE8F04144F003BDA37F0133EA
:105C7800A377BDE8F08100BFB7700708788C0608E5
:105C88002DE9F84F0446006844F06EFC4FF03009E7
:105C98000746E37F012B1ED82368D3F810B0D3F84A
:105CA80004A09BF8616009FB06B62436304644F030
:105CB80018FE314602468046504644F06BFC9BF87D
:105CC8001F30054633B1A8EB00023146504644F078
:105CD80061FC05460DB9BDE8F88F204644F017FC75
:105CE8002A46014606463846FFF714FF0546014690
:105CF800206844F04DF980B10A4A3B4601210A4820
:105D080043F0D5FB2846FDF769FF3146204644F0AD
:105D1800F4FCBDE8F84F44F0ACBCE37F0133E37713
:105D2800B7E700BFB7700708788C06082DE9F04F71
:105D3800BE4F89B04FF0FF324FF0FF3305A9BC4882
:105D480009F0EAF8059E069D3469002D40F0998017
:105D580004F12406257794F820309D42C0F28B8008
:105D680004F11803BFF35B8F53E8002F22F00202FF
:105D780043E800210029F7D1BFF35B8FBFF35B8FA6
:105D880053E8001F21F0040143E80012002AF7D16C
:105D9800BFF35B8FBFF35B8FA369BFF35B8FDB0739
:105DA800C8D5237F022B00F08F81032B00F0888158
:105DB80053BBDDF814A0DAF81050EB7F23BB504634
:105DC80044F0D2FB8146284644F0A1FB4FF4007210
:105DD800014606464846FFF79DFE80460146504666
:105DE80044F0D6F8002800F06781924A4B4601211A
:105DF800914843F05CFB4046FDF7F0FE31462846EB
:105E080044F07BFC44F035FCA37F002B92D1237F28
:105E1800012B40F07E81302394F8615004F1630631
:105E280094F8621003FB05453046243500F060FA0B
:105E3800314602462369284600F078FA0646C4F837
:105E48008400284644F043FD8146284644F044FD3A
:105E58008046284644F045FDE26D3044002A40F073
:105E68003C81002840F03481284644F061FD003828
:105E780018BF01202DE130460135303644F01EFDB3
:105E880069E7DDF81C80D6F804A095F81890B8F1F9
:105E9800000F22D02B8A18F1710F674808BF022122
:105EA800009318BF01214B460CBF644A644A43F073
:105EB80008FB95F81880304644F056FB804540F0C2
:105EC800EF80E37F013BE3776969204644F015FCE6
:105ED8002946504644F074F85CE7304644F044FBE9
:105EE800484540F09580237FD5F80C80B5F810B070
:105EF800002B49D1BBF11F0F42D1D8F80030BB426B
:105F08003ED1414604F1540308F11C0251F8040B38
:105F1800914243F8040BF9D10A881A808A78422101
:105F28009A705523E26D84F873305323C4F87B20AC
:105F380084F8743084F87630A36D84F87510C4F84A
:105F480077300023C4F8803094F860309A060FD177
:105F580094F8612094F820309A4209D294F862307B
:105F6800013B0F2B04D8012384F87F302377A0E767
:105F7800206844F0EFFA022384F87F300423F5E721
:105F8800204644F076FB94E7032B92D1302394F813
:105F9800619003FB0949D4F880305B4409F1240976
:105FA800C4F88030BBF1000F16D0484644F099FC85
:105FB80090B141465A46484644F0A5FC804628B967
:105FC800204A5B4602211C4843F071FAD4F87B3022
:105FD800A3EB0803C4F87B30D4F88020E36D9A4221
:105FE8000DD2484644F07DFC00287FF462AFD4F817
:105FF8008020E36D9A4202D2206844F0C1FA4846F4
:1060080044F096FC003818BF012084F87F00B5E7FB
:1060180095F81890304644F092FA81457FF449AFDC
:10602800237F052B10D184F81C8042E75553424347
:1060380000140024B7700708788C06081670070843
:106048003A70070855710708022B7FF432AF2A8A85
:106058004FF03009D4F8803094F861801344C4F8C4
:10606800803023681969D3F804B091F8613009FBCE
:10607800031124310846039144F033FC0399024686
:10608800584644F087FA00287FF413AFD4F87B30E1
:1060980013B1206844F05EFA09FB08402430AFE7EA
:1060A80095F81880304644F04AFA804502BFA37F2D
:1060B80003F1FF33A37707E7EB7F0133EB77A3E621
:1060C8002046FFF7DDFD9FE6204644F026FB9BE6D1
:1060D800022084F87F0004231AE094F9601040B984
:1060E8000029206802DA44F035FABDE644F048FA9F
:1060F800BAE6002914DA904202D8B9F1000F06D1A5
:10610800206844F027FA022384F87F30E3E702236B
:106118002377237F022B0ED1204644F0FEFA09E6AE
:10612800904202D8B8F1000F03D1206844F028FA51
:10613800E9E70323ECE7032B03D12046FFF7A0FD93
:10614800F8E5042B7FF4F6ADA37F2BB11D4A01219E
:106158001D4843F0A3F9EDE5206844F0F0F98046C6
:10616800204644F0D4F904F173030546024604F1CD
:106178007F0153F8040B8B4242F8040BF9D11B78CA
:106188002946404613700D22FFF7C4FC0646014617
:10619800206843F0FDFE78B10C4A434601210A48C5
:1061A80043F085F93046FDF719FD2946204644F0AD
:1061B800A4FA44F05EFABDE5A37F0133A377052373
:1061C8002377B7E57B710708788C0608B77007084E
:1061D800802938B50D46144621D083290DD019BB26
:1061E8008023032011715371832393710023E0707E
:1061F800043065702370A37038BD02231371012326
:106208005371002393710A23D37108224168A0189F
:1062180061F0E4FE064B0E201B882382E6E7044B60
:1062280002201B889380E1E76FF08500E4E700BF58
:1062380014CC07082DE9F04187690646D0F8248078
:10624800BA4228BF3A46B2FBF8F4C269234600684E
:1062580043F068FA0546C0B9B7FBF8F7A7420BD177
:10626800002205213068FCF755FB28B101250A4AB0
:1062780001210A4843F012F9F3692344F3613DB15F
:10628800074B0020B362BDE8F08100240125E7E751
:10629800706A6043F7E700BF9C710708788C0608AE
:1062A8000203000C81420B4607B509D30D4A0221AF
:1062B8000D4843F0FCF86FF0150003B05DF804FBDF
:1062C8006AB101391144814201D28B4207D90221B6
:1062D800009305481346054A43F0F3F8EBE700201E
:1062E800EBE700BFB3710708788C0608CA71070886
:1062F8000C290346084616D11B78252B12D009D83D
:10630800122B10D8084A42FA03F313F0010F08BF02
:106318000620704703F0FD02282A03D05A2B08BF35
:106328000A2070470A207047F6FFFBFF2DE9F0416D
:10633800984690F82C3086B0062A23F00C030446C1
:106348000F4680F82C304FF000038361C0E9043316
:106358000B7840F010810BBB4B795B0724D490F885
:106368002C309F070DD402234FF46852194600259C
:1063780084F8283084F829106285284606B0BDE8DC
:10638800F08144F009FA0028EDD1002319461A4695
:10639800EDE70223052145F20232E8E7032B36D167
:1063A8004E7916F0040604D0022305214FF410524A
:1063B800DDE790F82C308DF8076043F004038DF882
:1063C80008608DF8096080F82C3070230D7901A9D8
:1063D800ADF8043090F82930122D8DF80A6003F0DA
:1063E8000F0328BF122503968DF806300A232A4684
:1063F800ADF812608DF80B30438D4046ADF814604F
:106408005BBAADF8103061F08BFDA662B5E71B2BC7
:1064180000F0898009D8122B1AD01A2B61D0B34A00
:106428000121B34843F043F8BEE71E2BF7D14B795F
:106438005E07B9D40B7913F0030300F09780012BA2
:10644800A3D190F82C3043F0010380F82C309CE75E
:106458004B795E07A8D490F82C3043F0040380F8F9
:106468002C304A7812F002061FD1D5078B7822D536
:10647800B1F80350424619466DBAFFF7A9FEADB20E
:1064880085420BDAB7F803506DBAADB200231A464D
:1064980084F8283084F8296062856EE74246B97826
:1064A8002046FFF795FE051EF0DA022305264FF475
:1064B80010520025ECE72BB18E4A02218C4842F09D
:1064C800F6FFF2E7B1F80350414644F09BF96DBA84
:1064D800ADB2232DD6D941462046242544F092F961
:1064E800D4E74D7915F004057FF45EAF90F82C30B1
:1064F80043F0040380F82C308B783F2B0ED1CE78F4
:10650800002ED2D10D79032301A94046042D019311
:1065180028BF04252A4661F003FDB7E702230526B4
:106528004FF41052B4E74B7959073FF53DAF3B792B
:106538001A090CD19A070AD5DB0715D494F82C3020
:1065480003F00303032B3FF424AF002305E094F882
:106558002C209707C2F34003F0D594F82C2063F35E
:10656800410284F82C2010E70123F6E790F82C204C
:1065780063F30002F5E70A2A7FF451AF2A2B1BD8F0
:10658800222B7FF64CAFA3F12302072A3FF647AF31
:1065980001A151F822F000BF17660008276400081F
:1065A8009966000827640008276400080167000846
:1065B80027640008596700085A2B7FF430AF4D7ADA
:1065C80015F004057FF4F0AE90F82C3043F0040386
:1065D80080F82C308B783F2B40F0DD80CE78002E71
:1065E80040F0D9804FF4C0634046CDE90136B1F898
:1065F800075001A96DBAADB2082D28BF08252A4653
:1066080061F08EFC3246334684F8282053E07B7ACA
:1066180013F004037FF4C8AE90F82C2001AEADF857
:10662800043042F00402B370082380F82C208DF85F
:10663800073044F0B1F8002831464046ABBF236A22
:106648004FF0FF3302220322A8BF1BBA8DF80C209B
:106658000293636A1BBAC3F307228DF80D30C3F3A4
:1066680007438DF80E208DF80F3094F82C3043F046
:10667800040384F82C30B7F807506DBAADB20C2D6E
:1066880028BF0C252A4661F04BFC0023A36274E660
:106698007E7A16F004067FF487AE90F82C3043F02B
:1066A80004039D0780F82C3009D402264FF4685360
:1066B800002584F8286084F8296063855DE644F045
:1066C8006BF80028F1D1236A03B1013B94F82C1030
:1066D8001BBA626A082541F0040112BA84F82C102A
:1066E800C8F800300023C8F80420E2E71172070850
:1066F800788C0608F47107087B7A58073FF554AE82
:1067080094F82C30D7F8026043F00403B7F8075028
:10671800990784F82C307FF526AE204644F03CF8E3
:1067280000287FF420AE6DBA36BA206AADB2314681
:106738002A46FFF7B7FD20B1022305214FF4045282
:1067480015E6174B2361636AE6616B43A3611CE698
:106758007B7A5A073FF528AE90F82C30D7F80260BC
:1067680043F00803B7F8075080F82C309B077FF5F3
:10677800FAAD44F011F800287FF4F5AD6DBA36BAD9
:10678800206AADB231462A46FFF78CFD0028D3D1E6
:10679800044B6361D7E7022205264FF4105333E711
:1067A80071A804083D62000810B504690346204634
:1067B80040F8143B0122002147F0C4FE04F12C00EC
:1067C800024947F037FF002010BD00BF6D6900087F
:1067D80038B5034640681B695C681B6925685A68B8
:1067E8001AB19A680AB1DA683AB915480121154A06
:1067F80042F054FE6FF0150038BD1033BFF35B8FC5
:1068080053E8001F41F0010143E80012002AF7D1C4
:10681800BFF35B8F216909B90020EDE72B7A002BC4
:10682800FAD143F00AF928B1074A0121044842F095
:1068380035FEF1E7206943F08DF92872ECE700BFD7
:10684800608C06082C7207086D70070838B5046953
:1068580040680068BFF35B8F2569BFF35B8FED0766
:106868001FD40BB15D683DB90F4A1048012142F0B1
:1068780015FE6FF0150038BD90F820501DB1DD6889
:106888000DB90B4AF1E785791DB19D690DB9094A22
:10689800EBE7C4E9021263600274120A4274002032
:1068A800E9E76FF07700E6E756720708608C06089C
:1068B80075720708947207082DE9F347D0F804A009
:1068C800884606691546DAF804407768BFF35B8F97
:1068D8003369BFF35B8F9B073DD5236960685B68AD
:1068E800D3F8009043F003F8002201284FF000038A
:1068F800DAF80C0008BF99F81B90294618BF99F8D8
:106908001490CDE90023424642F089FF054650B96C
:106918006FF00B04114A0121114842F0BFFD2046D7
:1069280002B0BDE8F087014680F81890204643F091
:106938002FFB044618B12846FDF750F9EFE7FB692D
:10694800002BECD14FF0FF324FF0FF3306F114006B
:1069580008F07AFCE3E76FF00C04E0E7B57207088B
:10696800608C060870B550F82C3C5C686568BFF30D
:106978005B8F50F81C3CBFF35B8F9B0726D52B69B8
:1069880068685B681E6842F0B2FF01284FF0000299
:10699800A0684FF000030CBF96F8296096F82260B3
:1069A80042F039FF044630B9094A01210948BDE8D7
:1069B800704042F073BD01460676284643F0E8FA77
:1069C80020B12046FDF70AF9034AEEE770BD00BF83
:1069D800D0720708608C0608EA72070807B5084AEB
:1069E80092E80300CDE9000106488268126822B1E6
:1069F8006946904703B05DF804FB6FF05700F9E76C
:106A0800988C06080C86060800F01F0201215F28F2
:106A180001FA02F208B5034605D90C480C4A42F0BF
:106A280046FD002008BD1F284FF0B04106D8D1F818
:106A380088309A430CBF01200020F3E73F2802D892
:106A4800D1F89830F5E7D1F8A830F2E7288B060896
:106A58001F73070800F01F0201215F2801FA02F2E4
:106A680008B5034606D90B480B4A42F020FD6FF0E3
:106A7800150008BD1F284FF0B04103D8C1F8882081
:106A88000020F6E73F2802D8C1F89820F8E7C1F8B7
:106A9800A820F5E7288B06081F730708044B03EBAB
:106AA80040000023013320F8022B8B42FADB7047A9
:106AB800C80D00242DE9F041054600260F4F4FF080
:106AC8000108F4B26B78A34201D8BDE8F0812B78B5
:106AD8001C442046FFF798FF68B12046FFF7BAFF2D
:106AE80057F834303BB107EBC40204F01F04516877
:106AF80008FA04F098470136E3E700BF443B002456
:106B0800034680B1B0FA80F2C2F11F02D2B207493F
:106B180031F912004FF0B042D2F880100B43C2F89E
:106B28008030FCF707BBFF22F1E700BFC80D002447
:106B380030B5B0B1B0FA80F3C3F11F03DBB20B4834
:106B480050F833408C4204D100EBC3056D68954280
:106B580005D044B940F8331000EBC3004260002070
:106B680030BDFF23EBE76FF00F00F9E7443B00244B
:106B780060B1B0FA80F3C3F11F03DBB2044A00210D
:106B880042F8331002EBC30251607047FF23F5E768
:106B9800443B002400F003020F2304329200934088
:106BA800094A43EA900000F00303023352F8232015
:106BB800030C02EA104293FAA3F008B1B0FA80F08D
:106BC80022FA00F0704700BF00040058F8B50369C6
:106BD80000AF0C4603F1A005BFF35B8FD3F8A030DC
:106BE800BFF35B8FC3F38003994218D1184A6E46EE
:106BF800184B88B0002918BF13466A461649CDE9D4
:106C080005134FF40073ADF81C30144B42F8103FD5
:106C180000234FF4E4511248FBF786FBB546BFF357
:106C28005B8F5CB155E8003F43F0040345E8003250
:106C3800002AF7D1BFF35B8FBD46F8BD55E8003F8A
:106C480023F0040345E80032002AF3D0F6E700BF3A
:106C58005F730708677307086E730708030000016E
:106C6800108C06082DE9F0470546894690461F46D0
:106C7800D0F808A044F0F5F80446D0B1067FF30731
:106C88000AD590F8203018480121184A42F00FFC24
:106C98006FF07700BDE8F0873B464246494644F02E
:106CA80098F848B994F82030114A01210E4842F06A
:106CB800FEFB6FF01200EDE79DF8203026F0060687
:106CC80084F8218021466784284684F82430267772
:106CD800DAF818309847B0FA80F3227F5B0963F33B
:106CE80000022277D6E700BF108C060880730708D9
:106CF8009A73070870B50546866844F0B2F80446EA
:106D0800D8B1037FDB0709D490F820300C48012163
:106D18000C4A42F0CCFB6FF0770070BD0146F36976
:106D28002846984738B1237F03F00103227F63F395
:106D380000022277F1E70346F8E76FF01200ECE76C
:106D4800108C0608BC7307082DE9F341D0F80880B9
:106D5800174605460E46D8F83C30984700220023CF
:106D680039460B48FCF7BCFE044670B9094A3B4655
:106D780001210948009642F0A4FB2846D8F8403083
:106D88009847204602B0BDE8F0810676F5E700BFD7
:106D980064150024D7730708108C060813B5036917
:106DA8000C4691F82010D3F8A40046F0A6FA94F8FF
:106DB800203048B1094A01210090094842F081FB7E
:106DC8006FF0040002B010BD5B0601D10020F9E7A6
:106DD800237F43F002032377F8E700BF0574070811
:106DE800188C0608F8B591F9203091F82060002B2E
:106DF80001DB0020F8BD7306FBD047684C8CB7F860
:106E08004830C4F30A040069A34295BF033303342E
:106E18009B08A308D0F8A440402BD4F8E80498BFF6
:106E28005B009D0092B9A8424FF0000224BF401BAE
:106E3800C4F8E804204691F8201001F07F0146F0DC
:106E4800F1FA0028D5D06FF00400D3E7BA68121A17
:106E5800AA4207D20A4832460A4944F074FB6FF046
:106E68000B00C7E79AB206F07F01204646F0DAFA2F
:106E78000028E8D1D4F8E8342B44C4F8E834B8E75B
:106E8800188C060833740708F7B54668074603697F
:106E98007468D3F8A450640028469834A1B2A400BA
:106EA80046F0DFFA1022C5F8E844002128460124FC
:106EB80046F0B8FAD5F8E8344033C5F8E8347368D2
:106EC8009C420ED3284646F022F9054680B16FF061
:106ED800040402461549164844F035FB204603B021
:106EE800F0BDE1B200222846013446F09BFAE6E7FD
:106EF80002460146009040233846FFF7B3FE044699
:106F080028B12A460B490A4844F01DFBE6E7024629
:106F18000090402380213846FFF7A4FE044608B1BC
:106F28008022EFE73069FCF705F9D7E756740708C0
:106F3800188C06086B74070838B503690446D3F83B
:106F4800A45043681869FCF703F900212046FFF7AD
:106F5800D1FE38B10C490D4844F0FAFA6FF0040438
:106F6800204638BD20468021FFF7C4FE044600288D
:106F7800F0D1284646F0EBF802460028F0D0044944
:106F8800024844F0E0FAE9E785740708188C060817
:106F9800A874070838B503690546D3F8A440204605
:106FA80046F03AFA024630B10D490E4844F0CBFAA1
:106FB8006FF0040038BD0021142047F07BFC204608
:106FC80046F02DFA04460028F2D101462846FFF77C
:106FD800FDFD22460221284643F07DFF2046E9E7D1
:106FE800BC740708188C060870B503690446456820
:106FF800D3F8A40046F076F8024618B11A491B489F
:1070080044F0A1FA6668F069D8B143689847044625
:10701800B8B117490246154844F095FA002C19DB17
:1070280000F012FC024618B11249104844F08BFADD
:107038002869FCF7A1F810B12869FCF789F8002045
:1070480070BD0D48716983685B6843B90B4907488F
:1070580044F07EFA0A49054844F07AFAE0E798478E
:107068000028DDD0F2E700BFDC740708188C06089A
:10707800F2740708457507080C8606081075070896
:107088002C7507082DE9F341036906464768D3F8CC
:10709800A45000F0ADFB044640B13B4902463B48D2
:1070A80044F051FA204602B0BDE8F08176683848CD
:1070B80096F84A30D0F80880012B13D97169D8F8AE
:1070C8001830083153B93349304844F041FA32494D
:1070D8002E4844F03DFA6FF00404E3E7224698474F
:1070E8000028F0D1D8F8003071690BB92B49EBE7CB
:1070F8002748984704460028F8D196F84A30012BCB
:1071080014D97169D8F80C3008310BB92449DBE778
:1071180001AA1F4898470028F8D1019A214B9A42A2
:1071280004D02149194844F00EFAD0E7F06950B16B
:1071380003689847064630B11C490246134844F094
:1071480002FA002EC3DB40F2E4420021284660F038
:107158000EFF3B6828462B607B682B7140232B72FF
:107168003B6B6B727B6BEB7145F04EFF024620B1B7
:107178000F49064844F0E7F9ADE7284645F0E7FF30
:1071880000288FD0A7E700BF63750708188C06088A
:107198000C860608807507081A760708A27507087E
:1071A800BD750708006CDC02E1750708FD75070866
:1071B800327607082DE9F04FD0F810908BB00646CC
:1071C8004568D9F8A48000274FF0280A4FF0400BF3
:1071D8006B68BB4256D800274FF0280A4FF0400B87
:1071E8006B68BB4200F2858099F8803023F06A030F
:1071F80043F06A0389F880306B6B2BB999F88030BB
:1072080043F0010389F8803008F5C06108F5BA60D9
:10721800C8F8E4640823042208F59E6847F07DF85E
:10722800D5E910124FF0000A4FF0000B6FF007037A
:10723800012000270096CDE90330CDE906AB524B7B
:107248004046CDE9017708F079FA3168404647F0C1
:107258002FFAEB68984709AA3946A86945F0DDF87E
:10726800041E07DB099B3A461979186845F0E7F8C8
:10727800041E6BDAA31C69D044492246444844F0F2
:1072880062F930E0EB6B0AFB07F117F0800F07F0AB
:107298007F000B449A7E83F820700CBF42F04002B6
:1072A80042F020029A769A7E50B942F001029A760C
:1072B800EB6B5FB1EB6BB5F848200B441A8307E022
:1072C80022F00E0242F00E029A76F3E7A3F818B005
:1072D800EB6B3046194443F0D6FD044638B12D49CE
:1072E8002B4844F035F920460BB0BDE8F08F013744
:1072F8006EE7AB6B0AFB07F167F07F027C060B4475
:1073080083F820209A7E42F020029A760BD1D2B2DE
:1073180042F001029A76AB6B67B1AB6BB5F84820C7
:107328000B441A8308E09A7E22F00E0242F00E0205
:107338009A76F2E7A3F818B0AB6B3046194443F0DD
:10734800A2FD04460028CAD1013749E7A86A08B94E
:107358000024C8E7283546F0F4FE30B90E496FF02E
:1073680015040B4844F0F4F8BDE74FF4B011284673
:1073780044F0A8F80028EBD008496FF0040404484A
:1073880044F0E6F8AFE700BF7174000862760708BA
:10739800188C060846760708807607089C76070842
:1073A80073B5D0F8A46008460C46154643F062FD54
:1073B80018BB94F82030298A802BEA680B4602D142
:1073C800402928BF4023D018C91AE86030462982CE
:1073D80094F8201045F077FF58B194F82030084A07
:1073E80001210090074842F06CF86FF0040002B0E9
:1073F80070BD0121204643F041FD0020F7E700BFA2
:10740800B9760708188C060813B591F820300C4691
:10741800D0F8A400DBB9537EDB071ED4538AC0F82A
:10742800EC34538A402B28BF4023D26894F82010AC
:1074380045F024FF68B194F82030094A01210090F2
:10744800084842F03EF86FF0040002B010BD538ABD
:10745800EBE70121204643F011FD0020F5E700BFCE
:10746800EA760708188C06082DE9F34703690746EA
:10747800D3F8A4604FF0FF334FF0FF3201A906F5AF
:10748800BA6007F049FD9DF80430012B60D0022B4B
:1074980007D0002BEED106F29C41384643F04EFD52
:1074A800E8E79DF80590D6F8E48449F0800A40465C
:1074B800514643F0D6FC0546002143F0DFFC284640
:1074C80043F0FCFC04460028D4D019F07F0F19D1F2
:1074D800038ABBB1402BC2684FF08001304628BFF9
:1074E80040231D4645F0EFFE024620B13F49404883
:1074F80044F029F8BEE7238A5B1B2382E3682B4408
:10750800E360B7E7204643F0DDFC814660B12046E2
:1075180043F0DCFCE26800235146304645F0D3FED8
:1075280002460028A6D0E1E7284643F0C3FC4A46B5
:107538000146404643F0DBFC284643F0BFFC0246C8
:10754800002897D02946D8F81000FFF729FF91E7BF
:107558009DF80590D6F8E4844946BDF806A0404653
:1075680043F07FFC054643F0A9FC044648B921498D
:107578004A461F4843F0E7FF2146284643F07EFC71
:1075880078E751460C3042F076F9B9F1000F17D17F
:10759800BAF1400F14D1228AD6F8EC349A420FD2AD
:1075A800E068638A61699B1A0244411A30465B1A93
:1075B80095F82010402B28BF402345F05FFE59E77F
:1075C800284643F077FC00220146404643F08FFCF2
:1075D800284643F073FC024628B12946D8F8100023
:1075E800FFF712FF46E70146C7E700BF1A7707080B
:1075F800188C060843770708F7B591F8215001223F
:1076080003690C4605F00305D3F8A4706B1E022B22
:1076180088BF0025FFF7E6FB064698B9628C2B4623
:1076280094F820103846C2F30A0245F0C9FD48B163
:1076380094F820306FF004060090044A01210448B1
:1076480041F03FFF304603B0F0BD00BF5C7707084C
:10765800188C060813B503690C46D3F8A40045F046
:107668009CFD40B1054A234600900121044841F0A1
:1076780028FF6FF0040002B010BD00BF857707082F
:10768800188C060837B5036905460C4691F8201092
:10769800D3F8A40045F0C9FD024630B92146284672
:1076A80003B0BDE83040FFF79DBB94F82030054A91
:1076B80001210090044841F004FF6FF0040003B07A
:1076C80030BD00BFB3770708188C060873B5036987
:1076D80005460C4691F82010D3F8A40045F044FE66
:1076E80058B194F82030174A01210090164841F00B
:1076F800E8FE6FF0040002B070BD237F60F3410321
:107708002046237743F0DAFB064608B90020F2E763
:10771800204643F0AFFB94F92030002B07DA00280D
:10772800F4D1324621462869FFF73AFEEEE70028F1
:10773800ECD132462146286902B0BDE87040FFF717
:1077480063BE00BFDD770708188C060837B50D46FD
:10775800044645F0B0FD01238DF805508DF804303E
:10776800ADF806000022002301A904F5BA6046F02E
:10777800E7FD18B10249034843F0EAFE03B030BD03
:107788000D780708188C0608002307B5ADF80630F1
:1077980002238DF805108DF804300022002301A97A
:1077A80000F5BA6046F0CCFD18B10349034843F030
:1077B800CFFE03B05DF804FB0D780708188C0608A7
:1077C800002307B501930022002301A900F5BA6040
:1077D80046F0B6FD002803DA0349044843F0B8FE32
:1077E80003B05DF804FB00BF0D780708188C060885
:1077F80038B54FF0FF324FF0FF33104807F024FD43
:107808000546C8B90E4A1368591C11608BB90D4C4E
:10781800E36843F08073E360E36823F00073E36098
:10782800E3685B0105D400214FF47A7047F042F811
:10783800F6E7024807F0CCFC284638BD901400242F
:10784800943E00240048025810B54FF0FF324FF024
:10785800FF330A4807F0F8FC044660B9084A136881
:10786800013B136023B9074AD36823F08073D360C0
:10787800024807F0ADFC204610BD00BF901400245C
:10788800943E002400480258044A81680020D2F837
:10789800603123EA0103C2F860317047004402589E
:1078A800074A82B083680020D2F860111943C2F8F1
:1078B8006011D2F8602113400193019B02B0704718
:1078C80000440258324B10B518680B88C3F30B03F9
:1078D800132B31D813B96FF0850045E0013B122B0B
:1078E800F9D801A454F823F087790008DF78000854
:1078F800DF7800083D79000877790008DF7800080C
:10790800DF780008877900087B7900088779000804
:10791800DF780008DF780008DF7800087F79000842
:107928007F79000883790008DF7800086579000806
:1079380065790008174811E0D42B0FD003F6287397
:10794800C3F30B031C2BC6D8012404FA03F3124C0F
:1079580023420AD140F211142342BCD010600B68B4
:10796800B3F5805F0DD2002010BD4008F6E70B4844
:10797800F4E70B48F2E70B48F0E70B48EEE70B4853
:10798800ECE7C3F313330133B0FBF3F01060EAE71D
:107998008009002400366E0100101111006CDC0211
:1079A80000B4C404804A5D05405489000076B010D4
:1079B800904B13B5D3F83C2142F00402C3F83C21A4
:1079C800D3F83C2102F004020192019A1A6822F4C9
:1079D80080221A601A6842F480321A601A68940386
:1079E800FCD51A6842F480521A60824A13689804D7
:1079F800FCD500230093804B9A6942F440429A6177
:107A08009A6902F440420092009A9A699104FCD55E
:107A1800784B1A691A6902F03802182A16D11A68BE
:107A2800520706D41A6842F001021A601A6854070D
:107A3800FCD5704B1A6922F007021A611A6912F014
:107A4800380FFBD19A6922F00F029A61694B1A68C4
:107A580022F080721A601A6822F080621A601A682E
:107A680022F080521A609A6A22F0030242F002025F
:107A78009A629A6A22F47C7242F0C0029A62DA6AC6
:107A880022F00C02DA62DA6A42F00202DA621A6B57
:107A98006FF3080242F48B7242F001021A63DA6A49
:107AA80022F00102DA621A6B22F47E4242F400727A
:107AB8001A63DA6A42F48032DA621A6B22F4FE023E
:107AC80042F4C0221A63DA6A42F40032DA621A6BAC
:107AD80022F0FE4242F080721A63DA6A42F480228F
:107AE800DA621A6842F080721A601A689001FCD54E
:107AF8009A6A404C22F07C7242F400029A62DA6A76
:107B080022F4406242F48062DA62DA6A22F4007295
:107B1800DA621A6C6FF3080242F03B021A64DA6AFE
:107B280022F48072DA621A6C22F47E4242F4007205
:107B38001A64DA6A42F48002DA621A6C22F4FE02EB
:107B480042F480321A64DA6A42F40002DA621A6C89
:107B580022F0FE4242F098521A64DA6A42F08072C9
:107B6800DA621A6842F080521A6023689900FCD5DC
:107B7800224806F07BFEA3691E4A23F47063A361C2
:107B8800A36923F00F03A361E36923F0700343F0B3
:107B98004003E361E36923F4E06343F48063E36152
:107BA800A36923F0700343F04003A361236A23F021
:107BB800700343F040032362236923F0070343F073
:107BC80003032361136903F03803182BFAD10A4B16
:107BD8009A6942F440429A619A699204FCD5054A2E
:107BE8000020136923F400431361054B034A1A600C
:107BF80002B010BD00440258004802580076B01088
:107C080080090024132808D8054BC34013F0010F3E
:107C18000CBF6FF08500002070476FF0850070473B
:107C280032C70D0008B5074846F08BFA38B1064848
:107C3800FBF790FE0448FAF765F8002008BD6FF0DE
:107C48001200FBE73C880608557C00080A2838B56E
:107C58000446074D04D1AB680D2128465B68984758
:107C6800AB68E1B202485B689847204638BD00BF60
:107C78003C880608034610B4DA880C46006802F00F
:107C880040021979224383689C693CB1064BA4469B
:107C98005DF8044B134002F0B07260476FF0570074
:107CA8005DF8044B704700BF4000000603460A46D3
:107CB800F0B41979DB88006813430A4A012506697C
:107CC8009A4305FA01F5346808BF83F440238768AE
:107CD80023F48012DB074CBF2C43AC4334603B6871
:107CE800F0BC184701001000034637B5D0F8D000A3
:107CF80070B193F8D440836801A905695B68984717
:107D0800031E08D010DA0A4A02210A4843F053FD3C
:107D1800012003B030BD2A68019B53400122A240D4
:107D28001340003B18BF0123181E18BF0120F0E7BD
:107D380059780708F08B060808B5836E034A0121B5
:107D4800034843F038FD6FF0040008BD7778070852
:107D5800F08B0608F8B503690D4616464FF0FF325A
:107D68001C694FF0FF33271D3434384643F038FD83
:107D7800AA192946204605F0AFFB034658B16FF013
:107D88000404084A0121084843F015FD384607F065
:107D98001FFA2046F8BD204645F0A2FB0428FAD178
:107DA8000024F3E7A5780708F08B060810B5012131
:107DB8000446D0F8E40043F030FD034630B186288D
:107DC80004D0064A0221064843F0F5FC04F1D80025
:107DD8004FF4B011BDE81040FFF768BFC17807083D
:107DE800F08B060838B50446343045F054FB054698
:107DF8000D48D4F8E01083685B6803B198472DB14B
:107E08002046FFF799FF6FF0040038BDD4F8D03052
:107E180013B1204643F0ECFC204643F00DFD01234E
:107E28000020C4F8B030F0E70C86060870B5056984
:107E38000446D5F8E80046F084F9E8B12E46204615
:107E480056F8043B984701223046114646F07AFB23
:107E58000122002105F11C0046F074FB05F1B40075
:107E6800094946F0E7FB284643F0E6FC0748046169
:107E7800BDE87040FAF7A2BD054A0121054841F066
:107E88000DFB6FF0120070BD4DB804087806002491
:107E9800E9780708F08B0608F7B503691D69D5F876
:107EA800D800A8B105F1D80446F04BF920B96FF015
:107EB8000404204603B0F0BD4FF4D0112046FFF76C
:107EC800F5FE0028F3D14FF4FA70002146F0F2FCD9
:107ED8000021D5F8E40043F0A0FC041E03DA28468C
:107EE80043F0AAFCE5E7D5F8D000B0B346F029F98D
:107EF80068B395F8D43001224F4905F1C40702FA56
:107F080003F3D5F8D000C5E932138368DB690BB3F6
:107F18003946984704460028E1D105F1D0064FF4C8
:107F280080313046FFF7C2FE044650B94FF0E86191
:107F38003046FFF79FFE044678B100213046FFF730
:107F4800B5FE3946D5F8D00043F04CFCC7E76FF0D2
:107F58001204C4E76FF05704C1E72846FFF7C4FED0
:107F680060B902236FF01204C5F8B030D5F8D030EC
:107F7800002BB4D0284643F03BFCB0E72F4C012738
:107F8800D5F8E010A668C5F8B0700831B36963B9D0
:107F98002B4A6FF0040401212A4841F07FFA2A4A4B
:107FA8000121284841F07AFAE0E700222046984764
:107FB8000028EDD1D5F8E010F36808310BB9234A51
:107FC800E7E701AA204698470028F8D1019B204AF4
:107FD800934207D01F4A39461A486FF0850443F088
:107FE800EAFBDCE73368D5F8E01073B12046984720
:107FF80004460028D3D1D5E93A018368DB683BB150
:108008009847044638B1144ACAE76FF05704C6E7E0
:108018006FF05704F7E705F1340045F075FA40B101
:10802800AB6E0E4A012107486FF0040443F0C3FB0E
:108038009CE7C5F8B0003CE7C3B704080C860608FF
:1080480008790708F08B0608707907082C79070863
:10805800006CDC025279070886790708A1790708BD
:108068002DE9F843994603690D4616461C694FF0F9
:10807800FF324FF0FF33271D04F13408384643F030
:10808800AFFB4B4632462946404605F063F90346A6
:1080980068B904F11C004FF0FF324FF0FF3343F092
:1080A8009FFBD4F8B0407CB10A4A234600E00A4A54
:1080B8006FF004040121094843F07DFB384607F0BE
:1080C80087F82046BDE8F883404645F009FA0428B9
:1080D800FAD1F3E7E5790708CD790708F08B0608A8
:1080E8002DE9F843994603690D4616461C694FF079
:1080F800FF324FF0FF33271D04F13408384643F0B0
:108108006FFB4B4632462946404605F085F9034643
:1081180068B904F11C004FF0FF324FF0FF3343F011
:108128005FFBD4F8B0407CB10A4A234600E00A4A13
:108138006FF004040121094843F03DFB384607F07D
:1081480047F82046BDE8F883404645F0C9F90428B9
:10815800FAD1F3E70F7A0708F6790708F08B0608D3
:108168002DE9F8431C46D0F804809B88D8F80050C5
:108178000B440669089FAB42D6F8B8C005D8E38817
:10818800D8F804001344834207D91948194943F021
:108198002AFC6FF01500BDE8F88396F8AA3005FBB5
:1081A80002114FF0000901FB03C5E2881FFA89F3A9
:1081B8009A4201D80020EEE7A388294696F8AA201B
:1081C80038465A435FF0ACFEA18896F8AA30594366
:1081D800384609F10109FBF7C9F996F8AA30D8F829
:1081E800002002FB0355228903FB0277DDE700BF6D
:1081F800188B06083F7A07082DE9F843099F1D46A2
:108208000646894690469DF8203004693FB92248C1
:10821800224943F0E8FB6FF01500BDE8F883D4F875
:10822800EC1031B11C481E4943F0DDFB6FF00F0024
:10823800F3E733B91B49184843F0D5FB6FF05700F3
:10824800EBE7032D01D91849F5E7AB0702D520461E
:1082580004F006F801233B6084F8FC30C4E93B696C
:10826800C4E93D853B68C4F800312368196C21B125
:10827800196C226B914208D2196CC4F804115B6C1A
:108288009BB2994203D80020C7E70021F5E72046B2
:1082980003F0E6FFF7E700BF188B0608677A0708C0
:1082A8009A7A0708D07A0708137B070898B54068B8
:1082B80000AF046B036924B923B96FF05700BD46BA
:1082C80098BD33B10121103043F026FB0028F6DBBE
:1082D80014B3204645F035FF0346B0B921686C4613
:1082E80088B06A460D48CDE905014FF40071ADF834
:1082F8001C100B4942F8101F0A484FF4E251FAF7D4
:1083080013F86FF01200A546D9E7A3685B68002B45
:10831800D3D020469847D2E72046D0E7447B0708C9
:1083280003000001188B0608F7B54568074606697B
:10833800AB6873B14FF4D01105F1080043F0D1FADE
:10834800041E06DA3449354843F04DFB204603B095
:10835800F0BD2B694BB14FF4B01105F1100043F09B
:10836800C0FA041E01DA2E49EDE701AA0021A86A25
:1083780044F053F8041E07DB019B002219791868A2
:1083880044F05DF8041E01DA2649DCE72648A969AD
:1083980083681B6823B19847041E04DA2349D2E78F
:1083A8006FF05704FAE7D5E908018368DB6803B181
:1083B80098471023A6F8A830022386F8AA3001228D
:1083C800002106F1BC0046F0BDF8012206F1D400F8
:1083D800114646F0B7F8EB6A38469847144A3046D3
:1083E800136823F00D03136044F0F5FA04460028DF
:1083F800ACD1024606F13801304644F04AFB044647
:108408000028A3D13268D2F8043123F00103C2F85E
:108418000431084B186499E7607B0708188B060835
:10842800947B0708CB7B07080C860608E57B0708C2
:10843800004000520010005098B5406800AF046B2F
:10844800036924B923B96FF05700BD4698BD33B10D
:108458000021103043F060FA0028F6DB14B3204600
:1084680045F06FFE0346B0B921686C4688B06A468D
:108478000D48CDE905014FF40071ADF81C100B490A
:1084880042F8101F0A484FF4E251F9F74DFF6FF018
:108498001200A546D9E7A3681B68002BD3D0204655
:1084A8009847D2E72046D0E7447B0708030000013D
:1084B800188B06082DE9F843D0F804801D46B3F858
:1084C8000490D8F8006009EB0103089FB34207D86D
:1084D800B5F806E0D8F804C002EB0E03634507D9E7
:1084E8003348344943F07FFA6FF01500BDE8F8834C
:1084F800046952EA010094F8AA3030D14E452ED1D1
:10850800F4452CD12889B04229D10CFB00F138461A
:108518005943FBF72BF8D4F8B830BB421DD004F10F
:10852800BC05284606F0B6FE23680122C4F8B470DC
:10853800DA632268536B43F0010353634FF0FF3350
:108548004FF0FF32284606F07FFED4F8EC3023B90E
:108558002268536B23F0010353630020C6E75E4390
:108568004FF000094B4302FB0632D4F8AC601644C6
:10857800EA881FFA89F39A42EFD9AB88394694F80A
:10858800AA2030465A435FF0CBFCA98894F8AA3059
:108598005943304609F10109FAF7E8FF94F8AA307F
:1085A800D8F8002002FB03662A8903FB0277DFE77D
:1085B800188B06083F7A0708F8B5066905460F467E
:1085C80006F1D4044FF0FF334FF0FF32204606F097
:1085D8003BFED6F8EC30AB4209D00C490C4843F0CE
:1085E80002FA204606F0F4FD6FF01500F8BD012FE1
:1085F80001D00849F2E71C22002106F1EC005FF0E7
:10860800B6FC204606F0E4FD0020EFE70C7C0708E6
:10861800188B0608397C0708064A11680B6823F08E
:1086280004030B60044B5068196883685B6803B1E6
:10863800184770479807002404080024094B10B510
:10864800D3E90040084B196883681B6803B1984751
:10865800236843F004032360236843F0080323607E
:1086680010BD00BF980700240408002408B5EFF3E4
:108678001181102383F31288BFF36F8F094B0120F8
:1086880093F8482083F8480081F31188BFF36F8F6F
:1086980032B9FFF7D3FF5020BDE80840FAF74ABDCA
:1086A80008BD00BF9807002438B5436804693848F6
:1086B8006060196883681B6853B19847054650B1D4
:1086C800344A2B460121344840F0F1FE284638BD93
:1086D8006FF05705F4E7012204F10800114645F050
:1086E80031FF0122294604F1200045F02BFF04F157
:1086F80038002A4945F09EFF07232A46294684F870
:1087080061300423502084F85E5084F862300F23CF
:1087180084F85F5084F84C300C2384F8605084F857
:108728004D3084F8495084F84A5084F84B5041F051
:1087380023F81B4B1B491C681B4A2368226123F042
:108748007C43206923F0FF038B4203D147F2AC211D
:10875800884212D0216821EA0301144B0B4323609D
:1087680047F2AC232261226122612361236823F04E
:108778008043236023685B00FCD4236843F0040330
:108788002360236843F008032360FFF76FFF9DE72A
:108798000C8606089B7C0708208B0608C5BA0408C7
:1087A80098070024000DF000BC0A5917000DF0408E
:1087B800F8B58378C678EFF3118E102484F3128805
:1087C800BFF36F8F057890F801C05B1B2C463340D0
:1087D8009A4288BF9AB2AF18374007708EF3118853
:1087E800BFF36F8F8F188F421BD165450CD1EFF304
:1087F8001181102484F31288BFF36F8F04784470BA
:1088080081F31188BFF36F8F01799B1A94B2994253
:1088180005D345F047FF68B1084806F099FE2046A1
:10882800F8BD00EB040E01349EF805E0344001F871
:1088380001EBD8E7FFF71AFFF1E700BFD0070024E4
:1088480070B50D4614460CB9204670BD4FF0FF3286
:108858004FF0FF330B4806F0F7FC224629460A483A
:10886800FFF7A6FF064630B94FF0FF324FF0FF334F
:10887800064806F0E9FCA41B0248354406F0A8FCAB
:10888800A4B2E0E7A0070024F6070024B8070024F4
:108898001D4B014610B51B68EFF31184102282F3BB
:1088A8001288BFF36F8F5A68500605D45A68D207EA
:1088B8001DD46FF00A0015E01A6842F080421A6071
:1088C8001A6822F080421A600A221868400005D40B
:1088D8005868400602D458684007E7D5013AF4D1F1
:1088E8006FF0040084F31188BFF36F8F10BD5A68CE
:1088F8009207F5D4586810F04000F1D19B680B60DE
:10890800002BEFD1D5E700BF980700242DE9F743E6
:10891800D8078846144605D43148FFF749FF03B005
:10892800BDE8F083002A37D0EFF31185102383F3D5
:108938001288BFF36F8F5020FAF71EFC06465020AE
:10894800FAF706FC85F31188BFF36F8F0EB9FFF7AE
:1089580075FEDFF89490D9F800305A68510713D49F
:108968005B685A0610D41F4F4FF480332546C7F86A
:108978008831D9F800305B68DB070FD4BFF34F8F1D
:1089880020BF40BF20BFF4E7002401A8FFF780FF05
:1089980016B35020FAF7CEFB2046C0E701A8FFF730
:1089A80077FF4FF480320346C7F8882188B9291F1A
:1089B800019A89B2002DEBD0A94203D1002BD8D05F
:1089C8000192D6E7013D0123ADB208F80520120A4D
:1089D800F0E7002DCDD1DBE7FFF71EFEDCE700BF97
:1089E800E107002400E100E0980700242DE9F7439F
:1089F80001A8FFF74DFF002843D1284C0427019A0E
:108A0800804694F84B30014694F84CC094F84AE0FC
:108A1800A3EB0E055FFA82F93CEA05051ED194F82E
:108A2800601094F85F6094F861508E1B35EA060672
:108A38002AD108B184F84B30B8F1000F00D0019268
:108A48005020FAF785FBFFF7E7FD002384F848304C
:108A5800134803B0BDE8F04306F0BABBE018013391
:108A680080F84E900CEA03030120013F4FEA1222DE
:108A78004FF00108CCD108B184F84B30019200299D
:108A8800E6D103B0BDE8F083661801310D4086F8E1
:108A98006390012184F86050E7E700BF980700243D
:108AA800B8070024C3780F2B14D9C96B0B480B0ED9
:108AB80000EA911013708B02090603F47C0301F09D
:108AC800FE41034300200B4311686FF31E210B4343
:108AD800136070476FF08500704700BF00FF030008
:108AE800F8B50D4616460021502204465FF03FFABD
:108AF800A5F10803A91E5842C9B25841022E11BF58
:108B0800002308234FF000664FF400670FBF4FF0B3
:108B180000521E461F461A4606294FEA001016D86C
:108B28000E4DDFF840E015F801C00D4D35F8115035
:108B38005EF8211063614FF44053E561A163266438
:108B4800A264C4E903C0C4E908372046F8BD4FF061
:108B580080714FF480754FF0010CEBE727CD0708C3
:108B6800C85907085094060800487047D09406086A
:108B7800002370B5C0F8AC300446154644F091F9AE
:108B880038B1104A0121104843F09EF86FF00400F4
:108B980070BD0A2304F17406A5FB0323304606F0D2
:108BA80053FB58B1094A0121074843F08DF8204684
:108BB80044F0E8F9304606F06DFBE7E7D4F8AC007E
:108BC800E6E700BF017D0708388B0608167D070811
:108BD80070B59AB00E46144605461422002101A825
:108BE8005FF0C5F906A822463146FFF779FF082E3F
:108BF80041F2883206A90DBF40F2F963062001232D
:108C0800089318BFCDE90803002328460D93149351
:108C1800179344F000F8034640B1214A2148012146
:108C280043F052F86FF004001AB070BD082E19D145
:108C380040F2FA53022C4FF480604FF080610893A1
:108C48001CD004230124179300230D9041F288328D
:108C58001491284606A915940C9343F0DCFF78B1CB
:108C6800114ADBE705210122022C4FF48070CDE97F
:108C780008124FF08071E6D01446E4E70523E2E7D6
:108C880002231022039001A92846CDE901334FF4AD
:108C98008003CDE9043241F28832FFF769FFC3E768
:108CA800307D0708388B0608537D070870B59AB0E1
:108CB8000E46144600211422054601A85FF057F914
:108CC8002246314606A8FFF70BFF082E21D140F2B5
:108CD800FA53022C08932AD0042301241793002363
:108CE800102215940C934FF48003012406A92846FA
:108CF8000294CDE9043241F2883243F08CFFC0B1CE
:108D08000F4821460F4A42F0DFFF6FF004001AB007
:108D180070BD052301224FF08071022CCDE9083285
:108D28004FF0000314910D93D8D01446D6E70523CD
:108D3800D4E741F2883201A92846FFF719FFE6E790
:108D4800388B0608777D07082DE9F041D0F80480B4
:108D580094B004690F46154698F81C1098F820201E
:108D680068461E46FFF7BCFED8F81C30082B1AD1FF
:108D780045F6A523142202934FF4405311926946F5
:108D880041F288322046089306970F9643F043FF36
:108D98000246B0B11149124842F0A6FF6FF0150023
:108DA80014B0BDE8F0815A220123CDE902234FF027
:108DB800807308220E934FF4807307934FF4005387
:108DC800DCE741F288322946204643F0BBFF0246E1
:108DD80008B10449DFE7C4F8AC00E1E7947D07086F
:108DE800388B0608B87D0708002208B5C0F8AC2003
:108DF80041F2883243F00FFF024628B10349044884
:108E0800BDE8084042F070BF08BD00BF947D070868
:108E1800388B06082DE9F04F8046B3B00F4614464C
:108E2800002A3BD046687269A242154628BF2546EB
:108E380000292ADBCB17491943F100038A424FF076
:108E48000001994121D3C5F30B035BBBD8F81090FF
:108E5800484642F04EFF502200210AA85FF087F8EA
:108E680096F82020317F4846FFF720FF044618B3C4
:108E78006FF00F04864A0121864842F025FFD8F892
:108E880010005C3042F01EFF08E06FF015043B460E
:108E9800814A01217F48009540F013FB204633B0FA
:108EA800BDE8F08FA242D1D97C492A4679486FF0B3
:108EB800850442F019FFF1E7F369082BA3F1080ACA
:108EC80014BF012204220D92326AA2F1020EDEF1D1
:108ED800000242EB0E02DAF1000343EB0A03D20070
:108EE8001B010F920E93002DC9D0002CC7D196F804
:108EF80020204846317FFFF76BFE044628B1684AB8
:108F08000121644842F0E0FEB9E77269F369AA42B8
:108F180063D1082B46F29F030AA9109018BF60235B
:108F28001190D8F810000C93FFF75EFF7369214683
:108F3800D8F81020ED1AD8F804300392142293F8C8
:108F48001CB093F820A00DEB02005FF010F8594612
:108F580052461EA8FFF7C4FDBBF1080F22D140F20C
:108F6800FA52BAF1020F20922AD0042401232D9339
:108F780000232F9410242493022341F288321EA93F
:108F880006934FF480030398CDE9083443F043FE79
:108F9800D0B16FF00404434A01213E4842F094FEE8
:108FA800414AADE74FF0050C01224FF08071BAF14C
:108FB800020F25942C91CDE920C203D15346D6E760
:108FC8000524FBE71346D2E7384A05A90398FFF7BB
:108FD800CFFD0446002886D0E2E7082BD8F8100019
:108FE80009F19C0E109714BF4FF480734FF48063FF
:108FF8001193336A9A1E53425341DB02139390F83C
:109008009E30042B09F194030CBF4FF4405C4FF4DD
:10901800005CCDF848C05A7872B14FF0FF319140EA
:1090280037EA010108D101219140A94204D8ECB1E5
:109038006178914238BF1C4602339E45EBD1F369F3
:10904800B4B1082B1CD023780AA90C93FFF7CCFEE7
:10905800CCB16278012393401F44ED1A96F8202082
:109068004846317FFFF722FE04463CE71C46E3E70B
:10907800082B05D0BCF5405F14BF20232123E3E76C
:1090880042F2DE13E0E707F58057A5F58055E5E7DE
:10909800337E0708388B0608D07D0708157E070839
:1090A8004D7E0708697E07088C7E0708E0040700E4
:1090B80038B5CB630023154641F28832C0F8AC308E
:1090C800044643F0A8FD024630B10D490D4842F070
:1090D8000BFE6FF0040038BD2946204643F0ACFE75
:1090E800024608B10849F1E74FF0FF324FF0FF336D
:1090F80004F1740006F0A8F8D4F8AC00EBE700BF60
:10910800947D0708388B0608B87D0708F7B50D1E4B
:109118001C460FDB476815EB030C4FEAE5767F69C1
:1091280046F1000667454FF00007B74102D363B91F
:10913800184608E007482B46074A0121009440F0EA
:10914800C0F96FF0150003B0F0BD03B0BDE8F04002
:1091580042F0F4BD388B0608D07D070838B51546AF
:1091680004694268CB630023C4F8AC30D369082B88
:109178000BD10B6AB3F5405F07D0134A012113489E
:1091880042F0A2FD6FF0040038BD41F2883220465B
:1091980043F041FD024620B10D490C4842F0A4FDC0
:1091A800F0E72946204643F026FE024608B1094961
:1091B800F3E74FF0FF324FF0FF3304F1740006F08D
:1091C80043F8D4F8AC00DFE79E7E0708388B060822
:1091D800947D0708D07E07082DE9F04F0D1E97B043
:1091E800804692461E462FDB4768AA194FEAE57368
:1091F800796943F1000391424FF000029A4123D369
:10920800002E00F0AC80D0F81090484642F071FD76
:1092180097F82020397F02A8FFF762FCD9F8A4301C
:10922800382B049356D041D8322B4BD019D823F081
:109238001003022B17D1012305934FF48073099370
:109248004FF0807310930EE06FF015042B46454ADB
:1092580001214548009640F034F9204617B0BDE892
:10926800F08F342B2ED0D8F810304846089593F854
:109278009E30042B0CBF4FF440534FF400530A9315
:109288000023139397F82020397FFFF70FFD00285C
:1092980051D0D8F810005C3042F014FD334A012157
:1092A80031486FF0040442F00FFDD6E73E2B11D091
:1092B800A22BD8D1012305934FF4807309934FF063
:1092C8000073BFE7012305934FF4807309934FF0B0
:1092D8004073B7E7012305934FF44073F6E7B6F5FB
:1092E800807FB3464FEA152202A928BF4FF4807B3E
:1092F800404608950BEB0503013BB2EB132F524692
:109308001CBF5FFA85FBCBF5807B5B46FFF726FF2A
:10931800044608B1164A18E097F820204846397FD5
:10932800A6EB0B06FFF7C2FCDA445D44044608B11D
:10933800104A0AE06EB197F820204846397FFFF7B7
:1093480047FC04460028CAD00B4A0121064842F0CF
:10935800BBFCD8F810005C3042F0B4FC7DE7344622
:109368007BE700BFD07D0708388B0608E97E070831
:10937800177F07082E7F0708FF7E07082DE9F04FA3
:10938800D0F80480C3B004460569D8F81C30082B0F
:109398000ED0D8F82030022B0AD16FF0850BA94ADD
:1093A8000121A94842F090FC584643B0BDE8F08F2F
:1093B8002EAA0021D8F8240043F02FF8B0F1000BB2
:1093C80008DB2E9B00221979186843F038F8B0F1B1
:1093D800000B05DA9D495A469B4842F085FCE3E7B5
:1093E8009B4EB7683B683BB99A4A0121964842F0C0
:1093F8006BFC6FF0040BD7E74146304698470246AE
:109408000028F1D1BB6908F108090BB9924AECE7C9
:109418004946304698470028F8D1FB680BB98F4A6F
:10942800E3E70AAA4946304698470028F7DB0A9935
:109438000123D8F8180040F20112B1FBF3F6B0424C
:1094480002D201339342F8D104226B6228466A6043
:10945800D8F81420002A92FAA2F34FF00202B3FAC5
:1094680083F308BF4FF0FF332B610023AB60C5E9DE
:109478000523C5E90733D8F82020022A0ABF4FF090
:1094880080731A464FF08052EB600023EA62EB6368
:10949800C5E90C3302F0D0FF014608B1704AA4E7D1
:1094A80018220EA85EF063FD2B686E4A934215D110
:1094B8000123CDE90E3310934FF00113119303F5F7
:1094C8007F031293012641F288320EA9284613968B
:1094D80003F0DEF8814658B1634A86E7634A93424F
:1094E800F0D10223CDE90E33109303F58033E5E77D
:1094F8003246314605F15C0045F024F832464946CB
:1095080005F1740045F01EF8D8F810302046984749
:109518002769502249462EA85EF029FD662341F2AC
:1095280088322EA93846CDE9303643F074FB30B185
:109538004F4A3146444842F0C7FB4E4A55E7992303
:1095480041F288322EA93846309343F064FB08B1C3
:10955800494AEEE7042346F2996A339041F2883289
:10956800319310232EA93846CDF8C0A0329343F08A
:1095780052FB08B1414ADCE749F6661941F28832E4
:109588002EA93846CDF8C09043F045FB08B13C4AB7
:10959800CFE7082341F288322EA938463393CDF815
:1095A800C0A043F038FB08B1364AC2E741F288321E
:1095B8002EA93846CDF8C09043F02DFB039008B192
:1095C800314AB6E7314844F095FD324631462846DF
:1095D800FFF76CFB08B12E4A07E7D4F80490276917
:1095E800D9F81C30082B16D0D9F82030012B12D10D
:1095F800182314AA00212046FFF7A6FB834600285B
:1096080000F0FA806FF0150222490F486FF0150B31
:1096180042F06AFBC8E6012238461146FFF7D8FA3D
:10962800064600283CD01C4A0121074842F04CFB62
:10963800D8E90732012100920348184A3FF041FF58
:10964800D7E600BF477F0708388B0608707F0708F2
:109658000C8606088F7F0708AB7F0708CE7F0708B0
:10966800FD7F0708005000520E80070800A0005236
:1096780023800708F58007084680070869800708DF
:109688008C800708AF800708D2800708A0860100F1
:10969800078107082D8207081D8107080982070826
:1096A800012207232EA84FF0720A11468DF8683060
:1096B800FFF716FA4FF440733F96012641F28832BD
:1096C8002EA93846CDF8C0A034933D9643F0A3FAAE
:1096D80030B1A54A3146A54842F0F6FAA44AA3E7B4
:1096E80041F288321AA9384643F0E6FA0028F0D148
:1096F800324631463846FFF7D9FA08B19D4A93E712
:10970800324631463846FFF763FA834608B19A4A2B
:109718008AE7D9F82030324631462EA8022B14BFEA
:10972800012302238DF86830FFF7DAF941F2883215
:109738002EA93846CDF8C0A0CDF8D0B0CDF8FCB0F1
:109748003D9643F068FA08B18C4AC3E741F2883283
:109758001AA9384643F0B0FA0028F5D149F6404036
:1097680044F0C8FC4FF080733846FB604FF08053DC
:10977800FB6202F061FE08B1814A55E7D9F820A0E2
:10978800BAF1010F2BD1524608213846FFF78EFA5D
:10979800064608B17B4A47E7012208212EA8FFF7B1
:1097A8009FF947F28E1341F288322EA93093042391
:1097B800384634963F93CDF8F4A043F02CFA30B1F4
:1097C8006E4A0121694842F07FFA6F4A2CE741F25C
:1097D80088321AA9384643F0B5FA0028F0D1D9F8EA
:1097E8002020022A7FF404AF08213846FFF75EFAEA
:1097F80000283FF4FDAECDE7149A644B9A4201D09D
:10980800634902E79DF8563016AE012B96BF013327
:109818001023DB00F3180693069BB3426ED0F2794F
:10982800337843EA0223B3F57F4F40F0CF81F378D2
:1098380071799B00B27909023079502B41EA0241D3
:109848001AAA28BF502301432046FFF77DFA0028B3
:1098580040F0B98127694FF001084E4B07F1940A8F
:10986800D4F804900B93ADF824008DF82600C7F8BF
:109878009400C7F898005FFA88F108F10108524689
:109888001AA842F0A0F9B8F1050F0AF1020AF2D1BC
:109898001A9BC3F34148236908F1FF32012A50D8C3
:1098A8000422B8F1010F83F89E204DD10DAA1AA900
:1098B8003046FFF7F7F8002846D19DF8343098076E
:1098C80042D0414642462EA80493D4F810A0FFF790
:1098D80007F9049B990763D5424641465046FFF76E
:1098E80077F900285CDA2C4A0121204842F0ECF98B
:1098F8006FF0040229491D4842F0F6F922696368AD
:10990800B2F89C0002F108055969134693F894408F
:1099180034B1039E93F895400EB1B44200D203943B
:1099280002339D42F2D1039C0123A3405C1E0442F2
:1099380008BF0346C2F89030B1FBF3F3C2F88C308D
:1099480032E5032283F89E20D7F8A430FF2B47D1B5
:10995800D9F81C30042B00F09780082B3CD0022B40
:1099680000F09480022339E036810708388B060816
:10997800458107085D8107087581070890810708F8
:10998800B6810708D4810708EB810708534644507D
:1099980042820708030604075A820708D982070883
:1099A800B72201232EA95046CDE93023002341F2E6
:1099B800883235933C933F9343F02DF9002892D198
:1099C8000CAA0321204642F09BF900288BD19DF870
:1099D8003030DB0787D5B7E741F2ED23C7F8A4306D
:1099E800D9F81C30082B00F0DF8002234FF0000864
:1099F80087F8A830032387F89F80C7F8A030D9F8E4
:109A08001C30012B00F0D080022B14BF4FF0040A49
:109A18004FF0020A0BAB1AA9304613F8082009AB1D
:109A2800049242F05CF800280DDB049A9DF824307B
:109A380087F8A820C7F8A0309DF825209DF8263083
:109A4800134487F89F3008F10108D045E2D1D9F8CE
:109A58001C30042B40F0A8800CAA1AA9304642F00A
:109A6800C6F8002814DA704A0221704842F02CF92E
:109A78002369049393F8A930062B72D8DFE803F022
:109A880094730F78737373003823A7E7A223A5E7AD
:109A98009DF83030C3F3420387F8A930E8E74FF068
:109AA80040094FF001080DF123024146204642F0DB
:109AB80027F9002855DB9DF8233019EA030305939D
:109AC80072D1012204981146FFF782F8002848DB7A
:109AD8009DF823A0502223692EA849EA0A0A05996D
:109AE80007938DF823A05EF042FA4FF080720123AD
:109AF8003C929845059A0D92079ACDE9303392F831
:109B0800A92038D19A428DF834A047D10DF13502F9
:109B18000221204642F0F4F8002822DB0DAA022395
:109B28002EA92046FFF71AFB00281ADB0122049809
:109B38001146FFF7BBF8002813DB0DF1230241465D
:109B4800204642F0DDF800280BDB9DF8233019EAA7
:109B5800030F29D1364A01210093434633483FF089
:109B6800B0FC344AC0E64FF002094FF002089AE709
:109B78004FF08009F9E73121012A8DF835A030919D
:109B880002D0043A012A0CD80DAA0121204642F03D
:109B9800B7F80028E5DB01233093BFE70DAA434659
:109BA800BEE70DF13502BBE7F3780A2B89BF249B8A
:109BB8004FF48073C3F30312012388BF9340A7F8BF
:109BC8009C30083628E66FF0150293E64FF684724B
:109BD8009342F6D195F89E30042BF2D1F37871793F
:109BE8009B00B27909023079082B41EA02412EAA7A
:109BF80028BF082301432046FFF7A6F800287FF472
:109C08007DAE0DF1BB012B4605F1080711F8012FB8
:109C18000233FF2A04BF002283F8930083F89220BE
:109C28009F42F3D1CDE700BF73820708388B06083F
:109C38009A820708BE82070800487047D894060829
:109C4800044BB3F80C389B020B60002318464B609A
:109C5800704700BF00F0FF08064B186828B94FF49A
:109C6800807C4FF40050C3E900C0012010600B60F5
:109C7800704700BF983E002407B503461022012113
:109C880004480092044A3FF01CFC002003B05DF831
:109C980004FB00BF408B06080F8307080B4A536973
:109CA800DB0312D5002910DD00F1006300F01F006E
:109CB8000144BFF34F8F2039C2F85C3220330029AA
:109CC800F9DCBFF34F8FBFF36F8F704700ED00E0F3
:109CD80037B50468256915F0C06F09D0236E9BB2AB
:109CE8001D4A02211D481B01009301233FF0E9FB97
:109CF8001B4B63611B4B1D4209D00123009517487C
:109D08000121194A3FF0DDFB6FF004001EE0D4F892
:109D1800105115F0064F0AD0D4F860319BB20E4AA4
:109D28000E481B010093022319463FF0CAFB0F4B54
:109D3800C4F814310B4B1D4207D00D4A154207D009
:109D4800D4F814311343C4F81431002003B030BDE3
:109D580002230095D3E700BF61830708408B0608FC
:109D68000F00AF1F0000AE157C8307080F00AF9FE0
:109D78000000088070B5054610461A46EFF31186B4
:109D8800102383F31288BFF36F8F012383F31388A3
:109D9800104C636943F480736361BFF34F8FBFF363
:109DA8006F8F01F100615EF0BBF8002383F3138825
:109DB800636923F480736361BFF34F8FBFF36F8FC1
:109DC80086F31188BFF36F8F2869BDE87040FFF7ED
:109DD8007FBF00BF00ED00E0F7B517461A460646FC
:109DE8000D461C4642F035F850B90B482B460B4A35
:109DF800012100943FF065FB6FF0150003B0F0BD42
:109E080044B123463A462946304603B0BDE8F040FF
:109E1800FFF7B0BF2046F1E7408B0608928307089A
:109E2800F7B505463C220023684644F0ADFD286995
:109E3800DDE90067FFF74CFF044680B902462B694D
:109E48001B681969490703D4D3F810315B0708D593
:109E580052B106230A4A01210A483FF028FB6FF055
:109E68000404204603B0F0BD32463B46684644F041
:109E7800B0FDDDE9003213430CBF01220022DEE70A
:109E8800BC830708408B060810B503691C6829B114
:109E9800FFF7C6FF88B16FF0040019E0E368DA073E
:109EA80017D4D4F80C31DB0711D50D4BC4F80431A5
:109EB80003F18833C4F8043109E0E36843F001038F
:109EC800E360D4F80C3143F00103C4F80C310020EE
:109ED80010BD034B636003F188336360E1E700BFA3
:109EE800230167452DE9F84F0369B1F5801F9146B5
:109EF800314A1E688046926901F1006A35BF06F151
:109F08000C0706F58677103606F588763C6814F057
:109F1800010403D06FF00400BDE8F88FFFF780FF5D
:109F28000028F7D1DAE90023B3F1FF3F08BFB2F107
:109F3800FF3FEFD1DAE90223B3F1FF3F08BFB2F1E7
:109F4800FF3FE7D13B6843F002033B60BFF34F8F0D
:109F580009EB040159F804204B680AEB0401C1E934
:109F68000023BFF34F8F44F00DFD0A220023F6F7BC
:109F7800D5FA10F1640541F1000B33685B070FD582
:109F880044F000FD0A220023F6F7C8FA85427BEB6D
:109F98000101F2DA6423094A012109483FF087FAEE
:109FA800082C07D14046FFF73BFF3B6823F002032C
:109FB8003B60B1E70824CBE700200052D0830708B4
:109FC800408B0608013A2DE9F04781468A46571822
:109FD800DFF87C801D4E574501D2002012E0D9F8E9
:109FE8001030BAF5801F4FEA5A351C68D8F8183077
:109FF8002ABF803D0C3404F586742368DB0703D53B
:10A008006FF00400BDE8F0874846FFF709FF002815
:10A01800F6D12368AD0123F4FE5305F4FE55236001
:10A0280023681D4345F004052560236843F0200399
:10A038002360BFF34F8F4846FFF7F2FE2368334093
:10A0480023600028DCD10AF5005AC4E73BE0FFFF93
:10A05800002000522DE9F743012307460C46154618
:10A0680041F00CFF60B900956FF0150523461D4AB5
:10A0780001211D483FF025FA284603B0BDE8F083CA
:10A08800002DF9D0386941F0DDFE00213846FFF790
:10A09800FBFE18BB154E21462A46384604EA060937
:10A0A80004F5FF54FFF78EFF80461E3448462C44C3
:10A0B80004EA0601A1EB0901FFF7F0FD012138468A
:10A0C800FFF7E2FEB8F1000F08BF0546386918BF70
:10A0D8006FF00405043005F07BF8CDE76FF0040855
:10A0E800ECE700BFE1830708408B060800E0FFFFAC
:10A0F800F7B51C4617460123054622460E4641F091
:10A10800BDFE58B96FF015073346184A01211848A3
:10A1180000943FF0D6F9384603B0F0BD24B328695F
:10A1280041F090FE00212846FFF7AEFEC8B93A4636
:10A1380023463146284641F0AEFE0746012128460F
:10A14800FFF7A2FE002F214608BF0746304618BF7A
:10A158006FF00407FFF7A2FD2869043005F038F80E
:10A16800D9E76FF00407E9E72746D4E70C84070826
:10A17800408B06082DE9F843D0F80490904607462E
:10A188000D46D9F808001E4640F0B7FDB8F5001F87
:10A19800044616D1D9F808402846FCF7FBFC84424F
:10A1A8000CD1294640F0A9FD044640F0ABFD2046FD
:10A1B800FCF7DEFC0021204640F0ADFD0020BDE8A4
:10A1C800F883B8F5800F20D0B6F1806F19D0B6F1BA
:10A1D800C06F18D0B6F1007F1AD102263A460F494F
:10A1E8002046FCF7A5FCB0B9D9F80810284640F07D
:10A1F800BBFD2046314640F08EFD2046FCF780FC32
:10A20800DCE70126EAE70326E8E76FF08500D6E7F2
:10A218006FF01500D3E76FF00F00D0E72FC00408E8
:10A228001FB50C4B0C29D3F8082828BF0C2112BAEB
:10A238000C460192D3F8042812BA02920A46D3F8BF
:10A24800003801A91BBA03935DF06AFE204604B0EA
:10A2580010BD00BF00F0FF08174AD2F83031D2F81D
:10A268003011C3F300634902D2F830114FEA4303B7
:10A27800D2F8302148BF43F00103490148BF43F0F9
:10A288001003D2000C4A48BF43F01003D2F8301133
:10A29800D2F83021890248BF43F004031102074A6B
:10A2A80048BF43F008031269520648BF43F08003D1
:10A2B80003600020704700BF00440258004802585D
:10A2C80080B500AF8AB06A46094B0791CDE90530E1
:10A2D8004FF40073ADF82030064B42F8103F0023CE
:10A2E8004FF411510448F8F71FF8BD4680BD00BF70
:10A2F8006384070804000001708B06082DE9F74302
:10A3080098460B7A1646046943F0040307460D463F
:10A3180001220B720B46B2421AD904F118094FF008
:10A32800FF324FF0FF33484604F08EFF384641F0C5
:10A33800C8FE041E2DDA1B4A234601211A483FF0A5
:10A34800B6F8484604F044FF204603B0BDE8F08361
:10A358000AD2197A187D81EA000C1CF0010F01D08D
:10A3680040071CD589071AD401320C33D2B2D2E780
:10A37800012E384614BF05F114030023CDE9003837
:10A3880095E80E0041F040FF041E04DB013E0C3549
:10A39800F6B2002EECD1384641F095FED1E76FF0C9
:10A3A8001504D1E777840708708B060808B5044AB6
:10A3B800012104483FF072F86FF0040008BD00BFA7
:10A3C80093840708708B0608F7B542680023044693
:10A3D8000F460669D5685168214892680193012A99
:10A3E8008368DB6833D908314BB91E4A6FF004041F
:10A3F80001211D483FF052F8204603B0F0BD01AAE4
:10A4080098470028F1DB376306F118074FF0FF3251
:10A418004FF0FF33384604F017FF2B68204623F02F
:10A4280001032B6096F8621041F021FE2046019945
:10A4380000F0BEF8041E06DB96F861301BB12B68ED
:10A4480043F001032B60384604F0C2FED4E70BB991
:10A45800064ACBE701AA98470028D4DAF8E700BFF4
:10A468000C860608B1840708708B0608DF84070885
:10A47800F8B50446466805694FF0FF320021002709
:10A48800284644F05FF833682046984785F860709E
:10A4980085F86270012205F11800114644F052F85F
:10A4A800204600F051F8B368012B25D831691F4BBD
:10A4B800994230D014D81E4B99422ED01D4BCB1A3E
:10A4C800594259418900204641F01001FFF77CFFAD
:10A4D800041E26DA184A012118483EF0DFFF13E06F
:10A4E800174B99421BD003F5C31303F52063994218
:10A4F8000CBF0A210021E6E7124871688368083119
:10A508009B691BB96FF004042046F8BD3A4698478A
:10A518000028CBDAF6E70621D5E70221D3E70821A0
:10A52800D1E70123002485F86030EDE740420F00B1
:10A53800A0860100801A06000D850708708B0608A2
:10A5480040E133000C86060837B5456801AA0021AA
:10A55800286A41F062FF041E07DB019B002219797B
:10A56800186841F06CFF041E08DA0D4A23460121E1
:10A578000C483EF09CFF204603B030BD0A4869688D
:10A5880083681B683BB9094A012106486FF0040437
:10A598003EF084FFEFE7984704460028EBD0F2E747
:10A5A80031850708608B06080C8606084F85070862
:10A5B8002DE9F04F446885B003694FF00C0EE5684B
:10A5C80000200393DFF82881A36ADFF82891DFF8D9
:10A5D80028A1DFF828B10293029B8342039B1B6BDF
:10A5E80001930DD1C3F34202012A39D0022A66D061
:10A5F8003A4A3B4801213EF051FF6FF015001DE03B
:10A608000EFB00F7D4F824C0364A0CEB0706736833
:10A6180093421DD015D853451CD0A3EB0B025342CF
:10A6280053419B00019A534013F00E0F16D15CF86A
:10A6380007308B4212D1B36800202B6105B0BDE80A
:10A64800F08F434508D04B450CBF0A230023E9E7A8
:10A658000623E7E70223E5E70823E3E70130BBE742
:10A6680041F25C2E4FF47A6C40F2E2474FF4FA76EE
:10A6780002201D4B421EB1FBF2F2B3FBF2F2BCFB0F
:10A68800F2F4013CFF2C23D8BEFBF2F808F1FF38A6
:10A69800B8F1FF0F1CD8B6FBF2F9B9F10F0F17D8B4
:10A6A800B7FBF2F2013A0F2A12D8023848EA0943F6
:10A6B80043EA007343EA025343EA0423BCE740F247
:10A6C800145E4FF4167C4FF4FA7740F27716CFE712
:10A6D80001301128CED1054A8BE700BF8C850708C9
:10A6E800688B060840420F0000CA9A3B0786070895
:10A6F80040E13300404B4C00A0860100801A060060
:10A7080037B5456801AA0021E86841F086FE041EB5
:10A7180007DB019B00221979186841F090FE041E9E
:10A7280008DA0C4A234601210B483EF0C0FE2046B9
:10A7380003B030BD0948696883681B682BB1984726
:10A74800041E05DA064A2346EDE76FF05704F9E7D9
:10A758000024ECE73A860708908B06080C86060862
:10A768005886070843681B6803F1080252E8002F5F
:10A7780042F0010203F1080040E800210029F3D16A
:10A78800194A934223D0A2F54C4293421FD002F5B6
:10A79800806293421BD002F58062934217D002F583
:10A7A8008062934213D002F5444293420FD0A2F53F
:10A7B8001C4293420BD002F58062934207D002F507
:10A7C8001C42934203D002F58062934203D15A6837
:10A7D80042F040025A6053E8002F42F4807243E886
:10A7E80000210029F7D170470010014043681B6819
:10A7F80003F1080252E8002F22F0010203F10800D9
:10A8080040E800210029F3D1194A934223D0A2F548
:10A818004C4293421FD002F5806293421BD002F54E
:10A828008062934217D002F58062934213D002F5FA
:10A83800444293420FD0A2F51C4293420BD002F53A
:10A848008062934207D002F51C42934203D002F57E
:10A858008062934203D15A6822F040025A6053E85A
:10A86800002F22F4807243E800210029F7D17047B5
:10A87800001001402DE9F04182B080460D46436842
:10A8880000AF1E68002937D0586819698368DB68EB
:10A898006BB13A1D9847041E0CDA1B4A01211B486C
:10A8A8003EF0FCFD20460837BD46BDE8F0816FF05C
:10A8B8005704F2E7336823F4004333607B6803EB03
:10A8C8005503B3FBF5F30F2B19D86C468AB0D8F8AB
:10A8D80000306A460E490795CDE905134FF4007319
:10A8E800ADF820300B4B42F8103F00234FF41151C4
:10A8F8000648F7F719FDA5466FF01504D2E79BB295
:10A908000024F360CEE700BFDF840708088C060840
:10A91800C486070804000001F8B50C4603694168BD
:10A928001D682379012B18D0A3F1020EDEF1000671
:10A9380046EB0E06B6026279022A96BF464F4FF4DE
:10A94800005737F81270A279022A09D0042A2FD0AA
:10A95800003B18BF01231B0306E04FF4C066EAE77B
:10A96800B3FA83F35B091B07E2790968012A0CBF74
:10A978004FF4407C4FF0000CA5421CD10A6822F02D
:10A98800805222F4B05232431A430A604B6823F4CF
:10A9980040533B434B6043681A68936823F4407301
:10A9A80043EA0C0393602968BDE8F840FFF762BFEB
:10A9B8004FF48053D8E7D1F800E00EF4C06E764526
:10A9C80006D0D1F800E02EF4C06E4EEA06060E60FE
:10A9D80041680E68716801F440518F4204D0716873
:10A9E80021F440513943716041680E68316801F0C3
:10A9F80010218B4204D0316821F010210B433360C1
:10AA0800436819688B6803F440739C4505D08B68CC
:10AA180023F4407343EA0C038B604368D71E1B681A
:10AA28007E4299687E41C1F380318E4207D0032A65
:10AA38009A680CBF42F4804222F480429A602168EE
:10AA48002B68994205D0FFF715FF08B923682B60DA
:10AA5800F8BD0020FCE700BFD65907082DE9F043F0
:10AA680083B08046D0F8049000AFD9F80400D9F834
:10AA7800101083681B687BB19847054670B93A1D6A
:10AA88000021D9F8240041F0C8FC051E0EDA28463A
:10AA98000C37BD46BDE8F0836FF05705644A0121C5
:10AAA80064483EF0FBFC002DF1DBE8E77B68002200
:10AAB8001979186841F0C3FC051EE8DBD8F8046072
:10AAC800D8F8103034681D68236823F00103236028
:10AAD800B06843F036FB38B9574A012155486FF042
:10AAE80012053EF0DBFCD2E7D6E902018368DB6899
:10AAF80003B1984754E8003F43F00C0344E80032A0
:10AB0800002AF7D129464046FFF706FF054610B14F
:10AB18006FF01505BBE7337E1BB1A36843F008034C
:10AB2800A360737E1BB1636843F400436360B37E24
:10AB38001BB1636843F480336360F37E1BB16368C1
:10AB480043F400336360337F002B5BD03B4B9C4264
:10AB58003DD0A3F54C439C4239D003F580639C4219
:10AB680035D003F580639C4231D003F580639C4265
:10AB78002DD003F544439C4229D0A3F51C439C42A5
:10AB880025D003F580639C4221D003F51C439C42E9
:10AB98001DD003F580639C4219D0294B9C4216D0E6
:10ABA8006C4688B0D8F800306A462649CDE90513C6
:10ABB8004FF40073ADF81C30234B42F8103F0023CC
:10ABC8004FF4E2511B48F7F7AFFBA546A0E7D8F8CA
:10ABD80004301A68936843F4804393602368727F53
:10ABE80023F0787343EA425323602368B27F23F447
:10ABF800F81343EA02432360F37F1BB1A36843F4CD
:10AC08000043A36096F820301BB1236843F000533B
:10AC18002360236843F001032360E3699A02FCD5AB
:10AC2800E3695B02FCD5D9F82830404698472EE7FF
:10AC3800DB860708088C0608FB8607080010014019
:10AC4800000C005816870708030000012DE9F041A1
:10AC5800436802460D461C6803691E680B79012B80
:10AC680017D0981E41424141890295F805E0AF7915
:10AC7800BEF1020F96BF40484FF4005C30F81EC08A
:10AC8800022F09D0042F01D0002B6BD04FF4805035
:10AC980005E04FF4C061E8E7002B60D00020A3F185
:10ACA8000308B8F1010F04D86FF085031846BDE812
:10ACB800F0810BB1042FF7D0BCF5805F54D0BCF500
:10ACC800405F53D0BCF1000F0CBF012303239E4506
:10ACD800EAD141F008FC8742E6D1EB795BB3012B5E
:10ACE80046D1264B9C4226D0A3F54C439C4222D009
:10ACF80003F580639C421ED003F580639C421AD002
:10AD080003F580639C4216D003F544439C4212D05D
:10AD1800A3F51C439C420ED003F580639C420AD0E5
:10AD280003F51C439C4206D003F580639C4202D085
:10AD3800134B9C42B8D123682946104623F00103DF
:10AD48002360FFF7E9FD03460028ADD1226842F0F1
:10AD58000102226095E8030086E80300A6E74FF0A9
:10AD68008050A9E71846A7E70023B0E70223AEE71B
:10AD7800032BB6D098E700BFD6590708001001404A
:10AD8800000C005870B50B6806460C46988841F0D0
:10AD980058FD04280346D1E9191510D002280AD114
:10ADA800012A01D9012D0AD8328E92B209B105B112
:10ADB8000A80022508E0032A12D9032D12D9326B22
:10ADC80009B105B10A600425B5FBF3F5A26E2AB1F5
:10ADD800954213D91649174841F06FFD284670BDB2
:10ADE800012A02D9A26E012ADED896F83020D2B202
:10ADF80001B10DB90125E9E70A70FBE7521BA2660C
:10AE08007AB9226D04F1540104F150000832226528
:10AE1800626D013A626504F1680241F0EEFC606619
:10AE2800DCE7626E002AD9D005FB03226266D5E70B
:10AE380063870708D08B06082DE9F84306460C46B9
:10AE480091F8749004274FF002082368988841F01D
:10AE5800F8FC04280346E26D17D002280FD1B9F197
:10AE6800010F02D9216E01290FD8002A39D0216E8D
:10AE780001B1118889B2B8FBF3F531840CE0B9F15E
:10AE8800030F1FD9216E03291FD9CAB1216E01B141
:10AE980011683162B7FBF3F5226E2AB1AA4224D2B7
:10AEA8001F49204841F009FDE36E5B1BA9EB05052E
:10AEB80015F0FF09E36601D0002BC6D1BDE8F88381
:10AEC8001146E6E7B9F1010F02D9216E0129CCD864
:10AED8004AB1216E01B11178C9B2012586F8201056
:10AEE800DAE71146C6E71146F6E7521B22667AB939
:10AEF800A26C04F14C0104F148000832A264E26C2F
:10AF0800013AE26404F1600241F077FCE065CBE7C6
:10AF1800E26D002AC8D005FB0322E265C4E700BF42
:10AF280063870708D08B060808B502B933B104480F
:10AF3800044941F0C2FC6FF0850008BD1846FCE7E3
:10AF4800D08B06088187070870B5436805460669EF
:10AF5800DA68012A12D91E489968836808319B6902
:10AF68004BB100229847041E08DA1A491A4841F0E2
:10AF7800A4FC204670BD6FF05704F6E7336923B987
:10AF8800736006F1080004F023F90121686841F0B4
:10AF9800ACFC041E02DA14F1860FEAD16D680021B8
:10AFA800284641F0A2FC041E0BDB0948A968836807
:10AFB8001B684BB19847044618B10849064841F048
:10AFC8007CFC04EAE474D4E76FF05704F5E700BFAB
:10AFD8000C860608AF870708D08B0608D1870708B4
:10AFE8002DE9F04F87B080460E469B46914600AF4C
:10AFF800056932B92BB9002630461C37BD46BDE875
:10B00800F08FB3889A0400F11C814FF0FF324FF0A3
:10B01800FF3305F1080004F017F96E60002385F886
:10B028004430C5E90F33D8F81030D8F804A0FB60D5
:10B038001B68DAF800409E42B28840F00E81130582
:10B0480008D5B9F1000F00F005814FF4C121204661
:10B0580041F0C4FBB08841F0F4FB0346B9F1000F9E
:10B0680040F07D81C5F848900022EA6405F14C0162
:10B0780005F1600205F14800FB6041F0BEFBFB688A
:10B08800E865BBF1000F40F07381C5F850B00022AD
:10B098006A6505F1540105F1680205F1500041F0B7
:10B0A800ACFB002368661A46E86CAB63824240F04A
:10B0B80068810022D5F854C01146614540F0688186
:10B0C80093422CBFAB65AA652B6E3BB9AB6E2BB90F
:10B0D800EB6E1BB92B6F002B00F02B822268E36804
:10B0E80002F4006203F4C0231343BB60D8F80430B1
:10B0F8007B601B68FB60FA681B68D26803F4006316
:10B1080002F4C022134340F04A814946304641F0D8
:10B11800B2FB81465946304641F0ADFB81454E466B
:10B12800B8BF0646002EC0F2AA807B681B6AB342ED
:10B13800C0F03F81FB68D8F810101B68DB0702D508
:10B14800F86841F070FBFB68FA685B686FF30F03FF
:10B1580033435360C1E91B66D8F804301B681A688A
:10B1680042F001021A60DA68500200F129810120D8
:10B1780042F0C0FF2B6E2BB9AB6E1BB9EB6E0BB94F
:10B188002E6F3EB32946204641F0C4FB636913F491
:10B19800787300F035816E468AB06A468D4905910C
:10B1A8008D49CDE906134FF40073ADF820308B4B71
:10B1B80042F8103F00234FF411518948F7F7B4F8CB
:10B1C8006369B5465A0603D5A36943F04003A361F2
:10B1D8006FF00406D8F80430D8F8104019684B69A5
:10B1E800DB0700F16C81CB68580240F16B81DFF816
:10B1F8000C92084641F030FB002800F063810B6890
:10B20800DB0740F15F814B689BB263B923689B8879
:10B21800C3F34513192B06D829FA03F3DA0702D525
:10B22800084641F000FB0B68CA6803F4006302F4A7
:10B23800C0221343B3F5C02FDBD1084641F0F3FA1F
:10B24800D7E72B69002B7FF4E0AE6B689E427FF452
:10B25800DCAEE3E64FF4C021F9E6DAF81010C2F3E9
:10B268004513022918D0032919D0012935D1043BE7
:10B278001C2B8CBF00230123ABB96FF0850695F812
:10B28800443013B1002E3FF4B6AE00236B6005F1D5
:10B29800080003F09DFFAFE6043B0C2BE9E7082B01
:10B2A80001D0102BE9D1100405D5E36823F460130D
:10B2B80043F40023E3604B48DAF80C208368012A42
:10B2C800DAF80810DB6833D908315BB946494448D5
:10B2D8006FF0040641F0F1FAD1E74449404841F0E3
:10B2E800ECFACAE707F1140298470028EEDB7B69FD
:10B2F800002230681146013223FA02FC844540F2EC
:10B308001A81082AF6D16C468AB06A463849CDE9CE
:10B31800051059081B0A07910893052342F8103FA6
:10B3280000234FF421512E48F6F7FEFFA54644E0CE
:10B338000BB93049CBE707F1140298470028D6DA51
:10B34800F7E74FF4C02127E11BB1E36823F010535E
:10B358004AE1E36823F0105343F0005344E1D9F87D
:10B368000020AA64002A3FF47FAED9F804207CE6C6
:10B37800DBF800202A65002A3FF489AEDBF80420B8
:10B3880086E6A96C01EBC201013249680B448DE6DF
:10B39800286D00EBC1000131406802448DE6B3F529
:10B3A800C12F30460CBF4946594641F064FA06465B
:10B3B800B8E611490A4841F080FA6FF015065EE7D1
:10B3C8001A6842F400721A601A6891053FF5CFAE08
:10B3D800FAE700BF988807082ECD07080400000187
:10B3E800D08B06080C86060814880708EC8707081F
:10B3F800A3880708408807086C880708000202022B
:10B40800BB68B3F5C12F7FF4B5AE2B6E002B33D1DB
:10B41800AB6E8BB3DAF80060304641F01DFA014696
:10B428000028F9D1304641F0FEF92B689888C30707
:10B4380013D4D5F854C00B46634528D141F001FA1E
:10B4480091FBF0F300FB1313002B32D17368B1FBAF
:10B45800F0F16FF30F031943716030464FF4C021C8
:10B4680041F0BCF9336843F001033360F3685802D4
:10B4780014D4012042F03EFE00212268E368D9B9C5
:10B4880002F4006203F4C0231343BB6072E62A6D22
:10B4980002EBC302013352681144CDE7336843F429
:10B4A8000073336033689905E3D473691A07E0D4ED
:10B4B800F8E76FF01501E0E76FF015068AE691F8F6
:10B4C80030308CE64B69980503D58B6943F40073DB
:10B4D8008B618B6943F010038B618B6943F04003E8
:10B4E8008B618B6943F008038B614B686FF30F0323
:10B4F8004B6023689B88DA0402D4084641F093F92C
:10B5080094F844302BB9A66304F1200003F060FEE0
:10B51800B5E6E36B1BB1226C314640469847236879
:10B528009B8813F400537FF4AAAE636004F108000B
:10B53800ECE71E46A3E6204641F075F9A3684B4A9E
:10B5480023F0E04352F821201343A3609AF82530F2
:10B55800DB0703D5E36843F40043E360B38813F0E3
:10B56800020FE36814BF43F0007323F00073E36035
:10B57800B38813F0040FE36814BF43F0807323F01B
:10B588008073E360B18811F4006105D0B9F1000F50
:10B598003FF4D7AE4FF4C121204641F01FF9B388DC
:10B5A80013F0100FE36814BF43F4000323F40003FF
:10B5B800E360A36823F48003A360B388327D03F0BB
:10B5C800010322B99AF8252091077FF5BDAE33B95A
:10B5D800E368DA0003D4236843F480532360E36804
:10B5E80023F0105343F08063E360B388204913F0DD
:10B5F800010FE36814BF23F4800343F48003E3607E
:10B60800B288A368C2F3451223F01F03043A51F825
:10B61800222018491343A360E368DAF81C2023F0BA
:10B628000F031343E360E368DAF8182023F0F0030C
:10B6380043EA0213E360B288DAF81430C2F3451221
:10B648000732D20893FBF2F3012BFA68B8BF012343
:10B6580082F87430DBB2A268013B22F4F07251F830
:10B6680023301343A360FB681E60F3E4B896060812
:10B6780070970608309706084FF0E02310B59969CF
:10B688001C699B6900B103600B4A0C4812680029C9
:10B6980008BF1146002B08BF134614F4803F01D1A0
:10B6A800994205D20168114401604FF0E02109690F
:10B6B80000681044C01A10BD203F0024143F002425
:10B6C8000B4B1022002083F823204FF42F62094BE4
:10B6D8001A6046F66052084B1A6046F65F52074BEE
:10B6E80018604FF0E0235A61072298611A61704789
:10B6F80000ED00E01C3F0024203F0024143F0024FC
:10B70800684620F007018D46F1B541F054F904462A
:10B7180000200027FFF7B0FF1248134A03680760AC
:10B72800D2E900515B19114D41F10001C2E9003124
:10B73800D5E9006146F660529B1BB3FBF2F002FBB1
:10B7480000F39B1941F10001C5E90031084B21467E
:10B758001F6004F0EBFCF7F709FEBDE8F1408546F1
:10B76800704700BF143F0024C8330024C0330024AE
:10B77800183F00242DE9F341804601A8FFF77CFF1C
:10B7880026490027264A274E17603568D1E9003434
:10B79800C3182548D0E9002044F10004B3EB020C9B
:10B7A800C1E9003464EB0004204BBC4218681ADB82
:10B7B8001F4B46F6605E1B6813EB080347EB070850
:10B7C800A3FB0E32B3EB0C030EFB082262EB040260
:10B7D8009842974107DAB3F1807F72F10002A8BF5F
:10B7E8006FF07F43184630604FF0E02301380022A5
:10B7F8009C6958619A614FF00072C3F8042D019B4F
:10B80800A34238BF5B19D1E900201B1B9A1840F1ED
:10B818000000C1E9002002B0BDE8F081C83300246F
:10B82800143F0024203F0024C03300241C3F002480
:10B83800183F0024084B002010B51C68074B1B68F4
:10B84800E41AFFF719FF46F660532044B0FBF3F003
:10B85800034B186010BD00BFC8330024C033002458
:10B86800183F002438B541F0A6F8064B04460020DE
:10B878001D68FFF701FF84F31188BFF36F8F284419
:10B8880038BD00BFC833002410B541F094F8044611
:10B898000020FFF7F1FE054AD2E90031C01841F156
:10B8A800000184F31188BFF36F8F10BDC8330024E3
:10B8B800494B30B51A6902F03802102A00F0888026
:10B8C800182A0CD0002A40F085801A68434812F0E4
:10B8D800200F03D01B68C3F3C103D84030BD996A59
:10B8E8009D6ADC6A15F47C7FC5F305105A6BF5D0A8
:10B8F800C2F3CC0204F0010401F0030107EE900A40
:10B908006243B7EE006A0129B8EEE77A06EE902A9C
:10B91800FAEEE96A4ED002293ED000294AD11A68C7
:10B92800920627D519682D4AC1F3C1011B6BCA407D
:10B93800C3F3080307EE902AF8EEE75AC5EE877AB4
:10B9480007EE103AB8EEC77A37EE267A37EE067A5F
:10B9580067EE877A204B1B6BC3F34623013307EE50
:10B96800103AF8EEC76A87EEA67AFCEEC77A17EEA9
:10B97800900AB3E71B6BC3F3080307EE903AF8EE9F
:10B98800E77A77EEA67A77EE867A9FED156AC6EEA5
:10B99800076A67EEA67ADDE71B6BC3F3080307EEB9
:10B9A800903AF8EEE77A77EEA67A77EE867A9FED08
:10B9B8000D6AECE71B6BC3F3080307EE903AF8EE49
:10B9C800E77A77EEA67A77EE867A9FED076ADEE762
:10B9D800064883E7064881E7004402580090D003F0
:10B9E8000024744C001BB74B0024744A00366E01C7
:10B9F80000093D0008B5FFF75BFF0B4A0B49936947
:10BA08009269C3F3032302F00F02CB5C03F01F0318
:10BA180020FA03F3885C064A00F01F0023FA00F0BE
:10BA28001060044A136008BD0044025840CD07085E
:10BA38007C0900248009002408B5FFF7DBFF054BCB
:10BA4800054ADB69C3F30213D35C03F01F03D84034
:10BA580008BD00BF0044025840CD070808B5FFF7ED
:10BA6800C9FF054B054A1B6AC3F30213D35C03F0F5
:10BA78001F03D84008BD00BF0044025840CD070846
:10BA88004F4970B58C6A8E6ACD6A16F47C3FC6F34E
:10BA98000533CA6B00F0908007EE903AC2F3CC03EE
:10BAA800C5F3001204F00304B8EEE77A5343012CFF
:10BAB800B7EE006A06EE903AFAEEE96A6ED0022C0A
:10BAC8005ED0002C6AD10B689B0647D50A688B6B41
:10BAD800C2F3C1013B4AC3F30803CA4007EE902AE8
:10BAE800F8EEE75AC5EE877A07EE103AB8EEC77A4D
:10BAF80037EE267A37EE067A67EE877A304A936B06
:10BB0800C3F3462307EE103AB8EEC77A37EE067A43
:10BB1800C7EE876AFCEEE66AC0ED006A936BC3F372
:10BB2800064307EE103AB8EEC77A37EE067AC7EE44
:10BB3800876AFCEEE66AC0ED016A936BC3F306639D
:10BB480006EE903AF8EEE66A76EE866A87EEA67A10
:10BB5800FCEEC77A17EE903A836070BD8B6BDFED11
:10BB68001A5AC3F3080307EE903AF8EEE77A77EE2D
:10BB7800A67A77EE867AC5EE876A67EEA67ABDE77B
:10BB88008B6BDFED125AC3F3080307EE903AF8EE19
:10BB9800E77A77EEA67A77EE867AECE78B6BDFEDBD
:10BBA8000C5AC3F3080307EE903AF8EEE77A77EEFB
:10BBB800A67A77EE867ADEE7C0E90033CCE700BFE5
:10BBC800004402580090D0030024744C001BB74B6B
:10BBD8000024744A4F4970B58C6A8E6ACD6A16F093
:10BBE8007C7FC6F305534A6C00F0908007EE903ACC
:10BBF800C2F3CC03C5F3002204F00304B8EEE77ADD
:10BC08005343012CB7EE006A06EE903AFAEEE96A61
:10BC18006ED0022C5ED0002C6AD10B689B0647D5EB
:10BC28000A680B6CC2F3C1013B4AC3F30803CA405C
:10BC380007EE902AF8EEE75AC5EE877A07EE103A33
:10BC4800B8EEC77A37EE267A37EE067A67EE877A45
:10BC5800304A136CC3F3462307EE103AB8EEC77A9E
:10BC680037EE067AC7EE876AFCEEE66AC0ED006A30
:10BC7800136CC3F3064307EE103AB8EEC77A37EEF3
:10BC8800067AC7EE876AFCEEE66AC0ED016A136CB5
:10BC9800C3F3066306EE903AF8EEE66A76EE866A35
:10BCA80087EEA67AFCEEC77A17EE903A836070BDED
:10BCB8000B6CDFED1A5AC3F3080307EE903AF8EE5F
:10BCC800E77A77EEA67A77EE867AC5EE876A67EE28
:10BCD800A67ABDE70B6CDFED125AC3F3080307EE33
:10BCE800903AF8EEE77A77EEA67A77EE867AECE77E
:10BCF8000B6CDFED0C5AC3F3080307EE903AF8EE2D
:10BD0800E77A77EEA67A77EE867ADEE7C0E900333F
:10BD1800CCE700BF004402580090D0030024744CC4
:10BD2800001BB74B0024744A4F4970B58C6A8E6A61
:10BD3800CD6A16F47C7FC6F305134A6B00F0908039
:10BD480007EE903AC2F3CC0305F0010204F00304B5
:10BD5800B8EEE77A5343012CB7EE006A06EE903A44
:10BD6800FAEEE96A4ED0022C5ED0002C6AD10B683C
:10BD78009B0667D50A680B6BC2F3C1013B4AC3F344
:10BD88000803CA4007EE902AF8EEE75AC5EE877A0C
:10BD980007EE103AB8EEC77A37EE267A37EE067A0B
:10BDA80067EE877A304A136BC3F3462307EE103ADF
:10BDB800B8EEC77A37EE067AC7EE876AFCEEE66A0F
:10BDC800C0ED006A136BC3F3064307EE103AB8EEF2
:10BDD800C77A37EE067AC7EE876AFCEEE66AC0EDE8
:10BDE800016A136BC3F3066306EE903AF8EEE66A4F
:10BDF80076EE866A87EEA67AFCEEC77A17EE903A58
:10BE0800836070BD0B6BDFED1A5AC3F3080307EEAE
:10BE1800903AF8EEE77A77EEA67A77EE867AC5EE6C
:10BE2800876A67EEA67ABDE70B6BDFED125AC3F39C
:10BE3800080307EE903AF8EEE77A77EEA67A77EEFF
:10BE4800867AECE70B6BDFED0C5AC3F3080307EEB9
:10BE5800903AF8EEE77A77EEA67A77EE867ADEE71A
:10BE6800C0E90033CCE700BF004402580090D0037B
:10BE78000024744A001BB74B0024744C1FB5A0F56E
:10BE880080730B4319D19F4B1A6D02F00702042AE5
:10BE980031D8DFE812F02000BF0005004E01450050
:10BEA800186810F0005005D0002301A80193FFF78F
:10BEB80091FE019805B05DF804FBA0F500730B43F3
:10BEC8001BD1904B1A6D02F4E072802AE8D00CD88E
:10BED800002A40F09F80186810F00070EAD0002314
:10BEE80001A80293FFF720FFF0E0C02A00F02181AB
:10BEF800B2F5807F14D00020DCE7A0F580630B4307
:10BF08002DD1804B1A6D02F46062B2F5806FC7D0F4
:10BF1800DED9B2F5C06F00F00C81B2F5006FE9E729
:10BF2800DA6C196802F04052480706D52AB91B682E
:10BF3800C3F3C1037448D840BCE7724B1968C905FC
:10BF480003D5B2F1805F00F0F280186810F4003079
:10BF5800B0D0B2F1005F6D4818BF0020AAE7A0F585
:10BF680080530B431FD1674B1A6D02F4E042B2F5C0
:10BF7800005F95D0ACD9B2F5405F00F0DA80B2F539
:10BF8800804FB8D1DA6C196802F040521B68480734
:10BF980001D5002ACCD0D90503D5B2F1805F00F0D5
:10BFA800C680584BD1E7A0F500530B4321D1554A21
:10BFB800136D03F4E023B3F5403F00F089800DD8FA
:10BFC800B3F5803F00F0A880B3F5003F74D0002B94
:10BFD80091D105B05DF804EBFFF72EBDB3F5802FC6
:10BFE80063D0B3F5A02F86D11068484B10F4003009
:10BFF8005FE0A0F500230B4321D1424B9A6D02F478
:10C008004032B2F5803F10D0B2F5003FBAD0002AD6
:10C018007FF471AF186810F000603FF44BAF002355
:10C0280001A80193FFF72CFD43E7186810F00050B2
:10C038003FF440AF01A8FFF7CDFD03983AE7A0F51C
:10C0480080330B430DD12F4BDA6C1868D3037FF57F
:10C0580043AF10F000603FF42DAF01A8FFF710FDCB
:10C06800EBE7A0F580430B4339D1264A936D03F0E3
:10C07800E043B3F1405F2BD00DD8B3F1805F4BD0D4
:10C08800B3F1005F18D0002B7FF435AF05B05DF831
:10C0980004EBFFF7E3BCB3F1A04FA5D0B3F1C04F59
:10C0A80047D0B3F1804F7FF426AF1068184B10F4D7
:10C0B800807018BF1846FDE6106810F000503FF475
:10C0C800F9AE002301A80293FFF784FD0298F1E678
:10C0D800106810F004003FF4EDAE136828E7A0F5EF
:10C0E800004008437FF407AF064A136D03F040533E
:10C0F800B3F1805F0ED0B3F1005F0DD0002B7FF459
:10C10800FAAE71E7004402580090D00300366E0181
:10C1180000093D001068DFE6106810F000603FF489
:10C12800C9AE002301A80293FFF7AAFCCEE7024894
:10C13800C0E60248BEE600BF00093D000080BB0023
:10C1480070B505684B68EC68C4F30B441C44D30114
:10C1580084331D446A6802F470426A6005680E6898
:10C16800EA681D440136C2F30B42324442EA0442F3
:10C178006A600268CD68D4681A44C4F30A042C447F
:10C18800956805F47045956005688A68EE681D44F1
:10C198000132C6F30A06324442EA0442AA6002683F
:10C1A8001A44146924F00704146102680C691A44DB
:10C1B800146102688D69D41891F8302042EA05624A
:10C1C80091F8315042EA052291F8325042EA05428C
:10C1D800A26102681A44546924F0FF045461026899
:10C1E8004C691A44546104681C44E26922F4E06210
:10C1F80022F00702E2610268D1E907451A442C439C
:10C20800D46102684C6A1A4494620A69072A96BF84
:10C21800124C0124A45C02681A44D56A05F0E02592
:10C22800D5620268D518D1E90062921B8E6A624312
:10C238007443073242EA0442EA6202681A44146B01
:10C248006FF30A0414630268C96A1A441163016827
:10C25800CA5842F00102CA5070BD00BF50CD07084D
:10C2680010B590F8A02003460220012A14D083F8C4
:10C27800A1000124186883F8A040426B22F0010253
:10C2880042630020054A116419684A6B22434A63D5
:10C2980083F8A14083F8A00010BD00BF0010005033
:10C2A8002DE9F0410268136823F040531360836856
:10C2B80033B902684C68136823F080032343136082
:10C2C8000A680368022A49D103F5C07203F5C475E8
:10C2D80003F5C87403F5D073D1E912673E431660BD
:10C2E800CE6A5EB18E6A1E604F6BCB6A16683B439E
:10C2F8000F6B26F47C163B43334313602B684E6C5C
:10C3080023F01F0333432B608B6B2BB10B681BB9D6
:10C31800CB6B0568013B2B64CD68CE69002D6AD0D4
:10C328008F6BD1E90483002E42D0354343EA0803DA
:10C338001668D1E908CE2FB33B430F6C43EA0E03CE
:10C3480043EA0C033B432B433A4D35402B431360E0
:10C358008B68236003688A699A6439E0032A03BFFB
:10C3680003F5A07203F5A47503F5A87403F58072AC
:10C378001BBF03F5847503F5887403F5B07303F5E3
:10C388009073A9E743EA0E0343EA0C032B4326F410
:10C398007C5525F03F052B431360C36AB3F1805FDA
:10C3A800D6D14B69082BD3D1136843F00063CEE78D
:10C3B8001D43136845EA08056FB1086C3D4323F037
:10C3C8007063054323F03F031D4315608B682360AA
:10C3D8000020BDE8F08123F03F031D431560C36AC8
:10C3E800B3F1805FF2D14B69082BEFD1136843F0AA
:10C3F80000631360EAE7C6B18B6BD1E9087463B1D7
:10C408003343156823430C6C3B43234325F0706486
:10C4180024F47C54234313609CE71368344323F4C7
:10C428007C533C431C43146094E708234365012074
:10C43800CFE700BFC0C0FFF073B504463CF012FF61
:10C44800054614B9012002B070BD00236365266D4E
:10C45800002E69D1204640F0DDFB41F28833E168C7
:10C46800A365636B22681943E369906819432F4BEE
:10C478000340204619432369013B41EA03416369AC
:10C48800013B41EA032191602268216AD36823F4C1
:10C49800E0230B43D360216BA36B226843EA01437B
:10C4A80013612368E26B5A61226863681168013B73
:10C4B80021F4F85141EA032111603246A36D20218D
:10C4C80000932B4640F07EFB0028BBD12168636AAD
:10C4D800CA68013B22F0FF021343CB602268A168BF
:10C4E800136823F040030B4313602168D4E90A3032
:10C4F800D1F80821034322F0A0421343C1F80831C0
:10C508002268136843F001031360A369022B04D166
:10C518002268936843F002039360E368B3F1806F85
:10C528000CBF01230223236500208CE7F4F8E0F810
:10C5380038B5036804461A6A18685507216D1FD56F
:10C5480045031DD5182914D1226C127883F8502080
:10C55800236C01332364A36C013BA364A36C23B94C
:10C568002268136823F480231360204640F009FDF5
:10C5780038BD2829F2D1226C93F850301370E7E7C0
:10C58800950740D585033ED528291ED1A16C69B1F0
:10C5980012F47C5F0AD093F85030226C1370236C2D
:10C5A80001332364A36C013BA364E1E7A26C002A76
:10C5B800DED1022220465A6221680B6823F4E02368
:10C5C8000B6022653FF02AFCD2E7022218295A6242
:10C5D8002068036823F4E0230360226503D1204622
:10C5E8003FF01FFCC4E7082903D120463FF013FCA5
:10C5F800BEE7B1F5807FBBD1636D2046002B35D1F6
:10C6080040F09AFCB4E7110711D505030FD50822AD
:10C618005A6223681A68500205D51A6822F4102253
:10C628001A600223236520463FF0FEFBA0E7D107EE
:10C638001FD5C5031DD5012202255A622268136839
:10C6480023F4F8131360236865651A6850070BD53F
:10C658001A6822F004021A600C4AE36C9A65E06CCE
:10C6680040F09DFA002883D0204625653FF0CDFB99
:10C678007EE7D1067FF57CAFC2027FF579AF102245
:10C6880020465A623FF0D3FB72E700BF43CF04084D
:10C698002DE9F041B24B8CB002684FF0010E002733
:10C6A800DFF8C0829A426B4607BF012500220025A9
:10C6B8000122BEF1020F1F61C3E90077C3E90277C7
:10C6C80040F04A81A748A84E006810F0010F18BF33
:10C6D8004FF400764FF0000C08EB8C000CF10104CD
:10C6E800406810F0010F05D080EA060C1CF0020F1C
:10C6F80008BF1C6010F0100F05D080EA060C1CF073
:10C70800200F08BF5C6010F4807F05D080EA060C1B
:10C718001CF4007F08BF9C6010F4803F0DD080EAB5
:10C72800060C1CF4802F08D110F4003F0CBF44F411
:10C73800803C44F0807CC3F80CC010F0807F0BD0A4
:10C7480080EA060C1CF0806F06D1800154BF44F4C7
:10C75800803044F080701861022C4FF0010CBBD17E
:10C76800BEF1020F03F1180340F0F4807C4B186807
:10C7780010EA0C0004D0186820F001001860604628
:10C788007A4B1C68E70740F1E9801C6824F0010433
:10C798001C6040F002040CAB182707FB0237714BF2
:10C7A80057F8286C013E03EB8606D6F804C02CF433
:10C7B800807CC6F804C01E68F60740F1D9801E6860
:10C7C80026F001061E6065B3069E013E03EB860651
:10C7D800776847F002077760079E36B1013E03EBA2
:10C7E80086035E6846F020065E60099B5BB1013BEC
:10C7F80003F001039B0003F1A44303F534435E688F
:10C8080046F480265E600A9B5BB1013B03F001039E
:10C818009B0003F1A44303F534435E6846F0806649
:10C828005E600CAE182303FB05630E6853F830CC2A
:10C83800664500F0DD808F6853F8286CB74200F039
:10C84800EC804E6853F82C3C9E4202D1002E40F0FA
:10C85800E48018230CAFCE6803FB057757F8247CD7
:10C86800BE4202D1002E40F0D8800CAF0E6903FB07
:10C87800057353F8203C9E4202D1002E40F0CD8033
:10C888008E68384B013E03EB8606756825F44075C3
:10C8980045EA422545F4807575604E691D68013E7C
:10C8A800C5F30745AE4205D91D6825F47F0545EA5D
:10C8B80006451D600D681E68013D16F0010F4FEA20
:10C8C80085051D4400F014816A6822F0030242F0D5
:10C8D80001026A604A6842B1013A03EB82035A686E
:10C8E80022F0300242F010025A60CB68DF0340F1B8
:10C8F800DD80013B03F001039B0003F1A44303F532
:10C9080034435A6822F4E02242F480325A600B69B8
:10C91800DE0340F1DC80013B03F001039B0003F1DF
:10C92800A44303F534435A6822F4E02242F4403227
:10C938005A6020B10A4A136843F001031360A30741
:10C9480004D50A4A136843F00103136000200CB0B1
:10C95800BDE8F081A646ACE60026BBE604461AE729
:10C968000050005200B400522202040400A00052F9
:10C9780057F8306C002E3FF454AF013E03EB8606A7
:10C98800D6F804C02CF0010CC6F804C057F82C6C7B
:10C9980036B1013E03EB86035E6826F010065E6042
:10C9A80018230CAE03FB026353F8243C5BB1013B34
:10C9B80003F001039B0003F1A44303F534435E68CD
:10C9C80026F480365E6018230CAE03FB026353F82E
:10C9D800203C002B3FF425AF013B03F001039B00F3
:10C9E80003F1A44303F534435E6826F0807617E725
:10C9F8004F6853F82C6CB7420FD1CF6853F8246CAA
:10CA0800B7420AD10E6953F8203C9E4205D1664DC3
:10CA18002B6843F001032B6032E70CF1FF33624EC1
:10CA280006EB83035F6827F001075F6018230CAFEC
:10CA380003FB057353F82C3C33B1013B06EB83032E
:10CA48005E6826F010065E600CAE182303FB0563D3
:10CA580053F8286CB700554E3E44776827F4807722
:10CA6800776053F8243C5BB1013B03F001039B0062
:10CA780003F1A44303F534435E6826F480365E6010
:10CA880018230CAE03FB056555F8203C002B3FF43A
:10CA9800F7AE013B03F001039B0003F1A44303F548
:10CAA80034435D6825F080755D60E9E6002B3FF44E
:10CAB8002EAF013B03F001039B0003F1A44303F5F0
:10CAC80034435A6822F0E06242F080721EE7002B7D
:10CAD8003FF42FAF013B03F001039B0003F1A44394
:10CAE80003F534435A6822F0E06242F040721FE7CF
:10CAF8006E6826F0030646EA420646F001066E60B6
:10CB08004D6855B1013D03EB85035D6825F030059F
:10CB180045EA421545F010055D60CB68DD0320D578
:10CB2800013B03F001039B0003F1A44303F53443E5
:10CB38005D6825F4E02545EA824545F480355D6069
:10CB48000B69D9031FD5013B03F001039B0003F1D7
:10CB5800A44303F53443596821F4E02141EA8242B1
:10CB6800E4E6002BECD0013B03F001039B0003F14A
:10CB7800A44303F534435D6825F0E06545EA826522
:10CB880045F08075DBE7002B3FF4D3AE013B03F0A3
:10CB980001039B0003F1A44303F53443596821F0D2
:10CBA800E06141EA8262A0E700B40052FCB300529F
:10CBB8002DE9F04F066889B00446304641F06CFA1A
:10CBC8000390002840F06E81206841F037FA002871
:10CBD80000F06881D6F8083806F500652068C3F3C8
:10CBE8000D23C4F8D43441F029FA870704D5226804
:10CBF800536903F002035361206841F01FFAC0062D
:10CC08002DD52268936923F010039361D6F820800C
:10CC180008F4F01308F00F07B3F5802F40F04581B2
:10CC280047F6F07318EA030F14D02423C8F30A193F
:10CC3800304603FB07474A46D7F8601241F08FF9A0
:10CC4800D7F860324B44C7F86032D7F868324B44A3
:10CC5800C7F868322268936943F01003936120682B
:10CC680041F0ECF9010300F13381206841F0E6F965
:10CC780042030CD5274606F5106B4FF0000A2068D2
:10CC880041F0E8F90490049B002B40F0EB81206808
:10CC980041F0D4F9002813DA6B6823F001036B60C4
:10CCA80094F8CC34012B40F085820021204684F88A
:10CCB800CC1440F0EDFB2268536903F00043536144
:10CCC800206841F0BBF903050AD5AB68DF0702D538
:10CCD80020463EF0B2FC2268536903F400635361B6
:10CCE800206841F0ABF9000115D52268536903F0BB
:10CCF8000063536194F8CC34002B40F05F8201212B
:10CD08002368204684F8CC145B6DC3F38303C4F80E
:10CD1800D03440F0BDFB206841F090F9C10433D510
:10CD28006B68102123F001036B60206840F09BFFC3
:10CD380006F510634FF67F3122790398824200F29C
:10CD48004182EB6943F00113EB61E37B002B00F0B8
:10CD58005782D5F8843043F00B03C5F884306B6CE8
:10CD680043F00B036B64D6F8003804F29C4223F4BA
:10CD7800FE63C6F80038A179206801F051FD2268E9
:10CD8800536903F480535361206841F057F98204D2
:10CD980016D5206841F084F9206840F0AFFF276875
:10CDA800E071FEF727FEE2790146384601F0CAFA3B
:10CDB80020463EF00AFC2268536903F4005353618D
:10CDC800206841F03BF9030707D520463EF053FCA5
:10CDD8002268536903F008035361206841F02EF973
:10CDE800070600F11882206841F028F9C0020CD526
:10CDF800A04606F5126901272379BB4200F2298271
:10CE08002268536903F480135361206841F016F9CE
:10CE180081022AD5234606F532614FF0010C2079AC
:10CE280060451DD993F87C720868012F40F027826D
:10CE3800002880F22482D4F8D42482EA1040C20761
:10CE480000F11D8283F87B72B06940F08000B06108
:10CE58007069000600F113826B6843F400736B601D
:10CE68002268536903F400135361206841F0E6F81F
:10CE7800410007D520463EF0D4FB2268536903F0F1
:10CE880080435361206841F0D9F842070AD52368E6
:10CE98005D686B0702D520463EF0C9FB22685368DF
:10CEA8002B43536009B0BDE8F08FB3F5402F7FF4F2
:10CEB800D1AE082204F29C413046C8F30A1841F06A
:10CEC8004EF8242303FB0747D7F868324344BFE6EC
:10CED80006F53068A2460027206841F0B3F80490B0
:10CEE800049B002B3FF4C1AE049BDB0779D55FFAA6
:10CEF80087FB2068594641F0B5F810F0010F8146CC
:10CF08001FD00123C8F80830206894F806C000F53F
:10CF18003063016CBCF1010F03EB47139A6840F0D2
:10CF28008B8012F0080F07D0B348814209D9120448
:10CF380007D54FF4004203E012F0200F5AD0202208
:10CF48009A6019F0080F21D00823AB49C8F80830B7
:10CF580023681A6C03F530638A4203EB4713986819
:10CF680004D9000402D54FF4004098602046059289
:10CF7800FAF726FC059AA0498A4207D9A17901291E
:10CF880004D104F29C42206801F04AFC19F0100F09
:10CF980002D01023C8F8083019F0020F14D07369B2
:10CFA800190603D56B6843F480636B609AF85732AF
:10CFB800012B06D10023594620468AF8573240F003
:10CFC800EAF80223C8F8083019F0200F02D020230D
:10CFD800C8F8083019F4005F03D04FF40053C8F8BC
:10CFE8000830049B013708F120080AF1240A5B087D
:10CFF800049375E7DFF800C2614501D9120498D49B
:10D008001A69DAF87432C2F312029B1ACAF8683243
:10D018006FB9D4F864222AB904F29C42012101F0C4
:10D02800FFFB04E0D4F860221A44C4F86022594691
:10D038002046FAF78BFB84E7DFF8C0C1614507D1CA
:10D0480011043FF576AF9206F1D520229A60EEE7FB
:10D05800002FECD1D4F86432002BE8D104F29C42C2
:10D068003946DCE7049BDA0740F19B805FFA8AF3D4
:10D0780020681946079340F0FEFF10F0010F804624
:10D0880020D001210AF00F026B6B01FA02F223EAA9
:10D0980002036B63CBF80810A17901290DD1D7E9F8
:10D0A800072313443B62BAF1000F06D1636A23B920
:10D0B80004F29C42206801F0B3FB5FFA8AF1204633
:10D0C800FAF762FB18F0080F02D00823CBF80830F3
:10D0D80018F0100F02D01023CBF8083018F0400FCA
:10D0E80002D04023CBF8083018F0020F10D0514678
:10D0F800304640F0B8FDFB7D012B06D100235FFAD6
:10D108008AF12046FB7540F047F80223CBF8083037
:10D1180018F0800F45D0D7E909329A4241D8A3EBDD
:10D128000208FB6921689845059128BF984601F5D2
:10D13800106308F1030803EB4A134FEA98080693B3
:10D14800069B996989B24145D7E9093227D39342A9
:10D158000BD8059B0AF00F000121D3F83428814031
:10D1680022EA0102C3F834281BE0A3EB0209FB6999
:10D17800079A9945059828BF9946A37900931FFAFD
:10D1880089F3396A09F1030840F0D6FE3B6A4FEA91
:10D1980098084B443B62BB6A4B44BB62D0E793425E
:10D1A800D7D9049B0AF1010A24370BF1200B5B083D
:10D1B800049368E520463EF04FFA7CE520463EF0B1
:10D1C8003CFAA8E59960203353F8202C22F4001289
:10D1D80043F8202CC3F8E811D3F8E02122F4001218
:10D1E800C3F8E021D3F8E02142F00062C3F8E0215F
:10D1F800039A013203929FE50A30544F0A31544F83
:10D208006B6943F4005343F02B036B612B6943F0C4
:10D218000B032B61A7E5B369012204F257202427E9
:10D2280023F08003B36106F53263217991427FF6DA
:10D23800DAAD07FB02F1415C012907D1196841F019
:10D2480000611960196841F080411960013220338A
:10D25800EBE798F83C30D9F80020012B09D1002AD7
:10D2680007DA67F07F01204688F83B30C9B240F002
:10D27800ACF8013708F1240809F12009BCE50CF1E4
:10D28800010C24332031CAE52DE9F047054686B064
:10D2980088463BF0E7FF08218146286840F04BFAB2
:10D2A800044648BB696C2868090440F02EFB044614
:10D2B80010BB4FF0FF300823302669460494CDE9AF
:10D2C800000302232868CDE902630123059340F097
:10D2D8001FFA286840F04DFB044668B90746064621
:10D2E80040F22A5A2868436B13EA0A0F436B07D0A7
:10D2F8001A0719D508248463204606B0BDE8F087CC
:10D30800190308D43CB940F0E8F906462868012416
:10D3180040F0E3F907463BF0A5FFA0EB0900013018
:10D32800E0D14FF00044E7E7436B9B0701D50224A7
:10D33800E1E7446B14F0200401D02024DBE7044B20
:10D348003FBA36BA8363C8F80070C8F80460D3E7F8
:10D358003A0F001870B5044686B015461E4631B916
:10D36800436B43F000636363012006B070BD90F81F
:10D378003030012B4BD10022AB194263006D834240
:10D3880003D9636B43F00073EDE7032384F830306F
:10D398002368DA627302A26BA362012A4FF0FF329C
:10D3A80061626946206818BF6D02CDE900239022AA
:10D3B8000223CDE902230023CDE9043340F0A8F984
:10D3C8002268012ED36843F04003D360206811D946
:10D3D8000A232946E36240F0E2F9226880B10D4B46
:10D3E8009363636B03436363012384F83030002342
:10D3F800E362B9E709232946E36240F0B6F9ECE7AE
:10D40800D36B43F4014343F02A03D363ADE702200F
:10D41800ABE700BFFF0FE01F70B5044686B01546A6
:10D428001E4631B9436B43F000636363012006B0C5
:10D4380070BD90F83030012B4AD10022AB194263FD
:10D44800006D834203D9636B43F00073EDE7032358
:10D4580084F830302368DA627302A26B2362012AEF
:10D468004FF0FF32E1616946206818BF6D02CDE9CF
:10D47800002300239022CDE90433CDE9022340F0B4
:10D4880047F92268012ED36843F04003D36020682F
:10D4980011D928232946E36240F0B5F9226880B102
:10D4A8000C4B9363636B03436363012384F830304D
:10D4B8000023E362BAE718232946E36240F089F9BA
:10D4C800ECE7D36B43F4824343F01A03D363AEE72C
:10D4D8000220ACE7FF0FE01FF8B590F830300446A3
:10D4E8000E461546012BDFB257D100219642416303
:10D4F80005D9436B43F0006363633846F8BD036D99
:10D50800934203D2436B43F00073F5E7032380F89B
:10D518003030236C00689B0608D4214B8363636B0F
:10D5280043F08063636384F83070E6E740F0EDF819
:10D538008201236805D51A4A9A63636B43F4006332
:10D54800F0E7A26B012A03D0032A1BD076026D02F2
:10D558001846314640F071F90346206843B1104A35
:10D568008263626B13436363012384F83030C4E73A
:10D57800294640F07CF928B12368094A9A63636B0D
:10D588000343F0E70021206840F08BF90028F3D12D
:10D598000123074684F83030AFE70227ADE700BF24
:10D5A800FF0FE01F10B5C26D0346920F0A70C26DDF
:10D5B800C2F383624A7090F85F2002F003028A7017
:10D5C80090F85E20CA7090F85D200A7190F85C208F
:10D5D8004A71026E120DCA80B0F8622002F00F0282
:10D5E8000A72026EC2F3C0324A72026EC2F380320D
:10D5F8008A72026EC2F34032CA72026EC2F30032FD
:10D608000A7300224A73826B002A40F08380006EFE
:10D6180040F6FC7202EA8002586E42EA90720A6191
:10D628005A6EC2F3C2620A7593F8672002F00702C5
:10D638004A755A6EC2F342528A755A6EC2F38242D2
:10D64800CA755A6EC2F3C2320A7608690130986404
:10D658000A7E02F0070202329040012298640C7A96
:10D6680004F00F04A240DA64520A42431A654FF4E8
:10D67800007200205A655A6EC2F380324A765A6E9A
:10D68800C2F3C6128A765A6E02F07F02CA769A6E82
:10D69800D20F0A779A6EC2F341724A779A6EC2F332
:10D6A80082628A779A6EC2F38352CA779A6EC2F3FD
:10D6B800405281F8202081F82100B3F86A2002F056
:10D6C800010281F822209A6EC2F3C03281F8232029
:10D6D8009A6EC2F3803281F824209A6EC2F34032E7
:10D6E80081F825209A6EC2F3003281F826209A6EBE
:10D6F800C2F3812281F827209A6EC2F3012281F8B1
:10D7080028209B6EC3F3460381F82930012381F852
:10D718002A301CE0012A10D1026EB0F8660012040B
:10D7280002F47C1202430A610A69013292029A6485
:10D738001A654FF40072DA6499E702680449916344
:10D74800426B42F080524263012083F8300010BDE2
:10D75800FF0FE01FF0B595B014220021044604AF76
:10D7680038465AF004FC4FF480300021FEF786FB5F
:10D77800054648B9012384F830304FF000636363ED
:10D788000125284615B0F0BD7C4B984289BF7C4ED8
:10D798000026B0FBF6F601360798314608968DE864
:10D7A800030097E80E00206800F002FC20683FF0B4
:10D7B8009CFF36B1B5EB460F4FEA460307D3B5FBDE
:10D7C800F3F57048B0FBF5F001303BF053FD002352
:10D7D8002068039300F01AFC054648B9206840F019
:10D7E80075F904280AD12068E56300F00FFC78B1C8
:10D7F800012384F83030636B0343C0E70123E363FC
:10D808000021206840F081F828B14FF08050EFE700
:10D81800E36B012BF4D000264FF6FE7714E0314677
:10D82800206840F072F80028E2D15749206840F09B
:10D838001CF90028E9D1314620683FF066FF039BB8
:10D848000546C60F01330393039BBB4201D8002E44
:10D85800E5D0039BBB4214D8C5F380750023A563AC
:10D86800ADF80A303BF0FEFC054620683FF049FF62
:10D8780050B94FF08061012384F83030636B0B435B
:10D888007DE74FF08070B3E7A36B032B3ED0206891
:10D8980040F0BDF801460028EDD120683FF035FF83
:10D8A8000421E06620683FF030FF082120672068E7
:10D8B8003FF02BFF0C21606720683FF026FFA36B29
:10D8C800A067032B22D041F28736BDF80A102068E2
:10D8D80059B3A36B032B19D06164090440F0AEF867
:10D8E80001460028C7D120683FF00FFF0421E065FA
:10D8F80020683FF00AFF0821206620683FF005FFF6
:10D908000C21606620683FF000FFA06604212068B3
:10D918003FF0FBFE09A9000D20642046FFF742FEF8
:10D92800054688B14FF08051A5E70DF10A0140F096
:10D93800B3F8014600289ED13BF094FC401BB0424E
:10D94800C3D94FF0004196E7616C206809043FF0A5
:10D95800C2FF014600288ED14FF4007120683FF0C5
:10D96800EAFE00283FF40DAF2368084A9A63636B08
:10D9780003436363012384F8303001E7801A06000B
:10D9880000350C0010210100000010C1FF0FE01F3E
:10D998002DE9F04190F8303096B004460D46032B3F
:10D9A80000F0AB803BF05EFC0021064620683FF0AB
:10D9B800ACFE830100F1A680402120683FF0BBFE49
:10D9C80058B1636B636323680125524A9A63636B9A
:10D9D8000343636384F8305082E0616C2068090473
:10D9E8003FF093FF0028ECD140234FF0FF374FF072
:10D9F800600C049069462068CDE900730223CDE9E4
:10DA080002C3012305933FF083FE20683FF0E5FF42
:10DA18000028D6D106AF23685A6B12F4957F0AD036
:10DA28005A6B110771D45A6B920770D45B6B9B06C3
:10DA38001ED52020C7E75B6B180408D507F120081E
:10DA480020683FF04AFE47F8040B4745F8D13BF001
:10DA580009FC801B0130DED14FF00040B3E73FF0F6
:10DA68003CFE47F8040B3BF0FDFB801B0130F3D074
:10DA78002068426B12F48052F1D10699264B8363D9
:10DA8800C1F381132B70C1F340136B700B0A23F0A1
:10DA9800FF0343EA11639BB26B80079B1BBA6B6061
:10DAA800089BD9B22972C3F307216972C3F30351E2
:10DAB8001B0CA972099923F0FF03C8B20343AB8179
:10DAC800C1F38523AB73C1F30123EB73C1F30313D4
:10DAD80001F00F012B749DF82B306974AB74154657
:10DAE8004FF4007120683FF026FE38B12368094AD8
:10DAF8009A630123606384F830300125284616B004
:10DB0800BDE8F0814FF400605DE708205BE7022084
:10DB180059E700BFFF0FE01F3A0F0018032330B585
:10DB280089B080F83030836B04460D46032B02D051
:10DB3800B1F5004F03D1636B43F080531FE0B1F59B
:10DB4800804F24D10021006803913FF0DEFD10F0E2
:10DB5800007036D1049003A92046FFF795FB60B901
:10DB6800049B590330D5616C206809043FF0CDFE51
:10DB780018B9022120683FF0E2FE636B0343636338
:10DB8800636B43B323683E4A9A63012550E0F1B9B9
:10DB9800006803913FF0B9FD820112D403A9204621
:10DBA8000495FFF771FB0028E7D1049BDB030BD535
:10DBB800616C206809043FF0A8FE0028DDD1014609
:10DBC800D8E74FF40060D8E74FF08060D5E7436BA3
:10DBD80043F00063D3E74FF480300021FEF74EF99D
:10DBE800002847D0636827490393A368B0FBF1F284
:10DBF800CDE9043523690693636993420CD2A56D78
:10DC0800B5F5007F08D0B5F5807F29D11BBB8842C8
:10DC180002D91D4BB0FBF3F3079308AB002513E9BA
:10DC2800030003AB8DE803000ECB206800F0C0F9B9
:10DC38004FF4007120683FF07EFD30B12368012564
:10DC48000F4A9A63636B034363630123284684F88E
:10DC5800303009B030BD5A00B0FBF2F28A42D7E743
:10DC68000A491BB9884288BF1346D5E75D00B0FB57
:10DC7800F5F0F7E7636B43F00063636385E700BF84
:10DC8800FF0FE01F80F0FA0200E1F50540787D0102
:10DC9800F7B503680446C56A5A6B170420D52E07E2
:10DCA8001ED5836A1F2B19D9466A351D06F124072C
:10DCB800206804353FF011FD05F8080C030A05F843
:10DCC800073C030C000E05F8063C05F8050CBD42A0
:10DCD800EED1A36A2036203B6662A36203B0F0BD92
:10DCE8005A6BD0055BD54FF480729A632268D36B68
:10DCF80023F4414323F03A03D3632268D36B23F020
:10DD08008053D3632268D36823F04003D36015F0AF
:10DD1800080320D015F0220F09D0206800F030FA4F
:10DD280028B1636B0343204663633DF0D8FD236845
:10DD3800A907704A9A634FF0010384F830304FF016
:10DD48000003E36203D020463DF0C7FDC6E7204646
:10DD58003DF0BEFDC2E72A06C0D5226815F0220FA5
:10DD680093622268D3622268136509D0206800F0A4
:10DD780007FA28B1636B0343204663633DF0AFFDA8
:10DD8800012315F0300F84F830304FF00003E362C0
:10DD980002D020463DF09CFDAF079FD0D3E75A6BD9
:10DDA800560427D5280725D5236A1F2B96D9E66957
:10DDB800351D06F1240715F8043C043501A920682F
:10DDC800019315F8072C43EA0223019315F8062C52
:10DDD80043EA0243019315F8052C43EA02630193D1
:10DDE8003FF07EFCBD42E6D1236A2036203BE66147
:10DDF800236273E75A6B12F03A0F5A6B5ED09107A1
:10DE080003D5626B42F0020262635A6B120703D5B4
:10DE1800626B42F0080262635A6B970603D5626B25
:10DE280042F0200262635A6BD60603D5626B42F059
:10DE3800100262632F4A9A632268D36B23F49D739E
:10DE4800D3632268D36823F04003D3602268D36A7F
:10DE580043F40053D3622268D36843F08003D3604D
:10DE6800206800F08DF9636B226815F0080143EA19
:10DE780000036363D36823F08003D3604FF4006228
:10DE880023689A6308D0012384F830300023E362C2
:10DE980020463DF024FD21E728067FF51FAF636B80
:10DEA800002B3FF41BAF2268D36B23F08053D3635E
:10DEB80023681965012384F83030E9E7D2007FF53B
:10DEC8000DAF4FF0805205F0200520469A63236875
:10DED8001B6D5B0706D415B13FF06AFBFEE63FF009
:10DEE80065FBFBE615B13FF062FBF7E63FF05DFB33
:10DEF800F4E600BF3A0F001838B50D460446F0B1F5
:10DF080090F82C3003F0FF021BB980F82D203FF069
:10DF180050FB0223211D206884F82C3000F014F8EF
:10DF28006268294620683FF07CFB064A0020136897
:10DF380043F000431360012384F82C3038BD0120DE
:10DF4800FCE700BF00400052D1E9073230B50C6849
:10DF580013434D6A154A94B904682B43224013436E
:10DF68004A6813438A681343CA6813430A69134308
:10DF78004A6913438A6913430360002030BD04686B
:10DF88002B4324F4F84423430360436813404A684E
:10DF980013438A681343CA6813430A6913434A69D7
:10DFA80013438A6913434360E7E700BF0080FFFF1C
:10DFB80084B010B503AC84E80E00039B416813439A
:10DFC800059A1343069A1343079A1343044A0A40CF
:10DFD800134343600020BDE8104004B0704700BF01
:10DFE800002CC0FF0B6810B58360C468D1E901320A
:10DFF8001343CA6813430A691343034A224013436D
:10E00800C360002010BD00BFC0E0FEFF10B50023B4
:10E0180086B0044601A9CDE90133CDE903334FF4B5
:10E0280080530593FFF7DEFF0A4B4FF4FA521B6843
:10E03800B3FBF2F341F28832534343B1626B013BC5
:10E048001206FAD5044B0020A36306B010BD4FF0AA
:10E058000040FAE780090024C50020000346444830
:10E0680010B54FF4FA540068B0FBF4F0414C424349
:10E07800002A48D0586B204207D0800405D45A6B38
:10E08800540704D50420986310BD013AF0E75A6B91
:10E09800D00703D501229A630120F5E7364A9A632F
:10E0A8001A69D2B29142F7D15B6934481840002806
:10E0B800EAD0002B2ADB5A002BD49C002BD4D900A1
:10E0C8002BD41A012CD45C012DD4D9012ED41A02D8
:10E0D8002FD45C0230D4990231D4DA0232D45C03F2
:10E0E80033D4990334D4DA0335D41C0436D4590410
:10E0F80037D49A0438D413F0080F0CBF4FF480308B
:10E108004FF40000C0E74FF00040BDE74FF000704B
:10E11800BAE74020B8E78020B6E74FF48070B3E74D
:10E128004FF40070B0E74FF48060ADE74FF4006043
:10E13800AAE74FF48050A7E74FF40050A4E74FF444
:10E148008040A1E74FF400409EE74FF400309BE782
:10E158004FF4802098E74FF4002095E74FF48010A3
:10E1680092E74FF400108FE74FF480008CE700BF70
:10E178008009002445002000C500200008E0FFFDBC
:10E1880030B5002387B00C254FF48072044601A9EE
:10E19800CDE90323CDE901354FF480530593C368D6
:10E1A80043F08003C360C36823F04003C360FFF7F4
:10E1B80019FF074A29462046FFF750FFE368B0F1E8
:10E1C800007F23F0800308BF0020E36007B030BD64
:10E1D80000E1F505114B4FF4FA5102461B68B3FBF9
:10E1E800F1F341F288314B43ABB1516B11F0450F5C
:10E1F80007D0890405D4536B5B0704D504209063CA
:10E208007047013BF0E7506B10F0010014BF012389
:10E21800034B936370474FF0004070478009002418
:10E22800C50020000F4B4FF4FA5102461B68B3FBA0
:10E23800F1F341F288314B438BB1516B11F0450F2B
:10E2480008D0890406D4506B10F0040004D00420D0
:10E2580090637047013BEFE7034B936370474FF0C0
:10E268000040704780090024C500200003461E486E
:10E2780010B54FF4FA540068B0FBF4F041F288345A
:10E28800604358B35C6B14F0450F07D0A40405D461
:10E29800586B440704D50420986310BD0138F0E793
:10E2A800586BC00703D501229A630120F5E7186966
:10E2B800C0B28142F9D10D4999635B6913F460409A
:10E2C80002D11B0C1380E8E75A040AD413F4004F58
:10E2D8000CBF4FF480304FF48050DEE74FF0004021
:10E2E800DBE74FF40050D8E780090024C500200080
:10E2F800134B4FF4FA5102461B68B3FBF1F341F29A
:10E3080088314B43CBB1516B11F0450F07D08804CE
:10E3180005D4536B590704D5042090637047013B1B
:10E32800F0E7506B10F0010002D0012393637047AF
:10E33800536B5B0603D54023F8E74FF00040704766
:10E3480080090024022A4AD1274B284A0B449342C9
:10E3580039D9274B274A0B44934236D9A1F5740380
:10E36800254AA3F51053934231D9A1F18373234A67
:10E37800A3F5E74393422CD3214B224A0B44934203
:10E3880029D9214B214A0B44934226D3204B214AB9
:10E398000B44934223D3A1F1B7731F4AA3F55853F3
:10E3A80093421ED31D4B1E4A0B4493422CBF062397
:10E3B8000723C26822F47052C260C26842EA83230B
:10E3C800C360002070470F23F3E70E23F1E70D2306
:10E3D800EFE70C23EDE70B23EBE70A23E9E7092333
:10E3E800E7E70823E5E700BF405327FFFF340C00A9
:10E3F800401E1BFF3F420F007F4F120020D6130024
:10E4080060B6E5FE5FE3160000D3CEFE40771B0042
:10E41800C05BB3FEC091210020753800E05459FE5E
:10E42800E09C410084B02DE9F843044609A880E83F
:10E438000E0000239DF824609DF82E50194603F124
:10E448004002013304EB82020F2B5160F7D104F52F
:10E458000067002D6CD17B6843F002037B60A36BDF
:10E4680023F40013A363236843F040032360236865
:10E4780043F0800323600023C4F8003E9DF8293050
:10E48800012B5CD19DF82710002956D120464FF664
:10E498007F383FF02CFC102120463FF0E4FB01467A
:10E4A80020463FF003FC0843002304F51062C0B285
:10E4B8004FF0904C19464FF0006E00383B617B617D
:10E4C80018BF0120FB619E423BD8002204F530634F
:10E4D8004FF0904C4FF0006E11464FF67F38964241
:10E4E80042D83B6923F480733B610023A3616FF03A
:10E4F800804363619DF826301BB9A36943F010037C
:10E50800A361A269224B1343A3619DF82A301BB172
:10E51800A36943F00803A361012D05D1A36943F062
:10E52800804343F00403A361BDE8F84304B0704797
:10E53800A36B43F40013A3639DE71946A6E70321E1
:10E54800A4E7D2F80090B9F1000F0BDA3BB9C2F892
:10E5580000E011610133C2F808802032B3E7C2F845
:10E5680000C0F6E71160F4E7D3F80090B9F1000FA6
:10E578000BDA3AB9C3F800E019610132C3F8088030
:10E588002033ACE7C3F800C0F6E71960F4E700BF32
:10E5980000383C8030B54A780B78012A00EB4313E9
:10E5A80000F5006029D1D3F80029002A0BDAD3F846
:10E5B800002942F00062C3F80029D3F8002942F08C
:10E5C8008042C3F800290A780124C56B02F00F02C3
:10E5D80004FA02F225EA0202C2630978C26901F06C
:10E5E8000F018C4022EA0402C261184AD3F80019CC
:10E5F8000A40C3F80029002030BDD3F8002B002AB8
:10E608000BDAD3F8002B42F00062C3F8002BD3F8E2
:10E61800002B42F08042C3F8002B0A780124C56B16
:10E6280002F00F0204FA02F225EA0242C2630978F4
:10E63800C26901F00F018C4022EA0442C261044A17
:10E64800D3F8001B0A40C3F8002BD4E7007833EC5A
:10E658000078F3EFF7B54B7891F800C0012B6D4DBA
:10E6680000EB4C146C4E40F089800F6904F5106380
:10E678003FBB1F693D401D611D6945F400251D61B3
:10E688001D693540012A1D614DD1CA6902B15A611F
:10E698000B79012B0CD1D0F8083813F4807FD4F80B
:10E6A80000390CBF43F0005343F08053C4F80039DD
:10E6B800D4F8003943F00443C4F80039002003B00B
:10E6C800F0BD1F693E401E611E6935401D610D6920
:10E6D8008E68BCF1000F0CD1B54288BF0E611D6970
:10E6E80045F400251D610D691E69C5F31205354302
:10E6F800C8E73544494FD3F810C0013DB5FBF6F5DE
:10E70800AEB207EAC54545EA0C051D610D79012D34
:10E71800E9D11D6925F0C0451D6175071F6905F020
:10E72800C0453D43DEE7D4F8003943F00443C4F85C
:10E7380000390B79012B0DD00B69002BBED00A785C
:10E748000123D0F8344802F00F0293402343C0F865
:10E758003438B3E7D0F8083813F4807FD4F8003998
:10E768000CBF43F0005343F08053C4F800390092C3
:10E778000B8A0A78C9683FF0DFFB9FE7D4F8107B63
:10E7880004F530633E401E611E6935401D610E6907
:10E798008D68BCF1000F27D106B10D610D621E69AD
:10E7A800C5F3120535431D611D6945F40025012A8D
:10E7B8001D6102D1CA6802B15A610B79012B0CD1D3
:10E7C800D0F8083813F4807FD4F8003B0CBF43F02E
:10E7D800005343F08053C4F8003BD4F8003B43F0A7
:10E7E8000443C4F8003B69E7002ED8D02E44013E0C
:10E7F800B6FBF5F6B6B275430D62084D1F6905EA1A
:10E80800C6453D431D610D6A1E69C5F312053543B2
:10E81800CDE700BFFFFF07E00000F8FF0000F81F8A
:10E8280030B5114C00F53063056CA54203D9D0F81A
:10E83800004B002C16DB002401291C611C6944F4E0
:10E8480000241C611C6944F018041C611C6944F014
:10E85800C0441C6106D15A61D0F8003B43F08023C4
:10E86800C0F8003B002030BD0A30544F00287FD04C
:10E87800414B9A6902F44042B2F5404F1BD13F4BDD
:10E888003F4A0344934258D33E4A3F4B02449A427C
:10E8980066D33E4A02449A4264D33D4A02449A42AD
:10E8A80062D33C4A02449A4260D33B4A02449A42A9
:10E8B8001ED2012342E09A6902F44042B2F5004FA9
:10E8C8001AD1364B364A0344934249D3354A364B1C
:10E8D80002449A4246D9354A02449A4244D9344AB3
:10E8E80002449A4242D9334A02449A42E1D9013356
:10E8F80098423DD8002321E09B6903F44043B3F5D7
:10E90800804F0FD12C4B2D4A034493422AD32C4AD3
:10E918002C4B02449A4227D92B4A02449A4225D9C1
:10E928002A4AE1E72A4A2B4B02449A421CD31A4A44
:10E9380002449A421AD3284AB8E7062327490A68A4
:10E9480022F00F021A430A600A6802F00F0293428B
:10E9580010D0086800F00F00C01A18BF01207047D7
:10E968000523EBE70423E9E70323E7E70223E5E7C9
:10E97800012070470020704700480258FFAD43F05F
:10E988000024F400FF10E3F200639F02FF7382F596
:10E99800FFD621F8FF39C1FAFF9C60FD7FA77BF302
:10E9A800C0E1E400FF85FCF57FDE80027F647DF82E
:10E9B800FF42FEFA7F217FFDFFCDE4F700366E01AE
:10E9C8007F9AEBF97FCC0602FF66F2FB7F33F9FDF5
:10E9D8007FEB10FC80B14F017F4EB0FE002000524B
:10E9E80070B50546C8B1047874B10D4C0D4EB442EB
:10E9F80001D3002408E02168A94207D120463FF04E
:10EA0800A0FB002808BF0024204670BD2846F1F767
:10EA18009FFD0028F2D01C34E9E70446F4E700BF64
:10EA28000C8606083889060810B50446F3F7AEFBCD
:10EA380003480121034A3AF031FD20463FF08CFBA0
:10EA4800B88B0608E98807082DE9F843044600AFA3
:10EA58000D46EFF31188102383F31288BFF36F8FED
:10EA680004282A4AE9468AB098BF294B9668117C3F
:10EA78006A4694BF53F82030264BCDE9073140F25F
:10EA880001332548ADF82430244BCDE9050442F87C
:10EA9800103F00234FF431512148F3F745FCCD4690
:10EAA80045B1EB69C3F3080323B11E4A01211C4891
:10EAB8003AF0F4FC2EB130463FF0FDFD08B1037882
:10EAC80003B91948E9468AB06A46184B0790CDE958
:10EAD800053640F20133ADF82030154B42F8103FAF
:10EAE80000234FF411510E48F3F71EFC2946204627
:10EAF800CD46FFF799FF88F31188BFF36F8F304633
:10EB0800F4F744FCBD46BDE8F88300BF243F002469
:10EB1800E4970608F98807080F8907080500000127
:10EB2800B88B06083789070807890708588907082E
:10EB38000400000138B50A4B53F82040013053F85F
:10EB48002050A54200D838BD606830B1037EDB078D
:10EB580001D43FF0DEFA0834F3E723689847FAE770
:10EB6800F897060870B52C4B01222C4C86B02C4D1A
:10EB78001A70AC421BD303202A4C2B4DFFF7DAFF47
:10EB88000420FFF7D7FF26463034AE4213D3254C76
:10EB980001F0D0F8AC422AD301F0E0F839F075FC66
:10EBA800224A938923F00103938106B070BD54F87B
:10EBB800043B9847DDE754F80C3C059354F8103CA7
:10EBC800049354F8143C039354F8183C029354F8F3
:10EBD8001C3C019354F8203C009354E90A2354E95F
:10EBE8000C01F1F72DFE54F8303C5E65CBE7D4E913
:10EBF8000A23B3F1FF3F08BFB2F1FF3F05D052EA45
:10EC08000301206803D100F075FD3034C2E70849DC
:10EC1800183001F0A3F9F8E7EA4C00243C8906080B
:10EC2800408906084089060870890608B03400241F
:10EC3800DDE7040870B5E023144E86B0012203FB1B
:10EC480000660023124D044601931249CDE90423BE
:10EC58000F2201EB4021CDE9023218234FF4C07294
:10EC680003FB00550C4B30460095F1F7E9FD337C6A
:10EC78000A4A23F00403EE602C7433744FF40863DB
:10EC880004FB033313446B6006B070BDD03300241B
:10EC9800243F0024806A0024F3E204080062002470
:10ECA8007FB50020FFF746FF2B4B83F308882B4CDA
:10ECB800F0232B4D84F822300023E3772376637604
:10ECC800A37684F82030636A43F4E0236362F4F7A0
:10ECD800C9F9F4F745FB4FF0FF33A362E362214C17
:10ECE800F4F746FDF4F788FCF3F7AEF91E4800F098
:10ECF800DDFCF3F757F8AC422AD301201B4CFFF791
:10ED080019FF0220FFF716FF002501F00BF8184B3A
:10ED18004FF4BE4217499C612046174B0095059356
:10ED28000123CDE90155CDE90353144BF1F788FDD3
:10ED3800237C0646204623F0040323743FF0F0FCAE
:10ED48002846FFF777FF0D4A31462046F4F7DCFAEC
:10ED580054F8043B9847CEE7806A002400ED00E0B1
:10ED68003C8906083889060890350024B034002408
:10ED7800243F0024806C0024336207086DEB0008F0
:10ED880038B5064C064DAC4201D3002038BDD4E955
:10ED98000112204614343FF029FAF4E7D81300246E
:10EDA800EC13002430B585B0044BDDE90845029327
:10EDB800CDE900453FF0D8F905B030BD9386040889
:10EDC80038B5064C064DAC4200D338BD20463FF05E
:10EDD80032FA0028F9D11C34F5E700BFBC1300242F
:10EDE800D813002473B50C46EFF31181102585F371
:10EDF8001288BFF36F8FC5685DB125602B68C3604B
:10EE0800836901338361002081F31188BFF36F8F19
:10EE180011E052EA030603D16FF00B002560F3E717
:10EE2800CDE900230246083000F088FE18B9034BEC
:10EE38009B685B69236002B070BD00BF243F00245B
:10EE4800F7B50E4604469DF82010EFF31187102001
:10EE580080F31288BFF36F8F256AE068854245D238
:10EE68002568AC4219D0C5B128463FF049FA05F1EA
:10EE7800180001F003F9A2683146686959F050F8A2
:10EE880000232846C5F8983000F0D4FC04F10800A7
:10EE9800394600F0DBFD002036E0A268D9B13146E2
:10EEA800E06959F03DF8E369A26813446269934246
:10EEB800E36101D12369E361236A102104F124008D
:10EEC800013323623FF0FDFD0028DFD187F311886D
:10EED800BFF36F8F18E0A06931462369984208BFD5
:10EEE8006069801AA06159F01BF8E5E752EA03014E
:10EEF8000CD0084904F1080089684E613946CDE90B
:10EF08000023224600F01AFE03B0F0BD6FF0220085
:10EF1800DCE700BF243F0024F7B504460846EFF3BA
:10EF28001186102181F31288BFF36F8F216A00299F
:10EF38003BD0A268A16958F0F3FFA369A2682568CD
:10EF4800134462699342A36104BF2369A361AC427D
:10EF5800236A03F1FF33236236D02846002D34D0CC
:10EF68003FF0CEF905F1180001F088F86969A26848
:10EF78000027E06958F0D4FFE369A26828461344E3
:10EF880062699342E36104BF2369E361236A013341
:10EF98002362C5F8987000F04DFC04F10800314672
:10EFA80000F054FD384603B0F0BD52EA030111D019
:10EFB8000A4989684861314604F10800CDE900230F
:10EFC800224600F0BBFDEEE7002086F31188BFF370
:10EFD8006F8FE8E76FF02200F7E700BF243F0024B7
:10EFE8002DE9F341044617461E46EFF31188102316
:10EFF80083F31288BFF36F8F304BC2689B6872B17E
:10F008008068984217D057EA060216D188F311880B
:10F01800BFF36F8F6FF00F0002B0BDE8F08193F976
:10F028000E1001322161C4E9023288F31188BFF35E
:10F038006F8F0020F0E72169F3E793F90E1090F93C
:10F048000E30994230DA9942A8BF19463FF0B0F91C
:10F058000546224641461A48CDE9007600F06EFD85
:10F068000028E6D0EFF31186102383F31288BFF34C
:10F078006F8FA068D0B1236821699C420AD04BB138
:10F0880093F90E309942A8BF19466FF07F03994251
:10F09800B8BF19463FF08CF940B13146084800F036
:10F0A800D5FC6FF00A00B7E70025D2E7002DF4D1B0
:10F0B80086F31188BFF36F8FF3E700BF243F002466
:10F0C800EB4C0024F8B583680546002B40D0234A52
:10F0D800926893423FD1C368012B03D9013BC360B7
:10F0E8000020F8BDEFF31187102383F31288BFF3D4
:10F0F8006F8F016980683FF05BF92C68A54207D1E2
:10F108000023C5E9023387F31188BFF36F8FE7E760
:10F11800002CF5D0002604F11800D4E90032136061
:10F128005A60237CA66023F00203C4E900662374B6
:10F1380000F0A4FFAC6094F90E3020462B61C4F8AF
:10F14800986000F077FB3946054800F07FFCC7E778
:10F158006FF01500C5E74FF0FF30C2E7243F0024E9
:10F16800EB4C002473B51546EFF31186102282F399
:10F178001288BFF36F8F0468B4B12368426823F024
:10F1880003039442036008BF436023689B0704D0CD
:10F19800656820463FF0C1FC2C4686F31188BFF312
:10F1A8006F8F204602B070BD55EA0302F5D000F11A
:10F1B800080231461046CDE9005300F0BFFC002894
:10F1C800EFD1024B9B685C69EBE700BF243F00244A
:10F1D80070B5EFF31186102383F31288BFF36F8F96
:10F1E8000468A0421CD0DCB1002504F11800D4E961
:10F1F800003213605A60237CA56023F00203C4E93F
:10F208000055237400F03AFF2046C4F89850656111
:10F2180000F010FB31460B48BDE8704000F016BC0A
:10F22800D0E90232022110309A4218BF013340F867
:10F23800083C3FF046FC0028ECD186F31188BFF368
:10F248006F8F70BDEB4C002413B5EFF311811024C0
:10F2580084F31288BFF36F8F846844B1013C8460E3
:10F2680081F31188BFF36F8F002002B010BD52EAFE
:10F27800030406D181F31188BFF36F8F6FF00F007D
:10F28800F3E7CDE900230246014800F057FCECE71C
:10F29800EB4C0024F8B50546EFF31187102383F3F0
:10F2A8001288BFF36F8F00262C68A5421AD0CCB104
:10F2B800002604F11800D4E9003213605A60237C58
:10F2C800A66023F00203C4E90066237400F0D6FEAA
:10F2D8006FF00A0366612046C4F89830012600F0F2
:10F2E800A9FAE1E70023022105F11000AB603FF025
:10F2F800E8FB28B926B987F31188BFF36F8FF8BDEB
:10F3080039460248BDE8F84000F0A0BBEB4C0024A9
:10F318002DE9F04F044685B0624E4FF0FF3A4FF0AA
:10F32800FF3BEFF31187102383F31288BFF36F8F2E
:10F33800D4F8E4505DBB022104F1FC003FF012F95F
:10F3480000287FD004F1F409D4F8F4504D4500F0BA
:10F358008680002D00F083804FF0000805F118002A
:10F36800D5E9003213605A602B7CC5F8088023F079
:10F378000203C5E900882B7400F080FE01232846AB
:10F38800C5F81480C5F8983000F054FADCE7D4F8D2
:10F39800E8202B689542C4F8E43008BFC4F8E83088
:10F3A800D4F8FC3043F00203C4F8FC30EB6823F0D7
:10F3B800040343F00103EB606B6887F31188BFF324
:10F3C8006F8F28469847EFF31187102383F312882D
:10F3D800BFF36F8FEB68D80623F001024AD4EA60C6
:10F3E800EB689A0717D523F002033068EB6090B1F9
:10F3F8000368002278B141688D4249D10368002A28
:10F4080040D172683360904200D17360002340F8A5
:10F41800083BFFF7DDFED4F8FC3023F00203C4F804
:10F42800FC30DB053CD4D4F8E430003B18BF0123A2
:10F4380087F31188BFF36F8F002B3FF472AF3FF053
:10F448005BF96EE7D4F8FC30D90608D5C4F8FC009F
:10F4580087F31188BFF36F8F05B0BDE8F08F0023E5
:10F4680004F1EC02394610480293CDE900AB00F0F4
:10F478008BFC56E723F01103EB6005F11000FFF752
:10F48800A7FEADE713607368984208BF7260BDE7D6
:10F4980002461BB1196818460B46ABE71946FAE74E
:10F4A8000023C5E74C3F0024EB4C0024F8B5C368A3
:10F4B80004460E469A07C3F3400541D45F0741D47A
:10F4C8000B680BB983680B60E368D80745BFA3686E
:10F4D800022501253360376857B31C4B9A68D7F863
:10F4E800E0309A421ED13FF0DDF880F00100C0B252
:10F4F800D7F8FC30D907C3F380021CD5F2B1F8B1B4
:10F5080000232360D7F8E83073B9C7E9394438468F
:10F518003FF052F8E36843F00403E3603368A36004
:10F528002846F8BD0020E3E71C60C7F8E840EEE78E
:10F538006FF0150506E06FF0120503E01B07DFD535
:10F548006FF00F0500233360EAE700BF243F002473
:10F55800014601483FF08AB890360024F0B50446C9
:10F56800002089B0C4E9390004F1EC000E9DC4E91B
:10F578003B0004F1F400C4E93D0055B328790028A4
:10F5880040F2011008BF0120C4F8FC0000204FF031
:10F59800FF364FF0FF370094CDE90330CDE9010085
:10F5A8000D4B2046CDE9066700F0C8F855B129682B
:10F5B80011B120463FF07CF86B791BB1A38943F069
:10F5C8000103A381204600F095F8C4F8E04009B093
:10F5D800F0BD0120D8E700BF19F3000837B5019046
:10F5E8000846EFF31184102181F31288BFF36F8F5F
:10F5F800C16811F01E0F17D153EA020508D101A9FD
:10F60800FFF754FF84F31188BFF36F8F03B030BD49
:10F6180041F00801103040F8041C01998161034948
:10F6280000F09CFC0120EDE70020EBE701E6040870
:10F6380001460148FFF7D2BF90360024F0B585B0E7
:10F648000C4617461D460190EFF31183102181F3F4
:10F658001288BFF36F8F03A9204603933EF08DFFF6
:10F6680055EA0703039E09D101A92046FFF71EFFAB
:10F6780086F31188BFF36F8F05B0F0BDE3683A4693
:10F68800064904F1100043F00803E360019BA362FC
:10F698002B4600F063FC0120EAE700BF01E60408FE
:10F6A80001460148FFF7CABF9036002401230374BE
:10F6B80083810023C0E92033C0F88C30014B986067
:10F6C800704700BF243F002408B500F069FA70B104
:10F6D800074B9B68DB7B53B9EFF31180102383F34F
:10F6E8001288BFF36F8FBDE8084000F0C5BA08BDA7
:10F6F800243F002438B50446EFF31185102383F323
:10F708001288BFF36F8F037C5B070FD5183000F0AA
:10F71800B5FC237C204623F00403237400F08AF808
:10F7280029460548BDE8384000F090B985F31188AE
:10F73800BFF36F8F38BD00BFEB4C0024F0B5002538
:10F7480087B004460595109D04950F9D03950E9D61
:10F7580002950D9D01950C9DDDE912760095F1F756
:10F768006FF8B6F1FF3F08BFB7F1FF3F05D056EA83
:10F77800070305D12046FFF7BDFF204607B0F0BDBF
:10F788003A46334604F11800014900F0E7FBF4E774
:10F79800DDE704080A4A6FF00A019368C3F8981075
:10F7A8000849C3F894004B6843F080534B6000232A
:10F7B80083F31188BFF36F8F9368D3F8980070476D
:10F7C800243F002400ED00E038B5184CA168206AF9
:10F7D8000B68814214BF1A46002249680B605960C1
:10F7E800A368216A2AB9124AC3E900210B6023627F
:10F7F8000AE092F90E5093F90E00854212DD516825
:10F80800C3E900210B605360E569094B9D4200D0B4
:10F8180005B9E568A3689D4202D028463FF0A7F8DD
:10F82800A56138BD8A42DED01268DBE7243F002498
:10F83800403F002470B590F91020037C002A2FDB8C
:10F84800D9062DD11A4C63F07F0322460374216A2E
:10F8580052F81C3F934207D1C0E90021086020629A
:10F868000FE09942F8D01B68002BF5D093F90E6091
:10F8780090F90E50AE42F4DD5968C0E900310860D5
:10F888005860E569954200D005B9E568A3681A7C17
:10F89800D20606D1DA897F2A03D9AA690AB9A361EF
:10F8A80070BDAB4202D028463FF061F8A561F7E78A
:10F8B800243F002438B590F910200146037C002A23
:10F8C80004DA03F07F0303743EF018FF0D4D2A4657
:10F8D800AB6852F81C4F944200D004B9EC688B42D4
:10F8E80007D01A7CD20604D1DA897F2A01D9A26905
:10F8F8002AB1A34202D020463FF039F82346AB6133
:10F9080038BD00BF243F0024002A2DE9F8430CBF6E
:10F918004FF010084FF00808027C04460D4618EA1C
:10F92800020F65D148EA0203D2090CD10374B8F179
:10F93800080F7ED1A36813B120463EF0E7FE04F11C
:10F94800180610270FE003F07F0303743EF0D6FE7D
:10F95800EDE785F31188BFF36F8FEFF3118587F318
:10F968001288BFF36F8F304600F088FB0B30F0D061
:10F9780004F15807A66DB74211D04FF0000976B1CF
:10F9880030463EF0C3FE06F11800C6F8989000F025
:10F9980075FB3046FFF74EFFA66DB742EFD1294BF6
:10F9A8009B689C4245D1EFF30587003F18BF0127AC
:10F9B800DFF890904B4653F81C6F9E4200D00EB96A
:10F9C800D9F80C60D9F80830B34202D030463EF07E
:10F9D800CEFFB8F1100FC9F8186009D0204639F0E9
:10F9E800D3FE204600F066FA17B11748FFF75EFE0F
:10F9F800144B9B68A3421ED1EFF30583DBB9A289A0
:10FA0800D20711D585F31188BFF36F8F83F311885F
:10FA1800BFF36F8F0423184602DFEFF3118510231D
:10FA280083F31288BFF36F8F2846BDE8F843FFF7CA
:10FA3800B1BE0027BCE785F31188BFF36F8FBDE81F
:10FA4800F88300BF243F00249035002449B9EFF320
:10FA5800058030B9054B9A699B689A4201D0FFF737
:10FA680099BE81F31188BFF36F8F7047243F00243C
:10FA780070B50F4D06462B4653F81C4F9C4200D0DC
:10FA880004B9EC68AB681A7CD20604D1DA897F2AFB
:10FA980001D9A2692AB1A34202D020463EF067FFED
:10FAA80023463146AB610348BDE87040FFF7CEBF3F
:10FAB800243F0024EB4C002470B5EFF3118610238B
:10FAC80083F31288BFF36F8F1A4CA168206A0B6802
:10FAD800814214BF1A46002249680B605960A36826
:10FAE800216A2AB9144AC3E900210B6023620AE09B
:10FAF80092F90E5093F90E00854216DD5168C3E95C
:10FB080000210B605360E5690B4B9D4200D005B99D
:10FB1800E568A3689D4202D028463EF028FF30469B
:10FB2800A561BDE87040FFF735BE8A42DAD0126899
:10FB3800D7E700BF243F0024403F0024F8B5DDE9A3
:10FB480006670C461146EFF305833BB1002383F3A8
:10FB58001188BFF36F8F0423184602DF0D4B0E4A3E
:10FB680098681060EFF31182102282F31288BFF3B5
:10FB78006F8F9D6828463EF0E2FD32463B4605F110
:10FB88001800064900F0EAF92046BDE8F840FFF7FA
:10FB980001BE00BF243F0024543F0024DDE70408D1
:10FBA800F8B50446EFF31187102383F31288BFF3E7
:10FBB8006F8F037C49B203F01F02002A0CBF012695
:10FBC800002635D103F07F032A4D03743EF096FDDD
:10FBD800037C2A46817363F07F03037452F81C3F49
:10FBE800286A934207D1C4E9002004602C620DE022
:10FBF8009842F8D01B68002BF5D093F90EC08C45BD
:10FC0800F6DD5968C4E900310C605C60EC69944227
:10FC180000D004B9EC68AB689C4202D020463EF0A4
:10FC2800A6FEAC6187F31188BFF36F8F3046F8BD2D
:10FC38009B071CD585683EF061FD81732B689D424A
:10FC480009D16B68C4E900531C606C60EAE76A6814
:10FC58009A42F6D01B68002BF3D093F90E208A4203
:10FC6800F5DD5A68C4E9003214605C60DAE7817334
:10FC7800D8E700BF243F0024034648B9EFF30582C4
:10FC880032B9064A91699268914201D0FFF782BD64
:10FC980083F31188BFF36F8F704700BF243F0024A0
:10FCA800F8B550EA010305460C4603D13EF024FDA1
:10FCB8000020F8BDEFF31187102383F31288BFF3F8
:10FCC8006F8F144E144BB0681860FFF7F3FDB068DF
:10FCD8002A4623461149183000F040F9B368044613
:10FCE8001A7CC3F8947042F004021A746FF00A0286
:10FCF800C3F898200A4A536843F08053536000239E
:10FD080083F31188BFF36F8F3EF038FE201A20EA84
:10FD1800E070CEE7243F0024543F0024DDE70408C8
:10FD280000ED00E0024B03F11C02C3E90722704713
:10FD3800243F0024EFF31181102383F31288BFF3CB
:10FD48006F8F054B9A68D37B013BD37381F311887E
:10FD5800BFF36F8F704700BF243F0024EFF311807B
:10FD6800102383F31288BFF36F8F034B9A68D37BFA
:10FD78000133D373FFF77CBE243F0024014B9868FE
:10FD8800704700BF243F0024D3B5DDE90667089C0F
:10FD9800CDE90067FFF7D2FE1CB1034B9B685B6996
:10FDA800236002B0D0BD00BF243F0024027C03467C
:10FDB80012F01F0210D10A4988420DD0094908687B
:10FDC80068B1D9897F2909D893F90E20064B1B6899
:10FDD8009A42B8BF0020704700207047104670470D
:10FDE800D033002484090024583F0024044B012206
:10FDF800C01A044BC0105843034B1A54704700BF35
:10FE080070360024ABAAAAAAEB4C0024F8B50B4B19
:10FE180004460B4D1E7C18230A4F03FB0655284643
:10FE280000F02CF934B1BB5D28460749E21AD31714
:10FE380000F094F80023BB55F8BD00BF243F002410
:10FE480070360024EB4C0024F5FD0008F8B5EFF3FC
:10FE58001187102383F31288BFF36F8F124E134B51
:10FE6800B5681868A84206D13EF081FD87F311886D
:10FE7800BFF36F8FF8BD00221A60337C0C4AD35C45
:10FE8800002BF3D02846FFF791FF04460028EDD059
:10FE98002B7CDB06EAD1FFF797FCB369AB42E5D1CF
:10FEA8002046FFF7B3FFE1E7243F0024543F002436
:10FEB800EB4C0024EFF31181102383F31288BFF376
:10FEC8006F8F0A4A536A834207D1DB6F536281F30B
:10FED8001188BFF36F8F70471346002BF7D0DA6F86
:10FEE8008242F9D1C26FDA67F1E700BF243F0024EC
:10FEF800024B1868984208BF002070478809002400
:10FF080008B502466FF00041FFF7F2FFC8B18A4218
:10FF180015D2D0E90230B0F1FF3F08BFB3F1FF3F7F
:10FF280003D16FF00040801A08BD8B4270F10000C9
:10FF380001DB0548F7E79A4201D2981AF4E7002056
:10FF4800F2E78A42EDD3EFE7FEFFFF7F024B186826
:10FF580008B1FBF76FBC704790090024B3F1FF3F6D
:10FF680008BFB2F1FF3F2DE9F84F04469A461546FF
:10FF780098467AD00161EFF31187102383F3128832
:10FF8800BFF36F8FBAF1000FDFF8E89023DBFFF7BC
:10FF9800DDFF374B06461A68003A18BF012245199B
:10FFA8004AF100035219D9E9005143F100035519E8
:10FFB80043EB01080121DFF8C090C4E90223FFF7F1
:10FFC80097FFD9F804A0D8B9C4E9009ACAF8004044
:10FFD800C9F8044026E0D9E900136FF00102521A6B
:10FFE8004FF0FF3161EB0303521B63EB0A03012A55
:08FFF80073F100014FF000015C
:020000040801F1
:10000000BCBF01220023DAE7D0E9022ED4E9023C8A
:1000100093427CEB0E0B23DAD21A6EEB0C03C0E991
:1000200002234368C4E900031C604460FFF764FFD7
:1000300084420DD1104B1B68013309D111B9FFF770
:1000400089FF06463046FFF75FFF0021FBF796FB6E
:1000500087F31188BFF36F8F28464146BDE8F88FBC
:100060009B1A6CEB0E025045C4E90232B0D0006816
:10007000ADE70025A846EFE7900900248836002464
:1000800088090024F8B50446EFF31186102383F3A2
:100090001288BFF36F8F026872B3FFF72DFF184B02
:1000A0005B689C4208D0D2E90231D4E90275DB19C1
:1000B00041EB0501C2E90231D4E900320025844256
:1000C00013605A60C4E900550ED000200D4A136831
:1000D00023F001018C4204BF43F00103136086F357
:1000E0001188BFF36F8FF8BDFFF734FFFFF70CFFE8
:1000F0002946FBF743FBE8E76FF01500E6E700BF92
:10010000880900245C3F0024EFF31182102383F35D
:100110001288BFF36F8F064B40F001001B681B1A5B
:100120005842584182F31188BFF36F8F704700BF68
:100130005C3F00242DE9F0470023344E344D0C463B
:10014000DFF8D490334F30602B60D6F80080B8F1E0
:10015000000F10D14FF0FF3340462B60FFF7D4FE65
:100160004146FBF70BFB84F31188BFF36F8FBDE8AB
:10017000F047FFF76FBEFFF7BFFE6FF0004330B1EF
:10018000D0E90212994272F10002B8BF0B46434512
:10019000194684BF434641464FEAE37C38B1826842
:1001A000B2EB030AC26862EB0C0EC0E902AED9F8EA
:1001B0000020A8EB01014FF0000A4FF01008D21800
:1001C000D9F80430316043EB0C03C9E90023FFF791
:1001D00093FE0028B9D0D0E902120A43B5D13860A5
:1001E000D0E900210A6051600269C0E900AA84F3E5
:1001F0001188BFF36F8F9047EFF3118488F3128853
:10020000BFF36F8FC7F800A0E1E700BF603F002495
:10021000900900245C3F00248836002410B5EFF3D9
:100220001184102383F31288BFF36F8FFFF792FEC0
:10023000054AD2E90031C01841F1000184F3118868
:10024000BFF36F8F10BD00BF883600242DE9F04149
:100250000446EFF31186102383F31288BFF36F8FE8
:1002600003682BB186F31188BFF36F8FBDE8F0816F
:10027000FFF74AFF07460028F4D1D4E90A586A1C60
:1002800048F10003022A73F1000324D33EF07EFB01
:10029000281848EB0101012871F1000142DB3EF012
:1002A00075FB6FF00203281848EB010183426FF0E1
:1002B00000438B413BDB3EF069FB6FF001022D18E0
:1002C00048EB0103521B4FF0FF3161EB03031A4966
:1002D0002046FFF747FE236B01332363236A63B194
:1002E00086F31188BFF36F8F20469847EFF311868E
:1002F000102383F31288BFF36F8F54F8185FA54261
:10030000B0D0002DAED028463EF043FA0023C5F809
:10031000983086F31188BFF36F8F2846BDE8F0410F
:100320003EF002BA6FF001024FF0FF33CFE73A46DA
:100330004FF00043CBE700BF4D020108B3F1FF3F90
:1003400008BFB2F1FF3FF8B5044616461D4618D067
:10035000EFF31187102383F31288BFF36F8FFFF73A
:1003600091FE20460749DDE90623C4E90A2300235C
:10037000324623632B46FFF7F5FD87F31188BFF361
:100380006F8FF8BD4D02010870B50546EFF311847B
:10039000102686F31288BFF36F8FFFF773FE20B12C
:1003A00084F31188BFF36F8F70BD6B6A63B184F300
:1003B0001188BFF36F8F6B6A28469847EFF311845B
:1003C00086F31288BFF36F8F05F118003EF01BFA19
:1003D0000028E5D03EF0A8F921460248BDE870406B
:1003E000FFF738BBEC4C0024034610B5EFF3118443
:1003F000102282F31288BFF36F8FC16001218160E8
:100400000068834205D184F31188BFF36F8F002009
:1004100010BDD0E9003213605A600023C0E90033F8
:100420003EF00DFB21460248FFF714FBEFE700BF4B
:10043000EC4C0024F8B507460C4616463EF036F95B
:1004400008B10020F8BD0E4B9B68D3F88C50002DEE
:10045000F7D0221DF5D2EFF31184102383F3128815
:10046000BFF36F8F47F004012846B04784F311882B
:10047000BFF36F8F0028E4D040F8045BE2E700BFD1
:10048000243F00240146024A0020FFF7D3BF00BFEB
:100490008D860408064B07B54FF44062009305496A
:1004A0004FF0FF330448FFF75DF803B05DF804FB3D
:1004B0001098060800CC002490360024F0B50446BD
:1004C0008BB03EF01DFD042C2BD0354D286818B1A3
:1004D00015F0CEFF00232B601CB3324B9C4220D082
:1004E00001AB0026214602A802932F4B01960393ED
:1004F00043F0D5FC01983146013015F099FF0246D2
:10050000286070B106AF0199384640F083FD274B53
:10051000214604A80593049743F0C1FC2A68019B77
:10052000D654234D03F084F93EF0D7FB45F097F8FD
:100530003EF0E5FC01F09AFD1E4B0022D5F8F0409C
:100540001A7084B120460DF029FE30B3A06805F082
:10055000F9FED5F8F040002CF4D1D5F8F0301C4667
:10056000DB68002BFBD1C5F8EC400025124C01F0F4
:1005700037FF15F0E9F90DF001FF206815F078FF5D
:1005800025600E4C206815F073FF25603EF004FBDB
:100590000BB0BDE8F0403EF0A1BBE468DBE700BF74
:1005A0004C4100249844002449EB04088D0F0508B1
:1005B00020440024EC4C0024A03F00249C3F002455
:1005C00070B5164B0022044600EB81059A60C3E922
:1005D000002226460434306840F09CFC022818D1E2
:1005E00030680F4C206098B10E483EF04EFD2068F8
:1005F0003EF016FB0C4802F0B1F901F07DFD074911
:1006000020683EF008FB0023236001F075FD012007
:1006100070BDAC42DDD10020E3E700BF683F00249D
:10062000983F002458CD070861F8070873B50646BF
:100630003EF054FB06F01AF915F0ECFD054615F0F6
:10064000F5FD044606F01AF9641B0025A4F5806048
:10065000244C06F019F901F009FD00F027FC6B4667
:100660004FF400622049304600953EF071FA1F4B6E
:1006700001461860009B194413F01CFB4FF4005214
:1006800001AB1B49304601953EF062FA194B014619
:100690001860019B19440DF053FD06F01FFF294619
:1006A000D4F8E80006F012FD1621D4F8E80041F075
:1006B000E1F86621D4F8E80041F0DCF840F6B651E4
:1006C000D4F8E80041F0D6F8294604F1D80006F045
:1006D000FDFC094804F0F0FC084B01221A7002B03E
:1006E00070BD00BF20440024C38907089C3F00243C
:1006F000DA890708A03F002419630708EC4C00249E
:1007000009282DE9F0410546A4B000F0878001F0EA
:10071000C7FC044640B1002D40F08380424BD3F823
:10072000F040003C18BF01242846FFF77FFF3EF051
:1007300001FC002C6CD002AC3C4F01F043FD4FF4A7
:1007400000712046002640F04AFC3C6001F0B0FCFD
:100750000121054600F180083EF0A0FB344B354AEC
:1007600006AC3549354841F0A9FD06A800F00AFB62
:100770003349324841F0C7FD013614F8012B3149A5
:100780002E4841F0C0FD202EF6D12F492B4841F0D4
:1007900095FD44F065FF02212C48FFF711FF00236F
:1007A0003B6001F015FD0123294A0EA9404645F0A2
:1007B000DDFEA0B9029844F030F9039A04460146E0
:1007C00001AB01320EA845F0F3FF40B9039A019B3B
:1007D0009A4204D12146049857F0D5FBA0B14FF4BA
:1007E0007A703EF0D6FB0A23194A0EA9404645F01E
:1007F000BDFE01AB0EA8DDE9032146F08DF80EA881
:1008000046F0F6F901F032FC002128463EF046FBA6
:10081000104C6068FFF752FE0023636024B0BDE80F
:10082000F081002480E700BF20440024643F0024BE
:10083000F4890708058A07085D8A070874D6060840
:10084000AFEF07084DF80708289407084C980608EA
:100850006D8A0708683F00242DE9F04F804689B073
:10086000AA4E002841D00024202725463368012BBA
:1008700000F0B480B8F1000F40F0B48001264FF4CE
:10088000405301933EF081FB0390002C40F05E81C9
:100890004FF4C87BA1460BFB06F3012603F59C5AD7
:1008A00004930AF1080A01F069FD01F01DFD0546F7
:1008B0000290002800F0998047F0100701F0C8FC72
:1008C000934E306828B103781F4002D115F0D0FD57
:1008D0003760B9F1000F04D0002001F08BFF01F068
:1008E00083FF284609B0BDE8F08F01F0BFFB01F09F
:1008F00019FD05460028B6D1854FFFF797FE3EF05B
:1009000020FB3B68002B56D01A7822F020021A7088
:100910003B689A681C78127892B1586808B104F064
:10092000CBFB3B68012107A89B680793FFF748FEB4
:1009300098B93B6898683EF0A8FB764802F00EF83C
:1009400004217548FFF73CFE38B908217348FFF7CA
:1009500037FE10B1724802F001F8336818052CD543
:1009600000F0B8FF012828D16E4801F0F7FF4FF0E2
:1009700000096D4B706883F80090FFF79FFD3A689F
:10098000C6F804902AB11378990644BF43F02003B7
:10099000137033681A0512D500F09CFF441E4FF007
:1009A000300718BF0124336803F48073002B0CBF99
:1009B000254601245AE72C46C2E75C48D5E71BB917
:1009C00004F001042427EEE714F002044FF0280796
:1009D0001CBF83F48063C3F38024E4E702264FF452
:1009E00040134EE70326524B4BE73EF027FB0590A2
:1009F00080B13EF042FB68B101F094FC054648B975
:100A00003EF029FB04287FF45BAF032000F068FF71
:100A1000059D55E71CBB3EF011FB08B301F082FCBD
:100A2000F0B944483EF0FCF801F03AFC00283FD011
:100A3000414801F093FFB8F1000F02D03F4801F0A8
:100A40008DFF404601F0D4FD3D483EF01EFB3D4881
:100A500001F084FFB8F1000F01D044F000FE012442
:100A60003EF0ECFA2040C4B22EB101F05BFC10B9AC
:100A700003F04CFC06463EF088FA039B049A0546B8
:100A8000C31A9A4223D9B3FBFBF20BFB1235632D39
:100A900010D9B9F1000F04D0002001F0ABFE01F035
:100AA000A3FEC5F5C87066B3B04228BF304628E043
:100AB0002548BEE7B9F1000F04D101F0B5FE019859
:100AC00001F098FE0123C5F164000293EBE79A451B
:100AD00006D23EF05AFACDE90290DDF80890E2E63F
:100AE000B9F1000F04D0002001F084FE01F07CFE7B
:100AF000039B5344581B16B1B04228BF3046002810
:100B0000EBD015F0B7FB15F0FFFBE6E7683F0024DC
:100B10004841002467F807083C9806081C98060816
:100B2000D4EE070843EE0708EC4C00245DEE0708FE
:100B30000030300058CD070837F60708D4F0070812
:100B40008E8B07084CF1070863F607084FF0000981
:100B5000B6E600BF114B07B5186820B103B05DF8C9
:100B600004EB3EF092BA0E4B1A68012A0FD19A6834
:100B7000002A0CDD596851B109680C330948C9884D
:100B80000091094941F09AFB03B05DF804FB074866
:100B900003B05DF804EB01F0E1BE00BF983F002414
:100BA000683F002474D606087B8A0708DFF407082C
:100BB000F7B515F013FB01F059FC3DF0EDFF15F012
:100BC000C5FB3EF083FA01F0C9FD50483EF028F81D
:100BD0003EF0B9F901F006FB01F042FCB0FA80F0FA
:100BE0000021400901F074F910B9082001F03EFC21
:100BF00001F036FC18B901F03FFC01F037FC44F07D
:100C00002EFD3EF07CF900F0C1FE02F05DFF3F4892
:100C10003EF006F8002000F063FE01F021FC08B968
:100C200001F01CFB0120012501F034FA012001F044
:100C30002BFA4FF4807401F013FC354EFFF760FD82
:100C40003EF04DF8012001F04BFA284614F41067ED
:100C500054D015B92F4801F081FE3578002D3ED1D2
:100C600001F0FEFBFFF7F8FD0028EFD101F0F8FBE3
:100C7000044601F0FBF92046FFF7D8FC3EF061F98D
:100C8000012001F0FDFA01F0EBFB28B9224B012114
:100C900001A80193FFF794FC01F0C6FD1F4801F085
:100CA000A9FD01F0A1FD3378012B1AD101F08AFAD8
:100CB00000F0A0FC044601F08BFA0420FFF7FEFBD5
:100CC00001F0B2FD002001F095FD01F08DFD012045
:100CD00001F0DEFA032000F003FE0020B6E7002555
:100CE000C4E70F4B0F4F3B6001F006FA00F008FD20
:100CF000002304463B6001F0FFF9DEE7002CB3D08F
:100D000040F018FF384603B0F0BD00BF58CD0708CB
:100D1000ED4C00245AE20708848A0708303030007E
:100D20008C8A0708983F002408B50DF047FA00F0B8
:100D300023FB0421074841F03AFD3EF0F6F801F0AC
:100D400083FB02F0FBFD04F0B7FEBDE808400DF0A8
:100D500049BA00BF10450024014B1878704700BF06
:100D6000EC4C00249FED010A704700BF000000001A
:100D7000004870470076B0109FED010A704700BF31
:100D80003333534038B505462021F9F74DFA041E98
:100D900011DA21460024094837F05FFF214620225E
:100DA000074837F05AFFC4F1200228190021BDE896
:100DB000384057F0E0B81F2CF0DD38BD1C8B070819
:100DC000368B07080428034607B506D801460E48A7
:100DD00003B05DF804EB01F053BD0C4A06216846F0
:100DE00033F0CCFB052801DD38F0F9FC00F10803F5
:100DF0004422411C68466B4403F8082C01F040FD76
:100E000003B05DF804FB00BF5D8B0708628B070829
:100E1000F8B5244DAB7DDB0731D52E68706801280D
:100E20002DD9B168431ECA5C0A2A28D14A1E002B5C
:100E300001DC1A4608E0D45C0A2CFAD0013BF6E744
:100E40008C5C202C02D101329042F9D8002B0CDDB1
:100E5000541CA04209D15C1E0C448C4205D014F8ED
:100E6000017D0A2F0BD0202FF7D00144D21A11F8A0
:100E7000023C94083A2B00D10134013C00D2F8BD69
:100E800004220949304640F081F80421064801F067
:100E9000F7FC2B6904332B61AB7D43F00203AB7588
:100EA000EBE700BFA43F002412CC0708202200215A
:100EB000014857F060B800BFD844002438B500227C
:100EC0000B4C05460846A2606B6862754FF0FF3216
:100ED00063602560A161C4E903233DF0A1FE6B6856
:100EE0000BB90123A375BDE83840FFF791BF00BFE0
:100EF000A43F0024F8B503780446DBB10E4FD7F8C1
:100F0000B80018B12146EFF727FB98B12046EFF75C
:100F100035FB461C304643F083FD054650B1324652
:100F2000214657F001F805491C22081D57F00AF820
:100F3000C7F8B850F8BD00BF20440024D8440024AE
:100F40002DE9F347A24C06462368D3E9011040F08F
:100F5000B8FBA5688146042D00F20A82DFE815F08F
:100F6000050027013001CA010302731E042B15D8A6
:100F7000D4E900325B689A4200F08180012E0FD1E3
:100F8000236865689868266981192844761B0025BE
:100F90003DF029FE0746A846A56067E10D2E11DC4D
:100FA000022E13DDF31E0A2B10D8DFE813F06800C1
:100FB0000F00BD010F000F006F000F000F000F00AA
:100FC00024005D001B2E5ED07F2E5FD0A37D9A078C
:100FD00040F19680092E00F08A80202E40F0BE80DD
:100FE0004FF00008032120682F4684F8168003265E
:100FF00040F0BCF86CE077483DF012FEA0693DF08F
:101000000FFE2268636821699068C91A184401F0CC
:1010100037FC00252368D3E9011040F052FB484516
:1010200003D203216C4801F02BFC23682769D3F815
:101030000880D3F80490781908EB090140443DF08A
:10104000D2FDA9EB0701064608EB070001F018FCEA
:10105000236822695B689B1A5B1B981BFFF7B2FE33
:1010600023692B44236144E05C482E463DF0D8FDC3
:10107000206840F004F863681844FFF73BFF3046EF
:1010800002B0BDE8F0870123A36032E02669626800
:1010900096422ED92068B11A2B46D0F808C08B4250
:1010A00003EB02071BD1042BB4BF01270427F71B56
:1010B0003B461CF803201946013B02F0C002802A7F
:1010C000F7D0761A4FF001087F1A324640F055F8F3
:1010D000F01BFFF777FE23699B1B2361C9E01CF817
:1010E0000770202F01D10133D9E70127DFE7002363
:1010F000A375A37D4FF0FF3623F00203A375BEE76F
:10110000092E2BD123685A68C2B19B682269134407
:1011100013F8010C05F0BEFB80B1314B042601939E
:101120000025019B21695A1C206829440135019240
:101130001A7840F00FF8B542F3D16BE72368606886
:101140009D6801AB2169274A091A284409F0D8FD96
:1011500006460028CDD0431CE2D14FE71F2EC8DD44
:1011600006F0C00320682769802B0BBF8368F3B2A9
:10117000217D002104BFDB5D013103F1400208BF86
:10118000C9B2D2B221753944372A32469BBFDB0837
:10119000E525002503F006039CBF1D4105F003056E
:1011A0003FF0DEFF237DAB42A3D1013532E74F2E66
:1011B00004D05B2E40F0DC80022365E7042363E764
:1011C000A6F13003092B0FD803236675A36090E7BF
:1011D000A43F0024678B0708708B07088E8B0708D5
:1011E00012CC070874D606080023413EA360072EE0
:1011F0003FF67FAF01A353F826F000BF1D12010890
:101200007D120108BD120108E1120108F310010866
:1012100029130108F3100108810F0108E368062B68
:101220003FF767AF03F1010A524D2D3305EB8305FC
:10123000AB68002B3FF45DAF2668D4F80480B0683B
:101240002169014440443DF0CEFCC6F804800746C5
:10125000A9683046C4F80CA03FF06FFF22684FF039
:101260000108636826695568F61AED1A002E3FF7E3
:101270002FAFB8F1000F7FF4CDAE26E0E568002D6A
:10128000FFF637AF2668013DD4F80480B0682169C5
:10129000014440443DF0A7FC716807463046A1EB8D
:1012A0000801E5603FF062FFE268002AD6DB314BBF
:1012B000206803EB8203D3F8B810CDE723682569D3
:1012C0005B689D422CBF00250125002D7FF711AFE3
:1012D0002368294698682369184401F0D1FABFE6CB
:1012E000226963689A427FF604AF00250126A8466A
:1012F0002F46EDE67E2E3BD1637D313B072B37D861
:1013000001A252F823F000BF810F010871130108F8
:10131000371301082913010871130108711301081B
:10132000810F01082913010823685D682369ED1AFC
:101330000023A360C9E7206821694368994217D256
:1013400085685B1A01220D4415F8016F06F0C0068E
:10135000802E01D19A4204D13FF00FFF0023A360F9
:1013600057E60132F0E7462EDED0482E3FF408AEB5
:10137000002389E6204400242DE9F04F0B4B8BB06D
:1013800019686846CDF820C0091ACDF824D089081C
:10139000CDE90045CDE90267CDE90489CDE906AB89
:1013A00041F005FA0BB0BDE8F08F00BF20440024E7
:1013B00070B5067804461EB14FF0FF35284670BD63
:1013C0003DF087FEC31E0546012B0CD801210C48B9
:1013D000217001F055FA032DEED10A48836E60307A
:1013E0009E600EF047FFA388013B9BB2A380002BB9
:1013F000E4D10121044801F043FA6388A380DDE7CA
:10140000748B070820440024928B07082DE9F043D1
:1014100097B017461D460023044603A80493884648
:1014200007F001060EF00CFF0346002877D1F906FD
:1014300065D5DC20D4E9012142F0DDFB0446B8F19A
:10144000010FD4F8009007D14FEA091140F225307E
:1014500041F0060106F0AAF82146424601A811F023
:10146000E1FEC7F38002494601A80EF033FDB8F152
:10147000010F044601D1FFF757FC380602D40320C0
:1014800000F0E6F914B1204640F08DFB4FF0FF303C
:1014900000F0DEF9012005F083FF12F0E3F81EB141
:1014A0000121454801F0ECF90024FDB12C60ECB1BC
:1014B000049F4FF0FF3338466F60AB6040F0E3FDB0
:1014C000A0B101AA6946384640F00CFE019B6BB101
:1014D0005A68AA60002285F82C20186844F060F849
:1014E0002022014605F10C0056F07CFD1EB10121C1
:1014F000314801F0C5F9204617B0BDE8F0837A06FF
:1015000005D5DC2094E80E0042F02DFB96E7BB06E3
:1015100095D5204644F024F842F07BFB8EE74FF04F
:10152000FF3000F095F9022005F03AFF790602D568
:10153000A368206898471EB101211F4801F0A0F957
:10154000049C20460FF024FE1C4914F023F9F0B14E
:10155000049840F0ADFD0E2817D0C20705D48307CC
:1015600008D10268164B9A4204D143F0E8F940F4DE
:1015700080749AE70146002212480FF025FE1249B6
:10158000104840F019FE0120F1E70020EFE70F4B73
:101590009C420DD004990B4842F081FC049B0C49FD
:1015A000186814F0F7F8002814BF822401247CE79F
:1015B0004FF4006479E700BF748B0708ACD50608C8
:1015C000C8D0060874D60608289407089844002452
:1015D00088D5060808B503784BB901210170044885
:1015E00001F04EF93DF075FD03380128FAD808BD29
:1015F000748B0708F0B58BB00025202106A83FF0BA
:10160000EEFC36483DF00CFB079535483DF008FBF5
:101610003DF05FFD431E032B43D8DFE803F00235A6
:101620003F4707990229ECD1089B1A78052AE8D18F
:101630005F78412F05D02B4801F022F90023079352
:10164000E3E780240126284801F01AF903216846BF
:10165000ADF800408DF8026001F012F901AA0023F4
:10166000314603A80392214A8DF804300492204A9F
:10167000ADF8064005923A46ADF80840FFF7C6FEC1
:10168000C305DBD50BB0F0BD1A483DF0C9FA06A87A
:101690003FF0C7FC0020184B1870F3E700230793B6
:1016A000B6E7C1B206A83FF0F9FCB1E713483DF038
:1016B000B7FA079B43B90F483DF0B2FA06A83FF0CE
:1016C000B0FC4FF48070DDE700231122012106A851
:1016D000FFF79CFE10F4106F96D0D3E7768B0708C7
:1016E0006F940708A08C0608918B0708B1130108B6
:1016F000D51501088E8B0708ED4C0024948B070844
:1017000070B598B0494E202101A83FF068FC4848C8
:101710003DF086FA47483DF083FA45483DF080FAAF
:10172000B28A002302B1B38205A8029306930EF099
:1017300087FD044688B9404901A83DF062FA0128B6
:1017400005462BD13A483DF06BFA01A83FF069FC01
:101750003A4B20461D7018B070BD022005F020FEE7
:1017600033483DF05DFA0699354842F098FB029BFC
:10177000002BD5D001A83FF082FC09F003FA58B144
:101780000A2101A83FF08AFC2E4901A83DF039FA50
:101790000328C2D00428EDD100212CE0851E032DA2
:1017A000E5D801A353F825F0B91701081B17010864
:1017B000C1170108D31701081D483DF031FAA6E70B
:1017C0001B483DF02DFA01A83FF02BFC4FF4807030
:1017D000C1E71D483DF024FA002302933DF079FC57
:1017E000C1B203298DF8031097D004290CD11048F9
:1017F0003DF016FA01210023162201A8FFF706FE8C
:1018000010F4106F8CD0A6E701A83FF047FC9DF8BC
:1018100003300D2B03D10D483DF002FADEE7012124
:101820000DF1030001F02CF8D8E700BF204400249C
:101830008E8B0708058A0708978B0708ED4C002454
:1018400074D60608D38B07089C8B0708CC8B070837
:10185000014B1860704700BF94090024024B986A3E
:10186000003818BF01207047204400242DE9F041C2
:1018700006460D4600270DB9BDE8F08133780A2BE6
:1018800015D1A7B9012401210C4800F0F9FF331943
:10189000A542984604D013F8012B57B90A2A08D15B
:1018A000304621462D1B464600F0EAFFE3E70024C0
:1018B000EDE70D3A013457425741E9E7D88B070865
:1018C000024B0348197840F05BBA00BFEE4C00248D
:1018D00024C10608014B1878704700BFEE4C002465
:1018E000014B1870704700BFEE4C002410B5054C3A
:1018F00020680E2804D10449044801F0B5FB20609B
:1019000010BD00BF98090024C8880608C03F002405
:1019100010B5054C20680E2804D10449044801F094
:10192000C5FB206010BD00BF9C090024E4880608A8
:10193000E03F002410B5064C20680E2806D1054B68
:1019400080220549054801F009FB206010BD00BF59
:10195000A0090024EF4C00243C880608903700249E
:1019600010B5064C20680E2806D1054B802205498B
:10197000054801F0F3FA206010BD00BFA40900245F
:101980006F4D002420880608E037002470B502F06F
:1019900015F8044698B10A4B03600A48FDF724F88D
:1019A000054660B13CF0D1FB48B1074B29462046C3
:1019B000002223600123BDE8704004F0CBBB70BD62
:1019C00038C706086C7C070874C506086FF0130357
:1019D00002460B41DB0710B50C4615D50B490C48E8
:1019E00040F091FC022C03D0052C0BD0094900E0FB
:1019F0000949074840F087FC08490548BDE8104000
:101A000040F05CBC0649F4E710BD00BF6FF6070864
:101A100074D6060899F307084DF3070828940708B9
:101A200058F307082DE9F04F99B081460C469046CF
:101A300000AF00F03DFB28B9012528466437BD46BC
:101A4000BDE8F08F01239F4A07F10801803044F080
:101A50008DFD0028F0D1D7E91002D7E906139A428C
:101A600008BF884200F02C8197F83930002B40F0F5
:101A7000278107F108003DF048F95B28064606D1AA
:101A800007F10800D7E9062345F0ABF9E3E7002E9C
:101A9000F6D009F1FF3A1AF8015F2DBB304604F089
:101AA000F9FE20B107F108003DF02FF906463D2E62
:101AB0001CD107F108003DF028F922280CBF0123B2
:101AC000002388F8003040F0CB8007F108003DF09B
:101AD0000DF9222829D016D828B30A2823D0C1B25C
:101AE00020463DF02AF9F0E7B54206D00A2EB2D0E2
:101AF00007F108003DF018F9ADE707F108003DF0E7
:101B0000F5F80646C7E75C28E9D107F108003DF083
:101B1000EDF87628E3D861281CD80A2803D0552888
:101B200054D00028DBD1052509E007F108003DF07D
:101B3000ECF80A2803D0232807D00028F3D1EDB20F
:101B400007F1080045F054F877E707F108003DF089
:101B5000EBF8F4E7A0F16203142BC0D801A252F80D
:101B600023F000BF5D1C0108DF1A0108DF1A01081D
:101B7000DF1A0108C91B0108DF1A0108DF1A010872
:101B8000DF1A0108DF1A0108DF1A0108DF1A01084D
:101B9000DF1A0108BD1B0108DF1A0108DF1A01085E
:101BA000DF1A0108B91B0108DF1A0108C11B01086F
:101BB000411C0108C51B01080D2090E70A208EE793
:101BC00009208CE70B208AE70C2088E74FF00809F2
:101BD00009F108036E4623F00703ADEB030DEA4657
:101BE000E8460DEB090B07F108003DF07FF808F817
:101BF000010BD845F7D10023391D102250460AF8B1
